gplink-1.1.0
Copyright (c) 1998-2005 gputils project
Listing File Generated: 4-4-2018  14:53:46
 
 
Address  Value    Disassembly              Source
-------  -----    -----------              ------
                                           ;--------------------------------------------------------
                                           ; File Created by ChiponCC : aolisn inc.
                                           ; Version 3.0.4#6752 (Jul  6 2017 15:09:47) (MSVC)
                                           ; This file was generated Wed Apr 04 14:53:37 2018
                                           ;--------------------------------------------------------
                                           ; chipon port for the 16-bit core
                                           ;--------------------------------------------------------
                                           ;	.file	"../config_set.c"
                                           	.radix dec
                                           	.include "KF8S1024.inc"
                                           
                                           ;************************************************************ 
                                           ;       Header file for the KungFu8 
                                           ;       KF8S1024 
                                           ;       Microcontroller
                                           ; 
                                           ;       Copyright 2012-2013 ChipON, All rights reserved
                                           ;************************************************************ 
                                            
                                           T0                .EQU                0x01
                                           PCL               .EQU                0x02
                                           PSW               .EQU                0x03
                                           P0                .EQU                0x05
                                           P2                .EQU                0x06
                                           P1                .EQU                0x07
                                           P3                .EQU                0x08
                                           PCH               .EQU                0x0A
                                           INTCTL            .EQU                0x0B
                                           EIF1              .EQU                0x0C
                                           T1L               .EQU                0x0E
                                           T1H               .EQU                0x0F
                                           T1CTL             .EQU                0x10
                                           T2                .EQU                0x11
                                           T2CTL             .EQU                0x12
                                           PWMCTL            .EQU                0x15
                                           CMCTL1            .EQU                0x1A
                                           VRECAL            .EQU                0x1C
                                           ADCDATAH          .EQU                0x1E
                                           ADCCTL0           .EQU                0x1F
                                           OPTR              .EQU                0x21
                                           TR0               .EQU                0x25
                                           TR2               .EQU                0x26
                                           TR1               .EQU                0x27
                                           TR3               .EQU                0x28
                                           EIE1              .EQU                0x2C
                                           PCTL              .EQU                0x2E
                                           OSCCTL            .EQU                0x2F
                                           OSCCAL0           .EQU                0x30
                                           ANSEL             .EQU                0x31
                                           PUR               .EQU                0x35
                                           IOCL              .EQU                0x36
                                           OSCCAL1           .EQU                0x37
                                           ADCDATAL          .EQU                0x3E
                                           ADCCTL1           .EQU                0x3F
                                           T3L               .EQU                0x50
                                           CTCTL             .EQU                0x53
                                           T2CCR             .EQU                0x54
                                           OSCLDOCAL         .EQU                0x5E
                                           T1U               .EQU                0x5F
                                            
                                            
                                           
                                           ;Address:0x03 PSW Bits------------------
                                           RP0                .EQU                5
                                           TO                 .EQU                4
                                           PD                 .EQU                3
                                           Z                  .EQU                2
                                           DC                 .EQU                1
                                           CY                 .EQU                0
                                           _RP0               .EQU                5
                                           _TO                .EQU                4
                                           _PD                .EQU                3
                                           _Z                 .EQU                2
                                           _DC                .EQU                1
                                           _CY                .EQU                0
                                           
                                           ;Address:0x05 P0 Bits-------------------
                                           P05                .EQU                5
                                           P04                .EQU                4
                                           P03                .EQU                3
                                           P01                .EQU                1
                                           P00                .EQU                0
                                           _P05               .EQU                5
                                           _P04               .EQU                4
                                           _P03               .EQU                3
                                           _P01               .EQU                1
                                           _P00               .EQU                0
                                           
                                           ;Address:0x06 P2 Bits-------------------
                                           P21                .EQU                1
                                           P20                .EQU                0
                                           _P21               .EQU                1
                                           _P20               .EQU                0
                                           
                                           ;Address:0x07 P1 Bits-------------------
                                           P17                .EQU                7
                                           P16                .EQU                6
                                           P12                .EQU                2
                                           _P17               .EQU                7
                                           _P16               .EQU                6
                                           _P12               .EQU                2
                                           
                                           ;Address:0x08 P3 Bits-------------------
                                           P33                .EQU                3
                                           P32                .EQU                2
                                           P31                .EQU                1
                                           P30                .EQU                0
                                           _P33               .EQU                3
                                           _P32               .EQU                2
                                           _P31               .EQU                1
                                           _P30               .EQU                0
                                           
                                           ;Address:0x0B INTCTL Bits---------------
                                           AIE                .EQU                7
                                           PUIE               .EQU                6
                                           T0IE               .EQU                5
                                           P0IE               .EQU                3
                                           T0IF               .EQU                2
                                           P0IF               .EQU                0
                                           _AIE               .EQU                7
                                           _PUIE              .EQU                6
                                           _T0IE              .EQU                5
                                           _P0IE              .EQU                3
                                           _T0IF              .EQU                2
                                           _P0IF              .EQU                0
                                           
                                           ;Address:0x0C EIF1 Bits-----------------
                                           CTIF               .EQU                7
                                           ADIF               .EQU                6
                                           INT2IF             .EQU                5
                                           INT1IF             .EQU                4
                                           C1IF               .EQU                3
                                           PWM2IF             .EQU                2
                                           T2IF               .EQU                1
                                           T1IF               .EQU                0
                                           _CTIF              .EQU                7
                                           _ADIF              .EQU                6
                                           _INT2IF            .EQU                5
                                           _INT1IF            .EQU                4
                                           _C1IF              .EQU                3
                                           _PWM2IF            .EQU                2
                                           _T2IF              .EQU                1
                                           _T1IF              .EQU                0
                                           
                                           ;Address:0x10 T1CTL Bits----------------
                                           T1GC               .EQU                6
                                           T1CKS1             .EQU                5
                                           T1CKS0             .EQU                4
                                           T1SY               .EQU                2
                                           T1CS               .EQU                1
                                           T1ON               .EQU                0
                                           _T1GC              .EQU                6
                                           _T1CKS1            .EQU                5
                                           _T1CKS0            .EQU                4
                                           _T1SY              .EQU                2
                                           _T1CS              .EQU                1
                                           _T1ON              .EQU                0
                                           
                                           ;Address:0x12 T2CTL Bits----------------
                                           T2CKBS3            .EQU                6
                                           T2CKBS2            .EQU                5
                                           T2CKBS1            .EQU                4
                                           T2CKBS0            .EQU                3
                                           T2ON               .EQU                2
                                           T2CKPS1            .EQU                1
                                           T2CKPS0            .EQU                0
                                           _T2CKBS3           .EQU                6
                                           _T2CKBS2           .EQU                5
                                           _T2CKBS1           .EQU                4
                                           _T2CKBS0           .EQU                3
                                           _T2ON              .EQU                2
                                           _T2CKPS1           .EQU                1
                                           _T2CKPS0           .EQU                0
                                           
                                           ;Address:0x15 PWMCTL Bits---------------
                                           INT1SE             .EQU                6
                                           _INT1SE            .EQU                6
                                           
                                           ;Address:0x1A CMCTL1 Bits---------------
                                           CTCLKSEL1          .EQU                7
                                           CTCLKSEL0          .EQU                6
                                           CTVREFSEL1         .EQU                5
                                           CTVREFSEL0         .EQU                4
                                           _CTCLKSEL1         .EQU                7
                                           _CTCLKSEL0         .EQU                6
                                           _CTVREFSEL1        .EQU                5
                                           _CTVREFSEL0        .EQU                4
                                           
                                           ;Address:0x1F ADCCTL0 Bits--------------
                                           ADLR               .EQU                7
                                           CHS3               .EQU                5
                                           CHS2               .EQU                4
                                           CHS1               .EQU                3
                                           CHS0               .EQU                2
                                           START              .EQU                1
                                           ADEN               .EQU                0
                                           _ADLR              .EQU                7
                                           _CHS3              .EQU                5
                                           _CHS2              .EQU                4
                                           _CHS1              .EQU                3
                                           _CHS0              .EQU                2
                                           _START             .EQU                1
                                           _ADEN              .EQU                0
                                           
                                           ;Address:0x21 OPTR Bits-----------------
                                           PUPH               .EQU                7
                                           T0CS               .EQU                5
                                           T0SE               .EQU                4
                                           PSA                .EQU                3
                                           PS2                .EQU                2
                                           PS1                .EQU                1
                                           PS0                .EQU                0
                                           _PUPH              .EQU                7
                                           _T0CS              .EQU                5
                                           _T0SE              .EQU                4
                                           _PSA               .EQU                3
                                           _PS2               .EQU                2
                                           _PS1               .EQU                1
                                           _PS0               .EQU                0
                                           
                                           ;Address:0x25 TR0 Bits------------------
                                           TR05               .EQU                5
                                           TR04               .EQU                4
                                           TR03               .EQU                3
                                           TR01               .EQU                1
                                           TR00               .EQU                0
                                           _TR05              .EQU                5
                                           _TR04              .EQU                4
                                           _TR03              .EQU                3
                                           _TR01              .EQU                1
                                           _TR00              .EQU                0
                                           
                                           ;Address:0x26 TR2 Bits------------------
                                           TR21               .EQU                1
                                           TR20               .EQU                0
                                           _TR21              .EQU                1
                                           _TR20              .EQU                0
                                           
                                           ;Address:0x27 TR1 Bits------------------
                                           TR17               .EQU                7
                                           TR16               .EQU                6
                                           TR12               .EQU                2
                                           _TR17              .EQU                7
                                           _TR16              .EQU                6
                                           _TR12              .EQU                2
                                           
                                           ;Address:0x28 TR3 Bits------------------
                                           TR33               .EQU                3
                                           TR32               .EQU                2
                                           TR31               .EQU                1
                                           TR30               .EQU                0
                                           _TR33              .EQU                3
                                           _TR32              .EQU                2
                                           _TR31              .EQU                1
                                           _TR30              .EQU                0
                                           
                                           ;Address:0x2C EIE1 Bits-----------------
                                           CTIE               .EQU                7
                                           ADIE               .EQU                6
                                           INT2IE             .EQU                5
                                           INT1IE             .EQU                4
                                           C1IE               .EQU                3
                                           PWM2IE             .EQU                2
                                           T2IE               .EQU                1
                                           T1IE               .EQU                0
                                           _CTIE              .EQU                7
                                           _ADIE              .EQU                6
                                           _INT2IE            .EQU                5
                                           _INT1IE            .EQU                4
                                           _C1IE              .EQU                3
                                           _PWM2IE            .EQU                2
                                           _T2IE              .EQU                1
                                           _T1IE              .EQU                0
                                           
                                           ;Address:0x2E PCTL Bits-----------------
                                           VREEN              .EQU                7
                                           VREOE              .EQU                6
                                           SLVREN             .EQU                4
                                           POR                .EQU                1
                                           LVR                .EQU                0
                                           _VREEN             .EQU                7
                                           _VREOE             .EQU                6
                                           _SLVREN            .EQU                4
                                           _POR               .EQU                1
                                           _LVR               .EQU                0
                                           
                                           ;Address:0x2F OSCCTL Bits---------------
                                           CKOEN              .EQU                7
                                           IRCS2              .EQU                6
                                           IRCS1              .EQU                5
                                           IRCS0              .EQU                4
                                           _CKOEN             .EQU                7
                                           _IRCS2             .EQU                6
                                           _IRCS1             .EQU                5
                                           _IRCS0             .EQU                4
                                           
                                           ;Address:0x31 ANSEL Bits----------------
                                           ANS6               .EQU                6
                                           ANS3               .EQU                3
                                           ANS1               .EQU                1
                                           _ANS6              .EQU                6
                                           _ANS3              .EQU                3
                                           _ANS1              .EQU                1
                                           
                                           ;Address:0x35 PUR Bits------------------
                                           PUR5               .EQU                5
                                           PUR4               .EQU                4
                                           PUR2               .EQU                2
                                           PUR1               .EQU                1
                                           PUR0               .EQU                0
                                           _PUR5              .EQU                5
                                           _PUR4              .EQU                4
                                           _PUR2              .EQU                2
                                           _PUR1              .EQU                1
                                           _PUR0              .EQU                0
                                           
                                           ;Address:0x36 IOCL Bits-----------------
                                           IOCL5              .EQU                5
                                           IOCL4              .EQU                4
                                           IOCL3              .EQU                3
                                           IOCL2              .EQU                2
                                           IOCL1              .EQU                1
                                           IOCL0              .EQU                0
                                           _IOCL5             .EQU                5
                                           _IOCL4             .EQU                4
                                           _IOCL3             .EQU                3
                                           _IOCL2             .EQU                2
                                           _IOCL1             .EQU                1
                                           _IOCL0             .EQU                0
                                           
                                           ;Address:0x3F ADCCTL1 Bits--------------
                                           ADCS2              .EQU                6
                                           ADCS1              .EQU                5
                                           ADCS0              .EQU                4
                                           VCFG1              .EQU                3
                                           VCFG0              .EQU                2
                                           _ADCS2             .EQU                6
                                           _ADCS1             .EQU                5
                                           _ADCS0             .EQU                4
                                           _VCFG1             .EQU                3
                                           _VCFG0             .EQU                2
                                           
                                           ;Address:0x50 T3L Bits------------------
                                           T3L7               .EQU                7
                                           T3L6               .EQU                6
                                           T3L5               .EQU                5
                                           T3L4               .EQU                4
                                           T3L3               .EQU                3
                                           T3L2               .EQU                2
                                           T3L1               .EQU                1
                                           T3L0               .EQU                0
                                           _T3L7              .EQU                7
                                           _T3L6              .EQU                6
                                           _T3L5              .EQU                5
                                           _T3L4              .EQU                4
                                           _T3L3              .EQU                3
                                           _T3L2              .EQU                2
                                           _T3L1              .EQU                1
                                           _T3L0              .EQU                0
                                           
                                           ;Address:0x53 CTCTL Bits----------------
                                           CTEN               .EQU                7
                                           CTSTART            .EQU                6
                                           CTCAPS             .EQU                5
                                           CTCMS              .EQU                4
                                           CTCHSEL4           .EQU                4
                                           CTCHSEL3           .EQU                3
                                           CTCHSEL2           .EQU                2
                                           CTCHSEL1           .EQU                1
                                           CTCHSEL0           .EQU                0
                                           _CTEN              .EQU                7
                                           _CTSTART           .EQU                6
                                           _CTCAPS            .EQU                5
                                           _CTCMS             .EQU                4
                                           _CTCHSEL4          .EQU                4
                                           _CTCHSEL3          .EQU                3
                                           _CTCHSEL2          .EQU                2
                                           _CTCHSEL1          .EQU                1
                                           _CTCHSEL0          .EQU                0
                                           
                                           ;Address:0x5E OSCLDOCAL Bits------------
                                            
                                            
                                           ;--------------------------------------------------------
                                           ; config word(s)
                                           ;--------------------------------------------------------
                                           	__config 0x4c0
                                           ;--------------------------------------------------------
                                           ; external declarations
                                           ;--------------------------------------------------------
                                           
                                           	.extern STK12
                                           	.extern STK11
                                           	.extern STK10
                                           	.extern STK09
                                           	.extern STK08
                                           	.extern STK07
                                           	.extern STK06
                                           	.extern STK05
                                           	.extern STK04
                                           	.extern STK03
                                           	.extern STK02
                                           	.extern STK01
                                           	.extern STK00
                                           ;--------------------------------------------------------
                                           ; global declarations
                                           ;--------------------------------------------------------
                                           
                                           ;--------------------------------------------------------
                                           ; global definitions
                                           ;--------------------------------------------------------
                                           ;--------------------------------------------------------
                                           ; absolute symbol definitions
                                           ;--------------------------------------------------------
                                           ;--------------------------------------------------------
                                           ; compiler-defined variables
                                           ;--------------------------------------------------------
                                           ;--------------------------------------------------------
                                           ; initialized data
                                           ;--------------------------------------------------------
                                           ;--------------------------------------------------------
                                           ; overlayable items in internal ram 
                                           ;--------------------------------------------------------
                                           ;	.udata_ovr
                                           
                                           ;	code size estimation:
                                           ;	    0+    0 =     0 instructions (    0 byte)
                                           
                                           
                                           	.end
                                           ;--------------------------------------------------------
                                           ; File Created by ChiponCC : aolisn inc.
                                           ; Version 3.0.4#6752 (Jul  6 2017 15:09:47) (MSVC)
                                           ; This file was generated Wed Apr 04 14:53:39 2018
                                           ;--------------------------------------------------------
                                           ; chipon port for the 16-bit core
                                           ;--------------------------------------------------------
                                           ;	.file	"../debug_touch.c"
                                           	.radix dec
                                           	.include "KF8S1024.inc"
                                           
                                           ;************************************************************ 
                                           ;       Header file for the KungFu8 
                                           ;       KF8S1024 
                                           ;       Microcontroller
                                           ; 
                                           ;       Copyright 2012-2013 ChipON, All rights reserved
                                           ;************************************************************ 
                                            
                                           T0                .EQU                0x01
                                           PCL               .EQU                0x02
                                           PSW               .EQU                0x03
                                           P0                .EQU                0x05
                                           P2                .EQU                0x06
                                           P1                .EQU                0x07
                                           P3                .EQU                0x08
                                           PCH               .EQU                0x0A
                                           INTCTL            .EQU                0x0B
                                           EIF1              .EQU                0x0C
                                           T1L               .EQU                0x0E
                                           T1H               .EQU                0x0F
                                           T1CTL             .EQU                0x10
                                           T2                .EQU                0x11
                                           T2CTL             .EQU                0x12
                                           PWMCTL            .EQU                0x15
                                           CMCTL1            .EQU                0x1A
                                           VRECAL            .EQU                0x1C
                                           ADCDATAH          .EQU                0x1E
                                           ADCCTL0           .EQU                0x1F
                                           OPTR              .EQU                0x21
                                           TR0               .EQU                0x25
                                           TR2               .EQU                0x26
                                           TR1               .EQU                0x27
                                           TR3               .EQU                0x28
                                           EIE1              .EQU                0x2C
                                           PCTL              .EQU                0x2E
                                           OSCCTL            .EQU                0x2F
                                           OSCCAL0           .EQU                0x30
                                           ANSEL             .EQU                0x31
                                           PUR               .EQU                0x35
                                           IOCL              .EQU                0x36
                                           OSCCAL1           .EQU                0x37
                                           ADCDATAL          .EQU                0x3E
                                           ADCCTL1           .EQU                0x3F
                                           T3L               .EQU                0x50
                                           CTCTL             .EQU                0x53
                                           T2CCR             .EQU                0x54
                                           OSCLDOCAL         .EQU                0x5E
                                           T1U               .EQU                0x5F
                                            
                                            
                                           
                                           ;Address:0x03 PSW Bits------------------
                                           RP0                .EQU                5
                                           TO                 .EQU                4
                                           PD                 .EQU                3
                                           Z                  .EQU                2
                                           DC                 .EQU                1
                                           CY                 .EQU                0
                                           _RP0               .EQU                5
                                           _TO                .EQU                4
                                           _PD                .EQU                3
                                           _Z                 .EQU                2
                                           _DC                .EQU                1
                                           _CY                .EQU                0
                                           
                                           ;Address:0x05 P0 Bits-------------------
                                           P05                .EQU                5
                                           P04                .EQU                4
                                           P03                .EQU                3
                                           P01                .EQU                1
                                           P00                .EQU                0
                                           _P05               .EQU                5
                                           _P04               .EQU                4
                                           _P03               .EQU                3
                                           _P01               .EQU                1
                                           _P00               .EQU                0
                                           
                                           ;Address:0x06 P2 Bits-------------------
                                           P21                .EQU                1
                                           P20                .EQU                0
                                           _P21               .EQU                1
                                           _P20               .EQU                0
                                           
                                           ;Address:0x07 P1 Bits-------------------
                                           P17                .EQU                7
                                           P16                .EQU                6
                                           P12                .EQU                2
                                           _P17               .EQU                7
                                           _P16               .EQU                6
                                           _P12               .EQU                2
                                           
                                           ;Address:0x08 P3 Bits-------------------
                                           P33                .EQU                3
                                           P32                .EQU                2
                                           P31                .EQU                1
                                           P30                .EQU                0
                                           _P33               .EQU                3
                                           _P32               .EQU                2
                                           _P31               .EQU                1
                                           _P30               .EQU                0
                                           
                                           ;Address:0x0B INTCTL Bits---------------
                                           AIE                .EQU                7
                                           PUIE               .EQU                6
                                           T0IE               .EQU                5
                                           P0IE               .EQU                3
                                           T0IF               .EQU                2
                                           P0IF               .EQU                0
                                           _AIE               .EQU                7
                                           _PUIE              .EQU                6
                                           _T0IE              .EQU                5
                                           _P0IE              .EQU                3
                                           _T0IF              .EQU                2
                                           _P0IF              .EQU                0
                                           
                                           ;Address:0x0C EIF1 Bits-----------------
                                           CTIF               .EQU                7
                                           ADIF               .EQU                6
                                           INT2IF             .EQU                5
                                           INT1IF             .EQU                4
                                           C1IF               .EQU                3
                                           PWM2IF             .EQU                2
                                           T2IF               .EQU                1
                                           T1IF               .EQU                0
                                           _CTIF              .EQU                7
                                           _ADIF              .EQU                6
                                           _INT2IF            .EQU                5
                                           _INT1IF            .EQU                4
                                           _C1IF              .EQU                3
                                           _PWM2IF            .EQU                2
                                           _T2IF              .EQU                1
                                           _T1IF              .EQU                0
                                           
                                           ;Address:0x10 T1CTL Bits----------------
                                           T1GC               .EQU                6
                                           T1CKS1             .EQU                5
                                           T1CKS0             .EQU                4
                                           T1SY               .EQU                2
                                           T1CS               .EQU                1
                                           T1ON               .EQU                0
                                           _T1GC              .EQU                6
                                           _T1CKS1            .EQU                5
                                           _T1CKS0            .EQU                4
                                           _T1SY              .EQU                2
                                           _T1CS              .EQU                1
                                           _T1ON              .EQU                0
                                           
                                           ;Address:0x12 T2CTL Bits----------------
                                           T2CKBS3            .EQU                6
                                           T2CKBS2            .EQU                5
                                           T2CKBS1            .EQU                4
                                           T2CKBS0            .EQU                3
                                           T2ON               .EQU                2
                                           T2CKPS1            .EQU                1
                                           T2CKPS0            .EQU                0
                                           _T2CKBS3           .EQU                6
                                           _T2CKBS2           .EQU                5
                                           _T2CKBS1           .EQU                4
                                           _T2CKBS0           .EQU                3
                                           _T2ON              .EQU                2
                                           _T2CKPS1           .EQU                1
                                           _T2CKPS0           .EQU                0
                                           
                                           ;Address:0x15 PWMCTL Bits---------------
                                           INT1SE             .EQU                6
                                           _INT1SE            .EQU                6
                                           
                                           ;Address:0x1A CMCTL1 Bits---------------
                                           CTCLKSEL1          .EQU                7
                                           CTCLKSEL0          .EQU                6
                                           CTVREFSEL1         .EQU                5
                                           CTVREFSEL0         .EQU                4
                                           _CTCLKSEL1         .EQU                7
                                           _CTCLKSEL0         .EQU                6
                                           _CTVREFSEL1        .EQU                5
                                           _CTVREFSEL0        .EQU                4
                                           
                                           ;Address:0x1F ADCCTL0 Bits--------------
                                           ADLR               .EQU                7
                                           CHS3               .EQU                5
                                           CHS2               .EQU                4
                                           CHS1               .EQU                3
                                           CHS0               .EQU                2
                                           START              .EQU                1
                                           ADEN               .EQU                0
                                           _ADLR              .EQU                7
                                           _CHS3              .EQU                5
                                           _CHS2              .EQU                4
                                           _CHS1              .EQU                3
                                           _CHS0              .EQU                2
                                           _START             .EQU                1
                                           _ADEN              .EQU                0
                                           
                                           ;Address:0x21 OPTR Bits-----------------
                                           PUPH               .EQU                7
                                           T0CS               .EQU                5
                                           T0SE               .EQU                4
                                           PSA                .EQU                3
                                           PS2                .EQU                2
                                           PS1                .EQU                1
                                           PS0                .EQU                0
                                           _PUPH              .EQU                7
                                           _T0CS              .EQU                5
                                           _T0SE              .EQU                4
                                           _PSA               .EQU                3
                                           _PS2               .EQU                2
                                           _PS1               .EQU                1
                                           _PS0               .EQU                0
                                           
                                           ;Address:0x25 TR0 Bits------------------
                                           TR05               .EQU                5
                                           TR04               .EQU                4
                                           TR03               .EQU                3
                                           TR01               .EQU                1
                                           TR00               .EQU                0
                                           _TR05              .EQU                5
                                           _TR04              .EQU                4
                                           _TR03              .EQU                3
                                           _TR01              .EQU                1
                                           _TR00              .EQU                0
                                           
                                           ;Address:0x26 TR2 Bits------------------
                                           TR21               .EQU                1
                                           TR20               .EQU                0
                                           _TR21              .EQU                1
                                           _TR20              .EQU                0
                                           
                                           ;Address:0x27 TR1 Bits------------------
                                           TR17               .EQU                7
                                           TR16               .EQU                6
                                           TR12               .EQU                2
                                           _TR17              .EQU                7
                                           _TR16              .EQU                6
                                           _TR12              .EQU                2
                                           
                                           ;Address:0x28 TR3 Bits------------------
                                           TR33               .EQU                3
                                           TR32               .EQU                2
                                           TR31               .EQU                1
                                           TR30               .EQU                0
                                           _TR33              .EQU                3
                                           _TR32              .EQU                2
                                           _TR31              .EQU                1
                                           _TR30              .EQU                0
                                           
                                           ;Address:0x2C EIE1 Bits-----------------
                                           CTIE               .EQU                7
                                           ADIE               .EQU                6
                                           INT2IE             .EQU                5
                                           INT1IE             .EQU                4
                                           C1IE               .EQU                3
                                           PWM2IE             .EQU                2
                                           T2IE               .EQU                1
                                           T1IE               .EQU                0
                                           _CTIE              .EQU                7
                                           _ADIE              .EQU                6
                                           _INT2IE            .EQU                5
                                           _INT1IE            .EQU                4
                                           _C1IE              .EQU                3
                                           _PWM2IE            .EQU                2
                                           _T2IE              .EQU                1
                                           _T1IE              .EQU                0
                                           
                                           ;Address:0x2E PCTL Bits-----------------
                                           VREEN              .EQU                7
                                           VREOE              .EQU                6
                                           SLVREN             .EQU                4
                                           POR                .EQU                1
                                           LVR                .EQU                0
                                           _VREEN             .EQU                7
                                           _VREOE             .EQU                6
                                           _SLVREN            .EQU                4
                                           _POR               .EQU                1
                                           _LVR               .EQU                0
                                           
                                           ;Address:0x2F OSCCTL Bits---------------
                                           CKOEN              .EQU                7
                                           IRCS2              .EQU                6
                                           IRCS1              .EQU                5
                                           IRCS0              .EQU                4
                                           _CKOEN             .EQU                7
                                           _IRCS2             .EQU                6
                                           _IRCS1             .EQU                5
                                           _IRCS0             .EQU                4
                                           
                                           ;Address:0x31 ANSEL Bits----------------
                                           ANS6               .EQU                6
                                           ANS3               .EQU                3
                                           ANS1               .EQU                1
                                           _ANS6              .EQU                6
                                           _ANS3              .EQU                3
                                           _ANS1              .EQU                1
                                           
                                           ;Address:0x35 PUR Bits------------------
                                           PUR5               .EQU                5
                                           PUR4               .EQU                4
                                           PUR2               .EQU                2
                                           PUR1               .EQU                1
                                           PUR0               .EQU                0
                                           _PUR5              .EQU                5
                                           _PUR4              .EQU                4
                                           _PUR2              .EQU                2
                                           _PUR1              .EQU                1
                                           _PUR0              .EQU                0
                                           
                                           ;Address:0x36 IOCL Bits-----------------
                                           IOCL5              .EQU                5
                                           IOCL4              .EQU                4
                                           IOCL3              .EQU                3
                                           IOCL2              .EQU                2
                                           IOCL1              .EQU                1
                                           IOCL0              .EQU                0
                                           _IOCL5             .EQU                5
                                           _IOCL4             .EQU                4
                                           _IOCL3             .EQU                3
                                           _IOCL2             .EQU                2
                                           _IOCL1             .EQU                1
                                           _IOCL0             .EQU                0
                                           
                                           ;Address:0x3F ADCCTL1 Bits--------------
                                           ADCS2              .EQU                6
                                           ADCS1              .EQU                5
                                           ADCS0              .EQU                4
                                           VCFG1              .EQU                3
                                           VCFG0              .EQU                2
                                           _ADCS2             .EQU                6
                                           _ADCS1             .EQU                5
                                           _ADCS0             .EQU                4
                                           _VCFG1             .EQU                3
                                           _VCFG0             .EQU                2
                                           
                                           ;Address:0x50 T3L Bits------------------
                                           T3L7               .EQU                7
                                           T3L6               .EQU                6
                                           T3L5               .EQU                5
                                           T3L4               .EQU                4
                                           T3L3               .EQU                3
                                           T3L2               .EQU                2
                                           T3L1               .EQU                1
                                           T3L0               .EQU                0
                                           _T3L7              .EQU                7
                                           _T3L6              .EQU                6
                                           _T3L5              .EQU                5
                                           _T3L4              .EQU                4
                                           _T3L3              .EQU                3
                                           _T3L2              .EQU                2
                                           _T3L1              .EQU                1
                                           _T3L0              .EQU                0
                                           
                                           ;Address:0x53 CTCTL Bits----------------
                                           CTEN               .EQU                7
                                           CTSTART            .EQU                6
                                           CTCAPS             .EQU                5
                                           CTCMS              .EQU                4
                                           CTCHSEL4           .EQU                4
                                           CTCHSEL3           .EQU                3
                                           CTCHSEL2           .EQU                2
                                           CTCHSEL1           .EQU                1
                                           CTCHSEL0           .EQU                0
                                           _CTEN              .EQU                7
                                           _CTSTART           .EQU                6
                                           _CTCAPS            .EQU                5
                                           _CTCMS             .EQU                4
                                           _CTCHSEL4          .EQU                4
                                           _CTCHSEL3          .EQU                3
                                           _CTCHSEL2          .EQU                2
                                           _CTCHSEL1          .EQU                1
                                           _CTCHSEL0          .EQU                0
                                           
                                           ;Address:0x5E OSCLDOCAL Bits------------
                                            
                                            
                                           ;--------------------------------------------------------
                                           ; external declarations
                                           ;--------------------------------------------------------
                                           	.extern	_init_mcu
                                           	.extern	__KF8S_Get_Ver_General_
                                           	.extern	__KF8S_Lib_Set_General_Parameter
                                           	.extern	__KF8S_Init_Touch_General_
                                           	.extern	__KF8S_Touch_Process_General_
                                           	.extern	__KF8S_Touch_TEST_General_
                                           	.extern	_delay_ms
                                           	.extern	_delay_us
                                           	.extern	__R2PCL
                                           	.extern	_PSW_bits
                                           	.extern	_P0_bits
                                           	.extern	_P2_bits
                                           	.extern	_P1_bits
                                           	.extern	_P3_bits
                                           	.extern	_INTCTL_bits
                                           	.extern	_EIF1_bits
                                           	.extern	_T1CTL_bits
                                           	.extern	_T2CTL_bits
                                           	.extern	_PWMCTL_bits
                                           	.extern	_CMCTL1_bits
                                           	.extern	_ADCCTL0_bits
                                           	.extern	_OPTR_bits
                                           	.extern	_TR0_bits
                                           	.extern	_TR2_bits
                                           	.extern	_TR1_bits
                                           	.extern	_TR3_bits
                                           	.extern	_EIE1_bits
                                           	.extern	_PCTL_bits
                                           	.extern	_OSCCTL_bits
                                           	.extern	_ANSEL_bits
                                           	.extern	_PUR_bits
                                           	.extern	_IOCL_bits
                                           	.extern	_ADCCTL1_bits
                                           	.extern	_T3L_bits
                                           	.extern	_CTCTL_bits
                                           	.extern	_OSCLDOCAL_bits
                                           	.extern	__KF8_LIBi_channel_flag_
                                           	.extern	__KF8_LIBc_channel_
                                           	.extern	__KF8_LIBc_channel_Buf
                                           	.extern	__KF8_LIBi_Date_Change_
                                           	.extern	__KF8_LIBc_baseline_count_
                                           	.extern	__KF8_LIBi_buff_hit_
                                           	.extern	__KF8_LIBi_buff_baseline_
                                           	.extern	__KF8_LIBc_touch_count_
                                           	.extern	_CHS_AMOUNT
                                           	.extern	_TCS_AMOUNT
                                           	.extern	__KF8_Disturb_Protect_Circle_
                                           	.extern	__KF8_DoubleKey_Compages_Limitable_Circle_
                                           	.extern	__KF8_Key_Max_Pressed_Limitable_Circle_
                                           	.extern	__KF8_BaseLine_Update_Circle_Count_For_UP_
                                           	.extern	__KF8_BaseLine_Update_Circle_Count_For_Down_
                                           	.extern	__KF8_Define_Disturb_Channels_Amount_
                                           	.extern	__KF8_BasicLine_UP_Noise_Threshold_
                                           	.extern	__KF8_BasicLine_Down_Noise_Threshold_
                                           	.extern	__KF8_Data_Steady_Threshold_Set_
                                           	.extern	__KF8_Inside_Reference_Channel_Disturb_Threshold_Set_
                                           	.extern	__KF8_Inside_Reference_Channel_Declare_
                                           	.extern	__KF8_Config_Finger_Threshold
                                           	.extern	__KF8_TOUCH_CH_EN
                                           	.extern	_T0
                                           	.extern	_PCL
                                           	.extern	_PSW
                                           	.extern	_P0
                                           	.extern	_P2
                                           	.extern	_P1
                                           	.extern	_P3
                                           	.extern	_PCH
                                           	.extern	_INTCTL
                                           	.extern	_EIF1
                                           	.extern	_T1L
                                           	.extern	_T1H
                                           	.extern	_T1CTL
                                           	.extern	_T2
                                           	.extern	_T2CTL
                                           	.extern	_PWMCTL
                                           	.extern	_CMCTL1
                                           	.extern	_VRECAL
                                           	.extern	_ADCDATAH
                                           	.extern	_ADCCTL0
                                           	.extern	_OPTR
                                           	.extern	_TR0
                                           	.extern	_TR2
                                           	.extern	_TR1
                                           	.extern	_TR3
                                           	.extern	_EIE1
                                           	.extern	_PCTL
                                           	.extern	_OSCCTL
                                           	.extern	_OSCCAL0
                                           	.extern	_ANSEL
                                           	.extern	_PUR
                                           	.extern	_IOCL
                                           	.extern	_OSCCAL1
                                           	.extern	_ADCDATAL
                                           	.extern	_ADCCTL1
                                           	.extern	_T3L
                                           	.extern	_CTCTL
                                           	.extern	_T2CCR
                                           	.extern	_OSCLDOCAL
                                           	.extern	_T1U
                                           
                                           	.extern STK12
                                           	.extern STK11
                                           	.extern STK10
                                           	.extern STK09
                                           	.extern STK08
                                           	.extern STK07
                                           	.extern STK06
                                           	.extern STK05
                                           	.extern STK04
                                           	.extern STK03
                                           	.extern STK02
                                           	.extern STK01
                                           	.extern STK00
                                           ;--------------------------------------------------------
                                           ; global declarations
                                           ;--------------------------------------------------------
                                           	.global	_TOUCH_DEBUG_SEND_OUT
                                           	.global	_TOUCH_DEBUG_TRS_DEAL
                                           	.global	_TOUCH_CH_TRS_EN
                                           	.global	_T_buf
                                           	.global	_i_T_D
                                           	.global	_sentbuf1
                                           	.global	_sentbuf2
                                           	.global	_sentbuf3
                                           	.global	_sentbuf4
                                           
                                           ;--------------------------------------------------------
                                           ; global definitions
                                           ;--------------------------------------------------------
                                           UD_debug_touch_0	.udata
                                           _T_buf	.res	1
                                           
                                           UD_debug_touch_1	.udata
                                           _i_T_D	.res	1
                                           
                                           UD_debug_touch_2	.udata
                                           _sentbuf1	.res	1
                                           
                                           UD_debug_touch_3	.udata
                                           _sentbuf2	.res	1
                                           
                                           UD_debug_touch_4	.udata
                                           _sentbuf3	.res	1
                                           
                                           UD_debug_touch_5	.udata
                                           _sentbuf4	.res	1
                                           
                                           ;--------------------------------------------------------
                                           ; absolute symbol definitions
                                           ;--------------------------------------------------------
                                           ;--------------------------------------------------------
                                           ; compiler-defined variables
                                           ;--------------------------------------------------------
                                           UDL_debug_touch_0	.udata
                                           r0x1008	.res	1
                                           UDL_debug_touch_1	.udata
                                           r0x1009	.res	1
                                           UDL_debug_touch_2	.udata
                                           r0x1006	.res	1
                                           UDL_debug_touch_3	.udata
                                           r0x1007	.res	1
                                           ;--------------------------------------------------------
                                           ; initialized data
                                           ;--------------------------------------------------------
                                           
                                           ID_debug_touch_0	.idata
                                           _TOUCH_CH_TRS_EN
                                           	.db	0x00
                                           	.db	0x00
                                           	.db	0x00
                                           	.db	0x00
                                           	.db	0x00
                                           	.db	0x00
                                           	.db	0x00
                                           	.db	0x00
                                           	.db	0x00
                                           	.db	0x00
                                           	.db	0x00
                                           	.db	0x00
                                           	.db	0x00
                                           	.db	0x00
                                           	.db	0x00
                                           	.db	0x00
                                           
                                           ;--------------------------------------------------------
                                           ; overlayable items in internal ram 
                                           ;--------------------------------------------------------
                                           ;	.udata_ovr
                                           
                                           
                                           func._TOUCH_DEBUG_SEND_OUT	.code
                                           ;***
                                           ;  PostBlock Stats: dbName = C
                                           ;***
                                           ;entry:  _TOUCH_DEBUG_SEND_OUT	;Function start
                                           ; 2 exit points
                                           ;has an exit
                                           ;functions called:
                                           ;   _delay_us
                                           ;   _delay_us
                                           ;   _delay_us
                                           ;   _delay_us
                                           ;   _delay_us
                                           ;   _delay_us
                                           ;   _delay_us
                                           ;   _delay_us
                                           ;   _delay_us
                                           ;   _delay_us
                                           ;   _delay_us
                                           ;   _delay_us
                                           ;   _delay_us
                                           ;   _delay_us
                                           ;   _delay_us
                                           ;   _delay_us
                                           ;   _delay_us
                                           ;   _delay_us
                                           ;   _delay_us
                                           ;   _delay_us
                                           ;   _delay_us
                                           ;   _delay_us
                                           ;   _delay_us
                                           ;   _delay_us
                                           ;   _delay_us
                                           ;   _delay_us
                                           ;   _delay_us
                                           ;   _delay_us
                                           ;   _delay_us
                                           ;   _delay_us
                                           ;   _delay_us
                                           ;   _delay_us
                                           ;3 compiler assigned registers:
                                           ;   STK00
                                           ;   r0x1006
                                           ;   r0x1007
                                           ;; Starting PostCode block
                                           ;	op : LABEL
                                           ;	op : FUNCTION
                                           _TOUCH_DEBUG_SEND_OUT	;Function start
                                           ; 2 exit points
                                           ;	op : =
                                           ;	.line	322; "../debug_touch.c"	CLK_SET_IN;
                                           	SET	_TR0_bits, 1
                                           ;	op : =
                                           ;	.line	323; "../debug_touch.c"	DAT_SET_IN;
                                           	SET	_TR0_bits, 0
                                           ;	op : SEND
                                           ;	op : CALL
                                           ;	.line	324; "../debug_touch.c"	Touch_Delay1;
                                           	MOV	R0,# 0x05
                                           	BANKSEL	STK00
                                           	MOV	STK00, R0
                                           	MOV	R0,# 0x00
                                           	PAGESEL	_delay_us
                                           	CALL	_delay_us
                                           	PAGESEL	$
                                           ;	op : GET_VALUE_AT_ADDRESS
                                           ;	.line	328; "../debug_touch.c"	if(CLK_GET_STATE)
                                           	JB	_P0_bits, 1
                                           	JMP	_00078_DS_
                                           ;	op : SEND
                                           ;	op : CALL
                                           ;	.line	330; "../debug_touch.c"	Touch_Delay1;
                                           	MOV	R0,# 0x05
                                           	BANKSEL	STK00
                                           	MOV	STK00, R0
                                           	MOV	R0,# 0x00
                                           	PAGESEL	_delay_us
                                           	CALL	_delay_us
                                           	PAGESEL	$
                                           ;	op : GET_VALUE_AT_ADDRESS
                                           ;	.line	331; "../debug_touch.c"	if(!CLK_GET_STATE)
                                           	JNB	_P0_bits, 1
                                           	JMP	_00079_DS_
                                           ;	op : RETURN
                                           ;	.line	332; "../debug_touch.c"	return;
                                           	JMP	_00116_DS_
                                           ;	op : LABEL
                                           ;	op : GET_VALUE_AT_ADDRESS
                                           _00078_DS_
                                           ;	.line	334; "../debug_touch.c"	else if(!CLK_GET_STATE)
                                           	JNB	_P0_bits, 1
                                           	JMP	_00075_DS_
                                           ;	op : RETURN
                                           ;	.line	336; "../debug_touch.c"	return;
                                           	JMP	_00116_DS_
                                           ;	op : LABEL
                                           ;	op : RETURN
                                           _00075_DS_
                                           ;	.line	339; "../debug_touch.c"	return;
                                           	JMP	_00116_DS_
                                           ;	op : LABEL
                                           ;	op : =
                                           _00079_DS_
                                           ;	.line	341; "../debug_touch.c"	CLK_SET_OUT;
                                           	CLR	_TR0_bits, 1
                                           ;	op : =
                                           ;	.line	343; "../debug_touch.c"	CLK_SET_LOW;
                                           	CLR	_P0_bits, 1
                                           ;	op : SEND
                                           ;	op : CALL
                                           ;	.line	344; "../debug_touch.c"	Touch_Delay1;
                                           	MOV	R0,# 0x05
                                           	BANKSEL	STK00
                                           	MOV	STK00, R0
                                           	MOV	R0,# 0x00
                                           	PAGESEL	_delay_us
                                           	CALL	_delay_us
                                           	PAGESEL	$
                                           ;	op : =
                                           ;	.line	346; "../debug_touch.c"	CLK_SET_HIGH;		//ÉÏÉýÑØ
                                           	SET	_P0_bits, 1
                                           ;	op : SEND
                                           ;	op : CALL
                                           ;	.line	348; "../debug_touch.c"	Touch_Delay1;
                                           	MOV	R0,# 0x05
                                           	BANKSEL	STK00
                                           	MOV	STK00, R0
                                           	MOV	R0,# 0x00
                                           	PAGESEL	_delay_us
                                           	CALL	_delay_us
                                           ;	.line	350; "../debug_touch.c"	if(!DAT_GET_STATE)
                                           	PAGESEL	$
                                           ;	.line	352; "../debug_touch.c"	return;
                                           	JB	_P0_bits, 0
                                           ;	.line	355; "../debug_touch.c"	CLK_SET_LOW;			//ÏÂ½µÑØ
                                           	JMP	_00116_DS_
                                           	CLR	_P0_bits, 1
                                           ;	.line	358; "../debug_touch.c"	Touch_Delay1;
                                           	MOV	R0,# 0x05
                                           	BANKSEL	STK00
                                           	MOV	STK00, R0
                                           	MOV	R0,# 0x00
                                           	PAGESEL	_delay_us
                                           	CALL	_delay_us
                                           	PAGESEL	$
                                           ;	op : =
                                           ;	.line	360; "../debug_touch.c"	DAT_SET_OUT;
                                           	CLR	_TR0_bits, 0
                                           ;	op : =
                                           ;	.line	363; "../debug_touch.c"	j=5;
                                           	MOV	R0,# 0x05
                                           	BANKSEL	r0x1006
                                           	MOV	r0x1006, R0
                                           ;	op : =
                                           ;	.line	365; "../debug_touch.c"	for(step=0;step<5;step++)
                                           	BANKSEL	r0x1007
                                           	CLR	r0x1007
                                           ;	op : LABEL
                                           ;	op : <
                                           ;unsigned compare: left < lit(0x5=5), size=1
                                           _00108_DS_
                                           	MOV	R0,# 0x05
                                           	BANKSEL	r0x1007
                                           	SUB	R0, r0x1007
                                           ;comparing bytes at offset 0
                                           	JNB	PSW, 0
                                           	JMP	_00111_DS_
                                           ;	op : >
                                           ;swapping arguments (AOP_TYPEs 1/2)
                                           ;unsigned compare: left >= lit(0x5=5), size=1
                                           ;	.line	368; "../debug_touch.c"	switch(step)
                                           	MOV	R0,# 0x05
                                           	BANKSEL	r0x1007
                                           	SUB	R0, r0x1007
                                           ;comparing bytes at offset 0
                                           	JNB	PSW, 0
                                           	JMP	_00087_DS_
                                           ;	op : JUMPTABLE
                                           	MOV	R0,#high _00138_DS_
                                           	MOV	PCH, R0
                                           	MOV	R0,#_00138_DS_
                                           	BANKSEL	r0x1007
                                           	ADD	R0, r0x1007
                                           	JNB	PSW, 0
                                           	INC	PCH
                                           	MOV	PCL, R0
                                           _00138_DS_
                                           	JMP	_00082_DS_
                                           	JMP	_00083_DS_
                                           	JMP	_00084_DS_
                                           	JMP	_00085_DS_
                                           	JMP	_00086_DS_
                                           ;	op : LABEL
                                           ;	op : =
                                           _00082_DS_
                                           ;	.line	372; "../debug_touch.c"	j=5;
                                           	MOV	R0,# 0x05
                                           	BANKSEL	r0x1006
                                           	MOV	r0x1006, R0
                                           ;	op : =
                                           ;	.line	373; "../debug_touch.c"	T_buf=0x04;
                                           	MOV	R0,# 0x04
                                           	BANKSEL	_T_buf
                                           	MOV	_T_buf, R0
                                           ;	op : GOTO
                                           ;	.line	374; "../debug_touch.c"	}break;
                                           	JMP	_00087_DS_
                                           ;	op : LABEL
                                           ;	op : =
                                           _00083_DS_
                                           ;	.line	378; "../debug_touch.c"	j=8;
                                           	MOV	R0,# 0x08
                                           	BANKSEL	r0x1006
                                           	MOV	r0x1006, R0
                                           ;	op : =
                                           ;	.line	380; "../debug_touch.c"	T_buf=sentbuf1;
                                           	BANKSEL	_sentbuf1
                                           	MOVZ	R0, _sentbuf1
                                           	BANKSEL	_T_buf
                                           	MOV	_T_buf, R0
                                           ;	op : GOTO
                                           ;	.line	382; "../debug_touch.c"	}break;
                                           	JMP	_00087_DS_
                                           ;	op : LABEL
                                           ;	op : =
                                           _00084_DS_
                                           ;	.line	386; "../debug_touch.c"	j=8;
                                           	MOV	R0,# 0x08
                                           	BANKSEL	r0x1006
                                           	MOV	r0x1006, R0
                                           ;	op : =
                                           ;	.line	387; "../debug_touch.c"	T_buf=sentbuf2;
                                           	BANKSEL	_sentbuf2
                                           	MOVZ	R0, _sentbuf2
                                           	BANKSEL	_T_buf
                                           	MOV	_T_buf, R0
                                           ;	op : GOTO
                                           ;	.line	389; "../debug_touch.c"	}break;
                                           	JMP	_00087_DS_
                                           ;	op : LABEL
                                           ;	op : =
                                           _00085_DS_
                                           ;	.line	393; "../debug_touch.c"	j=8;
                                           	MOV	R0,# 0x08
                                           	BANKSEL	r0x1006
                                           	MOV	r0x1006, R0
                                           ;	op : =
                                           ;	.line	394; "../debug_touch.c"	T_buf=sentbuf3;
                                           	BANKSEL	_sentbuf3
                                           	MOVZ	R0, _sentbuf3
                                           	BANKSEL	_T_buf
                                           	MOV	_T_buf, R0
                                           ;	op : GOTO
                                           ;	.line	395; "../debug_touch.c"	}break;
                                           	JMP	_00087_DS_
                                           ;	op : LABEL
                                           ;	op : =
                                           _00086_DS_
                                           ;	.line	399; "../debug_touch.c"	j=8;
                                           	MOV	R0,# 0x08
                                           	BANKSEL	r0x1006
                                           	MOV	r0x1006, R0
                                           ;	op : =
                                           ;	.line	400; "../debug_touch.c"	T_buf=sentbuf4;
                                           	BANKSEL	_sentbuf4
                                           	MOVZ	R0, _sentbuf4
                                           	BANKSEL	_T_buf
                                           	MOV	_T_buf, R0
                                           ;	op : LABEL
                                           ;	op : =
                                           _00087_DS_
                                           ;	.line	404; "../debug_touch.c"	for(i_T_D=0;i_T_D<j;i_T_D++)
                                           	BANKSEL	_i_T_D
                                           	CLR	_i_T_D
                                           ;	op : LABEL
                                           ;	op : <
                                           _00104_DS_
                                           	BANKSEL	r0x1006
                                           	MOVZ	R0, r0x1006
                                           	BANKSEL	_i_T_D
                                           	SUB	R0, _i_T_D
                                           ;comparing bytes at offset 0
                                           	JNB	PSW, 0
                                           	JMP	_00107_DS_
                                           ;	op : BITWISEAND
                                           ;	.line	406; "../debug_touch.c"	if(T_buf&0x01)
                                           	BANKSEL	_T_buf
                                           	JB	_T_buf, 0
                                           	JMP	_00089_DS_
                                           ;	op : =
                                           ;	.line	407; "../debug_touch.c"	DAT_SET_HIGH;
                                           	SET	_P0_bits, 0
                                           ;	op : GOTO
                                           	JMP	_00090_DS_
                                           ;	op : LABEL
                                           ;	op : =
                                           _00089_DS_
                                           ;	.line	409; "../debug_touch.c"	DAT_SET_LOW;
                                           	CLR	_P0_bits, 0
                                           ;	op : LABEL
                                           ;	op : =
                                           _00090_DS_
                                           ;	.line	411; "../debug_touch.c"	CLK_SET_HIGH;
                                           	SET	_P0_bits, 1
                                           ;	op : SEND
                                           ;	op : CALL
                                           ;	.line	412; "../debug_touch.c"	Touch_Delay1;
                                           	MOV	R0,# 0x05
                                           	BANKSEL	STK00
                                           	MOV	STK00, R0
                                           	MOV	R0,# 0x00
                                           	PAGESEL	_delay_us
                                           	CALL	_delay_us
                                           	PAGESEL	$
                                           ;	op : =
                                           ;	.line	414; "../debug_touch.c"	CLK_SET_LOW;
                                           	CLR	_P0_bits, 1
                                           ;	op : SEND
                                           ;	op : CALL
                                           ;	.line	415; "../debug_touch.c"	Touch_Delay1;
                                           	MOV	R0,# 0x05
                                           	BANKSEL	STK00
                                           	MOV	STK00, R0
                                           	MOV	R0,# 0x00
                                           	PAGESEL	_delay_us
                                           	CALL	_delay_us
                                           	PAGESEL	$
                                           ;	op : RIGHT_OP
                                           ;	.line	417; "../debug_touch.c"	T_buf=T_buf>>1;
                                           	CLR	PSW, 0
                                           	BANKSEL	_T_buf
                                           	RRC	_T_buf
                                           ;	op : +
                                           ;	.line	404; "../debug_touch.c"	for(i_T_D=0;i_T_D<j;i_T_D++)
                                           	BANKSEL	_i_T_D
                                           	INC	_i_T_D
                                           ;	op : GOTO
                                           	JMP	_00104_DS_
                                           ;	op : LABEL
                                           ;	op : SEND
                                           ;	op : CALL
                                           _00107_DS_
                                           ;	.line	420; "../debug_touch.c"	Touch_Delay2;
                                           	MOV	R0,# 0x6e
                                           	BANKSEL	STK00
                                           	MOV	STK00, R0
                                           	MOV	R0,# 0x00
                                           	PAGESEL	_delay_us
                                           	CALL	_delay_us
                                           	PAGESEL	$
                                           ;	op : +
                                           ;	.line	365; "../debug_touch.c"	for(step=0;step<5;step++)
                                           	BANKSEL	r0x1007
                                           	INC	r0x1007
                                           ;	op : GOTO
                                           	JMP	_00108_DS_
                                           ;	op : LABEL
                                           ;	op : =
                                           _00111_DS_
                                           ;	.line	424; "../debug_touch.c"	DAT_SET_IN;
                                           	SET	_TR0_bits, 0
                                           ;	op : SEND
                                           ;	op : CALL
                                           ;	.line	425; "../debug_touch.c"	Touch_Delay2;	//±à³ÌÆ÷ÅÐ¶ÏÐèÒªÊ±¼ä
                                           	MOV	R0,# 0x6e
                                           	BANKSEL	STK00
                                           	MOV	STK00, R0
                                           	MOV	R0,# 0x00
                                           	PAGESEL	_delay_us
                                           	CALL	_delay_us
                                           	PAGESEL	$
                                           ;	op : =
                                           ;	.line	427; "../debug_touch.c"	CLK_SET_HIGH;
                                           	SET	_P0_bits, 1
                                           ;	op : SEND
                                           ;	op : CALL
                                           ;	.line	428; "../debug_touch.c"	Touch_Delay1;
                                           	MOV	R0,# 0x05
                                           	BANKSEL	STK00
                                           	MOV	STK00, R0
                                           	MOV	R0,# 0x00
                                           	PAGESEL	_delay_us
                                           	CALL	_delay_us
                                           	PAGESEL	$
                                           ;	op : SEND
                                           ;	op : CALL
                                           ;	.line	429; "../debug_touch.c"	Touch_Delay1;
                                           	MOV	R0,# 0x05
                                           	BANKSEL	STK00
                                           	MOV	STK00, R0
                                           	MOV	R0,# 0x00
                                           	PAGESEL	_delay_us
                                           	CALL	_delay_us
                                           	PAGESEL	$
                                           ;	op : SEND
                                           ;	op : CALL
                                           ;	.line	430; "../debug_touch.c"	Touch_Delay1;
                                           	MOV	R0,# 0x05
                                           	BANKSEL	STK00
                                           	MOV	STK00, R0
                                           	MOV	R0,# 0x00
                                           	PAGESEL	_delay_us
                                           	CALL	_delay_us
                                           	PAGESEL	$
                                           ;	op : GET_VALUE_AT_ADDRESS
                                           ;	.line	433; "../debug_touch.c"	if(DAT_GET_STATE)
                                           	JB	_P0_bits, 0
                                           	JMP	_00102_DS_
                                           ;	op : =
                                           ;	.line	435; "../debug_touch.c"	CLK_SET_LOW;
                                           	CLR	_P0_bits, 1
                                           ;	op : =
                                           ;	.line	436; "../debug_touch.c"	T_buf=0;
                                           	BANKSEL	_T_buf
                                           	CLR	_T_buf
                                           ;	op : SEND
                                           ;	op : CALL
                                           ;	.line	437; "../debug_touch.c"	Touch_Delay1;
                                           	MOV	R0,# 0x05
                                           	BANKSEL	STK00
                                           	MOV	STK00, R0
                                           	MOV	R0,# 0x00
                                           	PAGESEL	_delay_us
                                           	CALL	_delay_us
                                           	PAGESEL	$
                                           ;	op : =
                                           ;	.line	438; "../debug_touch.c"	for(i_T_D=0;i_T_D<6;i_T_D++)
                                           	BANKSEL	_i_T_D
                                           	CLR	_i_T_D
                                           ;	op : LABEL
                                           ;	op : <
                                           ;unsigned compare: left < lit(0x6=6), size=1
                                           _00112_DS_
                                           	MOV	R0,# 0x06
                                           	BANKSEL	_i_T_D
                                           	SUB	R0, _i_T_D
                                           ;comparing bytes at offset 0
                                           	JNB	PSW, 0
                                           	JMP	_00103_DS_
                                           ;	op : =
                                           ;	.line	440; "../debug_touch.c"	CLK_SET_HIGH;
                                           	SET	_P0_bits, 1
                                           ;	op : SEND
                                           ;	op : CALL
                                           ;	.line	441; "../debug_touch.c"	Touch_Delay1;
                                           	MOV	R0,# 0x05
                                           	BANKSEL	STK00
                                           	MOV	STK00, R0
                                           	MOV	R0,# 0x00
                                           	PAGESEL	_delay_us
                                           	CALL	_delay_us
                                           	PAGESEL	$
                                           ;	op : EQ_OP
                                           ;	.line	443; "../debug_touch.c"	if(i_T_D!=5)
                                           	BANKSEL	_i_T_D
                                           	MOVZ	R0, _i_T_D
                                           ;	.line	445; "../debug_touch.c"	T_buf=T_buf>>1;
                                           	XOR	R0,# 0x05
                                           	JNB	PSW, 2
                                           	JMP	_00099_DS_
                                           	CLR	PSW, 0
                                           	BANKSEL	_T_buf
                                           	RRC	_T_buf
                                           ;	op : GET_VALUE_AT_ADDRESS
                                           ;	.line	446; "../debug_touch.c"	if(DAT_GET_STATE)
                                           	JB	_P0_bits, 0
                                           	JMP	_00100_DS_
                                           ;	op : |
                                           ;	.line	447; "../debug_touch.c"	T_buf=T_buf|0x10;
                                           	BANKSEL	_T_buf
                                           	SET	_T_buf, 4
                                           ;	op : GOTO
                                           	JMP	_00100_DS_
                                           ;	op : LABEL
                                           ;	op : <
                                           ;unsigned compare: left < lit(0x10=16), size=1
                                           _00099_DS_
                                           ;	.line	451; "../debug_touch.c"	if(T_buf<16)   //´«Êä´íÎóµÄ£¬·ÀÏÂ·ÇÓ°ÏìÆäËûÊý¾Ý
                                           	MOV	R0,# 0x10
                                           	BANKSEL	_T_buf
                                           	SUB	R0, _T_buf
                                           ;comparing bytes at offset 0
                                           	JNB	PSW, 0
                                           	JMP	_00100_DS_
                                           ;	op : GET_VALUE_AT_ADDRESS
                                           ;	.line	453; "../debug_touch.c"	if(DAT_GET_STATE)
                                           	JB	_P0_bits, 0
                                           	JMP	_00094_DS_
                                           ;	op : INLINEASM
                                           	BANKSEL _T_buf
                                           	MOV R0,_T_buf
                                           	ADD R0,#(_TOUCH_CH_TRS_EN+0)
                                           	MOV R1,#0x01
                                           	BANKSEL _TOUCH_CH_TRS_EN
                                           	ST [R0],R1
                                           	
                                           ;	op : GOTO
                                           	JMP	_00100_DS_
                                           ;	op : LABEL
                                           ;	op : INLINEASM
                                           _00094_DS_
                                           	BANKSEL _T_buf
                                           	MOV R0,_T_buf
                                           	ADD R0,#(_TOUCH_CH_TRS_EN+0)
                                           	MOV R1,#0x00
                                           	BANKSEL _TOUCH_CH_TRS_EN
                                           	ST [R0],R1
                                           	
                                           ;	op : LABEL
                                           ;	op : =
                                           _00100_DS_
                                           ;	.line	479; "../debug_touch.c"	CLK_SET_LOW;
                                           	CLR	_P0_bits, 1
                                           ;	op : SEND
                                           ;	op : CALL
                                           ;	.line	480; "../debug_touch.c"	Touch_Delay1;
                                           	MOV	R0,# 0x05
                                           	BANKSEL	STK00
                                           	MOV	STK00, R0
                                           	MOV	R0,# 0x00
                                           	PAGESEL	_delay_us
                                           	CALL	_delay_us
                                           	PAGESEL	$
                                           ;	op : +
                                           ;	.line	438; "../debug_touch.c"	for(i_T_D=0;i_T_D<6;i_T_D++)
                                           	BANKSEL	_i_T_D
                                           	INC	_i_T_D
                                           ;	op : GOTO
                                           	JMP	_00112_DS_
                                           ;	op : LABEL
                                           ;	op : =
                                           _00102_DS_
                                           ;	.line	485; "../debug_touch.c"	CLK_SET_LOW;
                                           	CLR	_P0_bits, 1
                                           ;	op : SEND
                                           ;	op : CALL
                                           ;	.line	486; "../debug_touch.c"	Touch_Delay1;
                                           	MOV	R0,# 0x05
                                           	BANKSEL	STK00
                                           	MOV	STK00, R0
                                           	MOV	R0,# 0x00
                                           	PAGESEL	_delay_us
                                           	CALL	_delay_us
                                           	PAGESEL	$
                                           ;	op : LABEL
                                           ;	op : =
                                           _00103_DS_
                                           ;	.line	489; "../debug_touch.c"	CLK_SET_IN;
                                           	SET	_TR0_bits, 1
                                           ;	op : =
                                           ;	.line	490; "../debug_touch.c"	DAT_SET_IN;
                                           	SET	_TR0_bits, 0
                                           ;	op : LABEL
                                           ;	op : ENDFUNCTION
                                           _00116_DS_
                                           	CRET	
                                           ; exit point of _TOUCH_DEBUG_SEND_OUT
                                           
                                           
                                           
                                           func._TOUCH_DEBUG_TRS_DEAL	.code
                                           ;***
                                           ;  PostBlock Stats: dbName = C
                                           ;***
                                           ;entry:  _TOUCH_DEBUG_TRS_DEAL	;Function start
                                           ; 2 exit points
                                           ;has an exit
                                           ;functions called:
                                           ;   _delay_us
                                           ;   _delay_us
                                           ;   _delay_us
                                           ;   _delay_us
                                           ;   _delay_us
                                           ;   _delay_us
                                           ;   _delay_us
                                           ;   _delay_us
                                           ;   _delay_us
                                           ;   _delay_us
                                           ;   _delay_us
                                           ;   _delay_us
                                           ;   _delay_us
                                           ;   _delay_us
                                           ;   _delay_us
                                           ;   _delay_us
                                           ;   _delay_us
                                           ;   _delay_us
                                           ;   _delay_us
                                           ;   _delay_us
                                           ;   _delay_us
                                           ;   _delay_us
                                           ;   _delay_us
                                           ;   _delay_us
                                           ;   _delay_us
                                           ;   _delay_us
                                           ;   _delay_us
                                           ;   _delay_us
                                           ;   _delay_us
                                           ;   _delay_us
                                           ;   _delay_us
                                           ;   _delay_us
                                           ;3 compiler assigned registers:
                                           ;   STK00
                                           ;   r0x1008
                                           ;   r0x1009
                                           ;; Starting PostCode block
                                           ;	op : LABEL
                                           ;	op : FUNCTION
                                           _TOUCH_DEBUG_TRS_DEAL	;Function start
                                           ; 2 exit points
                                           ;	op : INLINEASM
000413   9906     MOV	R1, #0x6             	MOV R1,#High(__KF8_TOUCH_CH_EN+0)
000414   9800     MOV	R0, #0               	MOV R0,#(0)
000415   80f5     ADD	R0, #0xf5            	ADD R0,#Low(__KF8_TOUCH_CH_EN+0)
000416   7003     JNB	0x3, 0               	JNB PSW,0
000417   ff11     INC	R1                   	INC R1
                                           	PAGESEL __R2PCL
000418   d70d     CALL	#0x70d              	CALL __R2PCL
                                           	PAGESEL $
000419   8080     ADD	R0, #0x80            	ADD R0,#(_TOUCH_CH_TRS_EN+0)
00041a   9901     MOV	R1, #0x1             	MOV R1,#0x01
00041b   6d03     SET	0x3, 5               	BANKSEL _TOUCH_CH_TRS_EN
00041c   f748     ST	[R0], R1              	ST [R0],R1
                                           	
                                           ;	op : INLINEASM
00041d   6503     CLR	0x3, 5               	BANKSEL __KF8_LIBc_channel_
00041e   50a2     MOV	R0, 0xa2             	MOV R0,__KF8_LIBc_channel_
00041f   80f5     ADD	R0, #0xf5            	ADD R0,#Low(__KF8_TOUCH_CH_EN+0)
000420   9906     MOV	R1, #0x6             	MOV R1,#High(__KF8_TOUCH_CH_EN+0)
000421   7003     JNB	0x3, 0               	JNB PSW,0
000422   ff11     INC	R1                   	INC R1
                                           	PAGESEL __R2PCL
000423   d70d     CALL	#0x70d              	CALL __R2PCL
                                           	PAGESEL $
000424   8080     ADD	R0, #0x80            	ADD R0,#(_TOUCH_CH_TRS_EN+0)
000425   6d03     SET	0x3, 5               	BANKSEL _TOUCH_CH_TRS_EN
000426   f701     LD	R1, [R0]              	LD R1,[R0]
000427   a900     XOR	R1, #0               	XOR R1,#0x00
000428   7203     JNB	0x3, 2               	JNB PSW,2
000429   c50f     JMP	#0x50f               	JMP Label_x_y_z_a
                                           	
                                           ;	op : =
                                           ;	.line	64; "../debug_touch.c"	CLK_SET_IN;
00042a   6925     SET	0x25, 1              	SET	_TR0_bits, 1
                                           ;	op : =
                                           ;	.line	65; "../debug_touch.c"	DAT_SET_IN;
00042b   6825     SET	0x25, 0              	SET	_TR0_bits, 0
                                           ;	op : SEND
                                           ;	op : CALL
                                           ;	.line	66; "../debug_touch.c"	Touch_Delay1;
00042c   9805     MOV	R0, #0x5             	MOV	R0,# 0x05
00042d   6503     CLR	0x3, 5               	BANKSEL	STK00
00042e   51dd     MOV	0xdd, R0             	MOV	STK00, R0
00042f   9800     MOV	R0, #0               	MOV	R0,# 0x00
                                           	PAGESEL	_delay_us
000430   d6d2     CALL	#0x6d2              	CALL	_delay_us
                                           	PAGESEL	$
                                           ;	op : GET_VALUE_AT_ADDRESS
                                           ;	.line	70; "../debug_touch.c"	if(CLK_GET_STATE)
000431   7905     JB	0x5, 1                	JB	_P0_bits, 1
000432   c43b     JMP	#0x43b               	JMP	_00007_DS_
                                           ;	op : SEND
                                           ;	op : CALL
                                           ;	.line	72; "../debug_touch.c"	Touch_Delay1;
000433   9805     MOV	R0, #0x5             	MOV	R0,# 0x05
000434   6503     CLR	0x3, 5               	BANKSEL	STK00
000435   51dd     MOV	0xdd, R0             	MOV	STK00, R0
000436   9800     MOV	R0, #0               	MOV	R0,# 0x00
                                           	PAGESEL	_delay_us
000437   d6d2     CALL	#0x6d2              	CALL	_delay_us
                                           	PAGESEL	$
                                           ;	op : GET_VALUE_AT_ADDRESS
                                           ;	.line	73; "../debug_touch.c"	if(!CLK_GET_STATE)
000438   7105     JNB	0x5, 1               	JNB	_P0_bits, 1
000439   c43f     JMP	#0x43f               	JMP	_00008_DS_
                                           ;	op : RETURN
                                           ;	.line	74; "../debug_touch.c"	return;
00043a   c50f     JMP	#0x50f               	JMP	_00045_DS_
                                           ;	op : LABEL
                                           ;	op : GET_VALUE_AT_ADDRESS
                                           _00007_DS_
                                           ;	.line	76; "../debug_touch.c"	else if(!CLK_GET_STATE)
00043b   7105     JNB	0x5, 1               	JNB	_P0_bits, 1
00043c   c43e     JMP	#0x43e               	JMP	_00004_DS_
                                           ;	op : RETURN
                                           ;	.line	78; "../debug_touch.c"	return;
00043d   c50f     JMP	#0x50f               	JMP	_00045_DS_
                                           ;	op : LABEL
                                           ;	op : RETURN
                                           _00004_DS_
                                           ;	.line	81; "../debug_touch.c"	return;
00043e   c50f     JMP	#0x50f               	JMP	_00045_DS_
                                           ;	op : LABEL
                                           ;	op : =
                                           _00008_DS_
                                           ;	.line	83; "../debug_touch.c"	CLK_SET_OUT;
00043f   6125     CLR	0x25, 1              	CLR	_TR0_bits, 1
                                           ;	op : =
                                           ;	.line	85; "../debug_touch.c"	CLK_SET_LOW;
000440   6105     CLR	0x5, 1               	CLR	_P0_bits, 1
                                           ;	op : SEND
                                           ;	op : CALL
                                           ;	.line	86; "../debug_touch.c"	Touch_Delay1;
000441   9805     MOV	R0, #0x5             	MOV	R0,# 0x05
000442   6503     CLR	0x3, 5               	BANKSEL	STK00
000443   51dd     MOV	0xdd, R0             	MOV	STK00, R0
000444   9800     MOV	R0, #0               	MOV	R0,# 0x00
                                           	PAGESEL	_delay_us
000445   d6d2     CALL	#0x6d2              	CALL	_delay_us
                                           	PAGESEL	$
                                           ;	op : =
                                           ;	.line	88; "../debug_touch.c"	CLK_SET_HIGH;		//ÉÏÉýÑØ
000446   6905     SET	0x5, 1               	SET	_P0_bits, 1
                                           ;	op : SEND
                                           ;	op : CALL
                                           ;	.line	90; "../debug_touch.c"	Touch_Delay1;
000447   9805     MOV	R0, #0x5             	MOV	R0,# 0x05
000448   6503     CLR	0x3, 5               	BANKSEL	STK00
000449   51dd     MOV	0xdd, R0             	MOV	STK00, R0
00044a   9800     MOV	R0, #0               	MOV	R0,# 0x00
                                           	PAGESEL	_delay_us
00044b   d6d2     CALL	#0x6d2              	CALL	_delay_us
                                           ;	.line	92; "../debug_touch.c"	if(!DAT_GET_STATE)
                                           	PAGESEL	$
                                           ;	.line	94; "../debug_touch.c"	return;
00044c   7805     JB	0x5, 0                	JB	_P0_bits, 0
                                           ;	.line	97; "../debug_touch.c"	CLK_SET_LOW;			//ÏÂ½µÑØ
00044d   c50f     JMP	#0x50f               	JMP	_00045_DS_
00044e   6105     CLR	0x5, 1               	CLR	_P0_bits, 1
                                           ;	.line	101; "../debug_touch.c"	Touch_Delay1;
00044f   9805     MOV	R0, #0x5             	MOV	R0,# 0x05
000450   6503     CLR	0x3, 5               	BANKSEL	STK00
000451   51dd     MOV	0xdd, R0             	MOV	STK00, R0
000452   9800     MOV	R0, #0               	MOV	R0,# 0x00
                                           	PAGESEL	_delay_us
000453   d6d2     CALL	#0x6d2              	CALL	_delay_us
                                           	PAGESEL	$
                                           ;	op : =
                                           ;	.line	102; "../debug_touch.c"	DAT_SET_OUT;
000454   6025     CLR	0x25, 0              	CLR	_TR0_bits, 0
                                           ;	op : =
                                           ;	.line	104; "../debug_touch.c"	j=5;
000455   9805     MOV	R0, #0x5             	MOV	R0,# 0x05
000456   6503     CLR	0x3, 5               	BANKSEL	r0x1008
000457   51a4     MOV	0xa4, R0             	MOV	r0x1008, R0
                                           ;	op : =
                                           ;	.line	106; "../debug_touch.c"	for(step=0;step<5;step++)
                                           	BANKSEL	r0x1009
000458   03a3     CLR	0xa3                 	CLR	r0x1009
                                           ;	op : LABEL
                                           ;	op : <
                                           ;unsigned compare: left < lit(0x5=5), size=1
                                           _00037_DS_
000459   9805     MOV	R0, #0x5             	MOV	R0,# 0x05
                                           	BANKSEL	r0x1009
00045a   38a3     SUB	R0, 0xa3             	SUB	R0, r0x1009
                                           ;comparing bytes at offset 0
00045b   7003     JNB	0x3, 0               	JNB	PSW, 0
00045c   c4b9     JMP	#0x4b9               	JMP	_00040_DS_
                                           ;	op : >
                                           ;swapping arguments (AOP_TYPEs 1/2)
                                           ;unsigned compare: left >= lit(0x5=5), size=1
                                           ;	.line	109; "../debug_touch.c"	switch(step)
00045d   9805     MOV	R0, #0x5             	MOV	R0,# 0x05
                                           	BANKSEL	r0x1009
00045e   38a3     SUB	R0, 0xa3             	SUB	R0, r0x1009
                                           ;comparing bytes at offset 0
00045f   7003     JNB	0x3, 0               	JNB	PSW, 0
000460   c498     JMP	#0x498               	JMP	_00016_DS_
                                           ;	op : JUMPTABLE
000461   9804     MOV	R0, #0x4             	MOV	R0,#high _00067_DS_
000462   510a     MOV	0xa, R0              	MOV	PCH, R0
000463   9868     MOV	R0, #0x68            	MOV	R0,#_00067_DS_
                                           	BANKSEL	r0x1009
000464   20a3     ADD	R0, 0xa3             	ADD	R0, r0x1009
000465   7003     JNB	0x3, 0               	JNB	PSW, 0
000466   0b0a     INC	0xa                  	INC	PCH
000467   5102     MOV	0x2, R0              	MOV	PCL, R0
                                           _00067_DS_
000468   c46d     JMP	#0x46d               	JMP	_00011_DS_
000469   c479     JMP	#0x479               	JMP	_00012_DS_
00046a   c481     JMP	#0x481               	JMP	_00013_DS_
00046b   c489     JMP	#0x489               	JMP	_00014_DS_
00046c   c491     JMP	#0x491               	JMP	_00015_DS_
                                           ;	op : LABEL
                                           ;	op : =
                                           _00011_DS_
                                           ;	.line	113; "../debug_touch.c"	j=5;
00046d   9805     MOV	R0, #0x5             	MOV	R0,# 0x05
                                           	BANKSEL	r0x1008
00046e   51a4     MOV	0xa4, R0             	MOV	r0x1008, R0
                                           ;	op : INLINEASM
                                           	BANKSEL __KF8_LIBc_channel_
00046f   50a2     MOV	R0, 0xa2             	MOV R0, __KF8_LIBc_channel_
000470   80f5     ADD	R0, #0xf5            	ADD R0,#Low(__KF8_TOUCH_CH_EN+0)
000471   9906     MOV	R1, #0x6             	MOV R1,#High(__KF8_TOUCH_CH_EN+0)
000472   7003     JNB	0x3, 0               	JNB PSW,0
000473   ff11     INC	R1                   	INC R1
000474   530a     MOV	0xa, R1              	MOV PCH,R1
                                           	PAGESEL __R2PCL
000475   d70d     CALL	#0x70d              	CALL __R2PCL
                                           	PAGESEL $
000476   6503     CLR	0x3, 5               	BANKSEL _T_buf
000477   51a6     MOV	0xa6, R0             	MOV _T_buf,R0
                                           	
                                           ;	op : GOTO
                                           ;	.line	132; "../debug_touch.c"	}break;
000478   c498     JMP	#0x498               	JMP	_00016_DS_
                                           ;	op : LABEL
                                           ;	op : =
                                           _00012_DS_
                                           ;	.line	136; "../debug_touch.c"	j=8;
000479   9808     MOV	R0, #0x8             	MOV	R0,# 0x08
                                           	BANKSEL	r0x1008
00047a   51a4     MOV	0xa4, R0             	MOV	r0x1008, R0
                                           ;	op : INLINEASM
                                           	BANKSEL __KF8_LIBc_channel_
00047b   6003     CLR	0x3, 0               	CLR PSW,0
00047c   12a2     RLCR	0xa2                	RLCR __KF8_LIBc_channel_
                                           	BANKSEL __KF8_LIBi_buff_baseline_
00047d   80de     ADD	R0, #0xde            	ADD R0,#(__KF8_LIBi_buff_baseline_+0)
00047e   f701     LD	R1, [R0]              	LD R1,[R0]
                                           	BANKSEL _T_buf
00047f   53a6     MOV	0xa6, R1             	MOV _T_buf,R1
                                           	
                                           ;	op : GOTO
                                           ;	.line	151; "../debug_touch.c"	}break;
000480   c498     JMP	#0x498               	JMP	_00016_DS_
                                           ;	op : LABEL
                                           ;	op : =
                                           _00013_DS_
                                           ;	.line	155; "../debug_touch.c"	j=8;
000481   9808     MOV	R0, #0x8             	MOV	R0,# 0x08
                                           	BANKSEL	r0x1008
000482   51a4     MOV	0xa4, R0             	MOV	r0x1008, R0
                                           ;	op : INLINEASM
                                           	BANKSEL __KF8_LIBc_channel_
000483   6003     CLR	0x3, 0               	CLR PSW,0
000484   12a2     RLCR	0xa2                	RLCR __KF8_LIBc_channel_
                                           	BANKSEL __KF8_LIBi_buff_baseline_
000485   80df     ADD	R0, #0xdf            	ADD R0,#(__KF8_LIBi_buff_baseline_+1)
000486   f701     LD	R1, [R0]              	LD R1,[R0]
                                           	BANKSEL _T_buf
000487   53a6     MOV	0xa6, R1             	MOV _T_buf,R1
                                           	
                                           ;	op : GOTO
                                           ;	.line	172; "../debug_touch.c"	}break;
000488   c498     JMP	#0x498               	JMP	_00016_DS_
                                           ;	op : LABEL
                                           ;	op : =
                                           _00014_DS_
                                           ;	.line	176; "../debug_touch.c"	j=8;
000489   9808     MOV	R0, #0x8             	MOV	R0,# 0x08
                                           	BANKSEL	r0x1008
00048a   51a4     MOV	0xa4, R0             	MOV	r0x1008, R0
                                           ;	op : INLINEASM
                                           	BANKSEL __KF8_LIBc_channel_
00048b   6003     CLR	0x3, 0               	CLR PSW,0
00048c   12a2     RLCR	0xa2                	RLCR __KF8_LIBc_channel_
                                           	BANKSEL __KF8_LIBi_buff_hit_
00048d   80ee     ADD	R0, #0xee            	ADD R0,#(__KF8_LIBi_buff_hit_+0)
00048e   f701     LD	R1, [R0]              	LD R1,[R0]
                                           	BANKSEL _T_buf
00048f   53a6     MOV	0xa6, R1             	MOV _T_buf,R1
                                           	
                                           ;	op : GOTO
                                           ;	.line	192; "../debug_touch.c"	}break;
000490   c498     JMP	#0x498               	JMP	_00016_DS_
                                           ;	op : LABEL
                                           ;	op : =
                                           _00015_DS_
                                           ;	.line	196; "../debug_touch.c"	j=8;
000491   9808     MOV	R0, #0x8             	MOV	R0,# 0x08
                                           	BANKSEL	r0x1008
000492   51a4     MOV	0xa4, R0             	MOV	r0x1008, R0
                                           ;	op : INLINEASM
                                           	BANKSEL __KF8_LIBc_channel_
000493   6003     CLR	0x3, 0               	CLR PSW,0
000494   12a2     RLCR	0xa2                	RLCR __KF8_LIBc_channel_
                                           	BANKSEL __KF8_LIBi_buff_hit_
000495   80ef     ADD	R0, #0xef            	ADD R0,#(__KF8_LIBi_buff_hit_+1)
000496   f701     LD	R1, [R0]              	LD R1,[R0]
                                           	BANKSEL _T_buf
000497   53a6     MOV	0xa6, R1             	MOV _T_buf,R1
                                           	
                                           ;	op : LABEL
                                           ;	op : =
                                           _00016_DS_
                                           ;	.line	214; "../debug_touch.c"	for(i_T_D=0;i_T_D<j;i_T_D++)
                                           	BANKSEL	_i_T_D
000498   03a5     CLR	0xa5                 	CLR	_i_T_D
                                           ;	op : LABEL
                                           ;	op : <
                                           _00033_DS_
                                           	BANKSEL	r0x1008
000499   0ea4     MOVZ	R0, 0xa4            	MOVZ	R0, r0x1008
                                           	BANKSEL	_i_T_D
00049a   38a5     SUB	R0, 0xa5             	SUB	R0, _i_T_D
                                           ;comparing bytes at offset 0
00049b   7003     JNB	0x3, 0               	JNB	PSW, 0
00049c   c4b2     JMP	#0x4b2               	JMP	_00036_DS_
                                           ;	op : BITWISEAND
                                           ;	.line	216; "../debug_touch.c"	if(T_buf&0x01)
                                           	BANKSEL	_T_buf
00049d   78a6     JB	0xa6, 0               	JB	_T_buf, 0
00049e   c4a1     JMP	#0x4a1               	JMP	_00018_DS_
                                           ;	op : =
                                           ;	.line	217; "../debug_touch.c"	DAT_SET_HIGH;
00049f   6805     SET	0x5, 0               	SET	_P0_bits, 0
                                           ;	op : GOTO
0004a0   c4a2     JMP	#0x4a2               	JMP	_00019_DS_
                                           ;	op : LABEL
                                           ;	op : =
                                           _00018_DS_
                                           ;	.line	219; "../debug_touch.c"	DAT_SET_LOW;
0004a1   6005     CLR	0x5, 0               	CLR	_P0_bits, 0
                                           ;	op : LABEL
                                           ;	op : =
                                           _00019_DS_
                                           ;	.line	221; "../debug_touch.c"	CLK_SET_HIGH;
0004a2   6905     SET	0x5, 1               	SET	_P0_bits, 1
                                           ;	op : SEND
                                           ;	op : CALL
                                           ;	.line	222; "../debug_touch.c"	Touch_Delay1;
0004a3   9805     MOV	R0, #0x5             	MOV	R0,# 0x05
                                           	BANKSEL	STK00
0004a4   51dd     MOV	0xdd, R0             	MOV	STK00, R0
0004a5   9800     MOV	R0, #0               	MOV	R0,# 0x00
                                           	PAGESEL	_delay_us
0004a6   d6d2     CALL	#0x6d2              	CALL	_delay_us
                                           	PAGESEL	$
                                           ;	op : =
                                           ;	.line	224; "../debug_touch.c"	CLK_SET_LOW;
0004a7   6105     CLR	0x5, 1               	CLR	_P0_bits, 1
                                           ;	op : SEND
                                           ;	op : CALL
                                           ;	.line	225; "../debug_touch.c"	Touch_Delay1;
0004a8   9805     MOV	R0, #0x5             	MOV	R0,# 0x05
0004a9   6503     CLR	0x3, 5               	BANKSEL	STK00
0004aa   51dd     MOV	0xdd, R0             	MOV	STK00, R0
0004ab   9800     MOV	R0, #0               	MOV	R0,# 0x00
                                           	PAGESEL	_delay_us
0004ac   d6d2     CALL	#0x6d2              	CALL	_delay_us
                                           	PAGESEL	$
                                           ;	op : RIGHT_OP
                                           ;	.line	227; "../debug_touch.c"	T_buf=T_buf>>1;
0004ad   6003     CLR	0x3, 0               	CLR	PSW, 0
0004ae   6503     CLR	0x3, 5               	BANKSEL	_T_buf
0004af   11a6     RRC	0xa6                 	RRC	_T_buf
                                           ;	op : +
                                           ;	.line	214; "../debug_touch.c"	for(i_T_D=0;i_T_D<j;i_T_D++)
                                           	BANKSEL	_i_T_D
0004b0   0ba5     INC	0xa5                 	INC	_i_T_D
                                           ;	op : GOTO
0004b1   c499     JMP	#0x499               	JMP	_00033_DS_
                                           ;	op : LABEL
                                           ;	op : SEND
                                           ;	op : CALL
                                           _00036_DS_
                                           ;	.line	230; "../debug_touch.c"	Touch_Delay2;
0004b2   986e     MOV	R0, #0x6e            	MOV	R0,# 0x6e
                                           	BANKSEL	STK00
0004b3   51dd     MOV	0xdd, R0             	MOV	STK00, R0
0004b4   9800     MOV	R0, #0               	MOV	R0,# 0x00
                                           	PAGESEL	_delay_us
0004b5   d6d2     CALL	#0x6d2              	CALL	_delay_us
                                           	PAGESEL	$
                                           ;	op : +
                                           ;	.line	106; "../debug_touch.c"	for(step=0;step<5;step++)
0004b6   6503     CLR	0x3, 5               	BANKSEL	r0x1009
0004b7   0ba3     INC	0xa3                 	INC	r0x1009
                                           ;	op : GOTO
0004b8   c459     JMP	#0x459               	JMP	_00037_DS_
                                           ;	op : LABEL
                                           ;	op : =
                                           _00040_DS_
                                           ;	.line	234; "../debug_touch.c"	DAT_SET_IN;
0004b9   6825     SET	0x25, 0              	SET	_TR0_bits, 0
                                           ;	op : SEND
                                           ;	op : CALL
                                           ;	.line	235; "../debug_touch.c"	Touch_Delay2;	//±à³ÌÆ÷ÅÐ¶ÏÐèÒªÊ±¼ä
0004ba   986e     MOV	R0, #0x6e            	MOV	R0,# 0x6e
                                           	BANKSEL	STK00
0004bb   51dd     MOV	0xdd, R0             	MOV	STK00, R0
0004bc   9800     MOV	R0, #0               	MOV	R0,# 0x00
                                           	PAGESEL	_delay_us
0004bd   d6d2     CALL	#0x6d2              	CALL	_delay_us
                                           	PAGESEL	$
                                           ;	op : =
                                           ;	.line	237; "../debug_touch.c"	CLK_SET_HIGH;
0004be   6905     SET	0x5, 1               	SET	_P0_bits, 1
                                           ;	op : SEND
                                           ;	op : CALL
                                           ;	.line	238; "../debug_touch.c"	Touch_Delay1;
0004bf   9805     MOV	R0, #0x5             	MOV	R0,# 0x05
0004c0   6503     CLR	0x3, 5               	BANKSEL	STK00
0004c1   51dd     MOV	0xdd, R0             	MOV	STK00, R0
0004c2   9800     MOV	R0, #0               	MOV	R0,# 0x00
                                           	PAGESEL	_delay_us
0004c3   d6d2     CALL	#0x6d2              	CALL	_delay_us
                                           	PAGESEL	$
                                           ;	op : SEND
                                           ;	op : CALL
                                           ;	.line	239; "../debug_touch.c"	Touch_Delay1;
0004c4   9805     MOV	R0, #0x5             	MOV	R0,# 0x05
0004c5   6503     CLR	0x3, 5               	BANKSEL	STK00
0004c6   51dd     MOV	0xdd, R0             	MOV	STK00, R0
0004c7   9800     MOV	R0, #0               	MOV	R0,# 0x00
                                           	PAGESEL	_delay_us
0004c8   d6d2     CALL	#0x6d2              	CALL	_delay_us
                                           	PAGESEL	$
                                           ;	op : SEND
                                           ;	op : CALL
                                           ;	.line	240; "../debug_touch.c"	Touch_Delay1;
0004c9   9805     MOV	R0, #0x5             	MOV	R0,# 0x05
0004ca   6503     CLR	0x3, 5               	BANKSEL	STK00
0004cb   51dd     MOV	0xdd, R0             	MOV	STK00, R0
0004cc   9800     MOV	R0, #0               	MOV	R0,# 0x00
                                           	PAGESEL	_delay_us
0004cd   d6d2     CALL	#0x6d2              	CALL	_delay_us
                                           	PAGESEL	$
                                           ;	op : GET_VALUE_AT_ADDRESS
                                           ;	.line	243; "../debug_touch.c"	if(DAT_GET_STATE)
0004ce   7805     JB	0x5, 0                	JB	_P0_bits, 0
0004cf   c507     JMP	#0x507               	JMP	_00031_DS_
                                           ;	op : =
                                           ;	.line	245; "../debug_touch.c"	CLK_SET_LOW;
0004d0   6105     CLR	0x5, 1               	CLR	_P0_bits, 1
                                           ;	op : =
                                           ;	.line	246; "../debug_touch.c"	T_buf=0;
0004d1   6503     CLR	0x3, 5               	BANKSEL	_T_buf
0004d2   03a6     CLR	0xa6                 	CLR	_T_buf
                                           ;	op : SEND
                                           ;	op : CALL
                                           ;	.line	247; "../debug_touch.c"	Touch_Delay1;
0004d3   9805     MOV	R0, #0x5             	MOV	R0,# 0x05
                                           	BANKSEL	STK00
0004d4   51dd     MOV	0xdd, R0             	MOV	STK00, R0
0004d5   9800     MOV	R0, #0               	MOV	R0,# 0x00
                                           	PAGESEL	_delay_us
0004d6   d6d2     CALL	#0x6d2              	CALL	_delay_us
                                           	PAGESEL	$
                                           ;	op : =
                                           ;	.line	248; "../debug_touch.c"	for(i_T_D=0;i_T_D<6;i_T_D++)
0004d7   6503     CLR	0x3, 5               	BANKSEL	_i_T_D
0004d8   03a5     CLR	0xa5                 	CLR	_i_T_D
                                           ;	op : LABEL
                                           ;	op : <
                                           ;unsigned compare: left < lit(0x6=6), size=1
                                           _00041_DS_
0004d9   9806     MOV	R0, #0x6             	MOV	R0,# 0x06
                                           	BANKSEL	_i_T_D
0004da   38a5     SUB	R0, 0xa5             	SUB	R0, _i_T_D
                                           ;comparing bytes at offset 0
0004db   7003     JNB	0x3, 0               	JNB	PSW, 0
0004dc   c50d     JMP	#0x50d               	JMP	_00032_DS_
                                           ;	op : =
                                           ;	.line	250; "../debug_touch.c"	CLK_SET_HIGH;
0004dd   6905     SET	0x5, 1               	SET	_P0_bits, 1
                                           ;	op : SEND
                                           ;	op : CALL
                                           ;	.line	251; "../debug_touch.c"	Touch_Delay1;
0004de   9805     MOV	R0, #0x5             	MOV	R0,# 0x05
                                           	BANKSEL	STK00
0004df   51dd     MOV	0xdd, R0             	MOV	STK00, R0
0004e0   9800     MOV	R0, #0               	MOV	R0,# 0x00
                                           	PAGESEL	_delay_us
0004e1   d6d2     CALL	#0x6d2              	CALL	_delay_us
                                           	PAGESEL	$
                                           ;	op : EQ_OP
                                           ;	.line	253; "../debug_touch.c"	if(i_T_D!=5)
0004e2   6503     CLR	0x3, 5               	BANKSEL	_i_T_D
0004e3   0ea5     MOVZ	R0, 0xa5            	MOVZ	R0, _i_T_D
                                           ;	.line	255; "../debug_touch.c"	T_buf=T_buf>>1;
0004e4   a805     XOR	R0, #0x5             	XOR	R0,# 0x05
0004e5   7203     JNB	0x3, 2               	JNB	PSW, 2
0004e6   c4ed     JMP	#0x4ed               	JMP	_00028_DS_
0004e7   6003     CLR	0x3, 0               	CLR	PSW, 0
                                           	BANKSEL	_T_buf
0004e8   11a6     RRC	0xa6                 	RRC	_T_buf
                                           ;	op : GET_VALUE_AT_ADDRESS
                                           ;	.line	256; "../debug_touch.c"	if(DAT_GET_STATE)
0004e9   7805     JB	0x5, 0                	JB	_P0_bits, 0
0004ea   c4fe     JMP	#0x4fe               	JMP	_00029_DS_
                                           ;	op : |
                                           ;	.line	257; "../debug_touch.c"	T_buf=T_buf|0x10;
                                           	BANKSEL	_T_buf
0004eb   6ca6     SET	0xa6, 4              	SET	_T_buf, 4
                                           ;	op : GOTO
0004ec   c4fe     JMP	#0x4fe               	JMP	_00029_DS_
                                           ;	op : LABEL
                                           ;	op : <
                                           ;unsigned compare: left < lit(0x10=16), size=1
                                           _00028_DS_
                                           ;	.line	261; "../debug_touch.c"	if(T_buf<16)   //´«Êä´íÎóµÄ£¬·ÀÏÂ·ÇÓ°ÏìÆäËûÊý¾Ý
0004ed   9810     MOV	R0, #0x10            	MOV	R0,# 0x10
                                           	BANKSEL	_T_buf
0004ee   38a6     SUB	R0, 0xa6             	SUB	R0, _T_buf
                                           ;comparing bytes at offset 0
0004ef   7003     JNB	0x3, 0               	JNB	PSW, 0
0004f0   c4fe     JMP	#0x4fe               	JMP	_00029_DS_
                                           ;	op : GET_VALUE_AT_ADDRESS
                                           ;	.line	263; "../debug_touch.c"	if(DAT_GET_STATE)
0004f1   7805     JB	0x5, 0                	JB	_P0_bits, 0
0004f2   c4f9     JMP	#0x4f9               	JMP	_00023_DS_
                                           ;	op : INLINEASM
                                           	BANKSEL _T_buf
0004f3   50a6     MOV	R0, 0xa6             	MOV R0,_T_buf
0004f4   8080     ADD	R0, #0x80            	ADD R0,#(_TOUCH_CH_TRS_EN+0)
0004f5   9901     MOV	R1, #0x1             	MOV R1,#0x01
0004f6   6d03     SET	0x3, 5               	BANKSEL _TOUCH_CH_TRS_EN
0004f7   f748     ST	[R0], R1              	ST [R0],R1
                                           	
                                           ;	op : GOTO
0004f8   c4fe     JMP	#0x4fe               	JMP	_00029_DS_
                                           ;	op : LABEL
                                           ;	op : INLINEASM
                                           _00023_DS_
                                           	BANKSEL _T_buf
0004f9   50a6     MOV	R0, 0xa6             	MOV R0,_T_buf
0004fa   8080     ADD	R0, #0x80            	ADD R0,#(_TOUCH_CH_TRS_EN+0)
0004fb   9900     MOV	R1, #0               	MOV R1,#0x00
0004fc   6d03     SET	0x3, 5               	BANKSEL _TOUCH_CH_TRS_EN
0004fd   f748     ST	[R0], R1              	ST [R0],R1
                                           	
                                           ;	op : LABEL
                                           ;	op : =
                                           _00029_DS_
                                           ;	.line	289; "../debug_touch.c"	CLK_SET_LOW;
0004fe   6105     CLR	0x5, 1               	CLR	_P0_bits, 1
                                           ;	op : SEND
                                           ;	op : CALL
                                           ;	.line	290; "../debug_touch.c"	Touch_Delay1;
0004ff   9805     MOV	R0, #0x5             	MOV	R0,# 0x05
000500   6503     CLR	0x3, 5               	BANKSEL	STK00
000501   51dd     MOV	0xdd, R0             	MOV	STK00, R0
000502   9800     MOV	R0, #0               	MOV	R0,# 0x00
                                           	PAGESEL	_delay_us
000503   d6d2     CALL	#0x6d2              	CALL	_delay_us
                                           	PAGESEL	$
                                           ;	op : +
                                           ;	.line	248; "../debug_touch.c"	for(i_T_D=0;i_T_D<6;i_T_D++)
000504   6503     CLR	0x3, 5               	BANKSEL	_i_T_D
000505   0ba5     INC	0xa5                 	INC	_i_T_D
                                           ;	op : GOTO
000506   c4d9     JMP	#0x4d9               	JMP	_00041_DS_
                                           ;	op : LABEL
                                           ;	op : =
                                           _00031_DS_
                                           ;	.line	295; "../debug_touch.c"	CLK_SET_LOW;
000507   6105     CLR	0x5, 1               	CLR	_P0_bits, 1
                                           ;	op : SEND
                                           ;	op : CALL
                                           ;	.line	296; "../debug_touch.c"	Touch_Delay1;
000508   9805     MOV	R0, #0x5             	MOV	R0,# 0x05
000509   6503     CLR	0x3, 5               	BANKSEL	STK00
00050a   51dd     MOV	0xdd, R0             	MOV	STK00, R0
00050b   9800     MOV	R0, #0               	MOV	R0,# 0x00
                                           	PAGESEL	_delay_us
00050c   d6d2     CALL	#0x6d2              	CALL	_delay_us
                                           	PAGESEL	$
                                           ;	op : LABEL
                                           ;	op : =
                                           _00032_DS_
                                           ;	.line	299; "../debug_touch.c"	CLK_SET_IN;
00050d   6925     SET	0x25, 1              	SET	_TR0_bits, 1
                                           ;	op : =
                                           ;	.line	300; "../debug_touch.c"	DAT_SET_IN;
00050e   6825     SET	0x25, 0              	SET	_TR0_bits, 0
                                           ;	op : INLINEASM
                                           Label_x_y_z_a:
                                           	
                                           ;	op : LABEL
                                           ;	op : ENDFUNCTION
                                           _00045_DS_
00050f   0008     CRET                     	CRET	
                                           ; exit point of _TOUCH_DEBUG_TRS_DEAL
                                           
                                           
                                           ;	code size estimation:
                                           ;	  420+   91 =   511 instructions ( 1204 byte)
                                           
                                           
                                           	.end
                                           ;--------------------------------------------------------
                                           ; File Created by ChiponCC : aolisn inc.
                                           ; Version 3.0.4#6752 (Jul  6 2017 15:09:47) (MSVC)
                                           ; This file was generated Wed Apr 04 14:53:42 2018
                                           ;--------------------------------------------------------
                                           ; chipon port for the 16-bit core
                                           ;--------------------------------------------------------
                                           ;	.file	"../init_mcu.c"
                                           	.radix dec
                                           	.include "KF8S1024.inc"
                                           
                                           ;************************************************************ 
                                           ;       Header file for the KungFu8 
                                           ;       KF8S1024 
                                           ;       Microcontroller
                                           ; 
                                           ;       Copyright 2012-2013 ChipON, All rights reserved
                                           ;************************************************************ 
                                            
                                           T0                .EQU                0x01
                                           PCL               .EQU                0x02
                                           PSW               .EQU                0x03
                                           P0                .EQU                0x05
                                           P2                .EQU                0x06
                                           P1                .EQU                0x07
                                           P3                .EQU                0x08
                                           PCH               .EQU                0x0A
                                           INTCTL            .EQU                0x0B
                                           EIF1              .EQU                0x0C
                                           T1L               .EQU                0x0E
                                           T1H               .EQU                0x0F
                                           T1CTL             .EQU                0x10
                                           T2                .EQU                0x11
                                           T2CTL             .EQU                0x12
                                           PWMCTL            .EQU                0x15
                                           CMCTL1            .EQU                0x1A
                                           VRECAL            .EQU                0x1C
                                           ADCDATAH          .EQU                0x1E
                                           ADCCTL0           .EQU                0x1F
                                           OPTR              .EQU                0x21
                                           TR0               .EQU                0x25
                                           TR2               .EQU                0x26
                                           TR1               .EQU                0x27
                                           TR3               .EQU                0x28
                                           EIE1              .EQU                0x2C
                                           PCTL              .EQU                0x2E
                                           OSCCTL            .EQU                0x2F
                                           OSCCAL0           .EQU                0x30
                                           ANSEL             .EQU                0x31
                                           PUR               .EQU                0x35
                                           IOCL              .EQU                0x36
                                           OSCCAL1           .EQU                0x37
                                           ADCDATAL          .EQU                0x3E
                                           ADCCTL1           .EQU                0x3F
                                           T3L               .EQU                0x50
                                           CTCTL             .EQU                0x53
                                           T2CCR             .EQU                0x54
                                           OSCLDOCAL         .EQU                0x5E
                                           T1U               .EQU                0x5F
                                            
                                            
                                           
                                           ;Address:0x03 PSW Bits------------------
                                           RP0                .EQU                5
                                           TO                 .EQU                4
                                           PD                 .EQU                3
                                           Z                  .EQU                2
                                           DC                 .EQU                1
                                           CY                 .EQU                0
                                           _RP0               .EQU                5
                                           _TO                .EQU                4
                                           _PD                .EQU                3
                                           _Z                 .EQU                2
                                           _DC                .EQU                1
                                           _CY                .EQU                0
                                           
                                           ;Address:0x05 P0 Bits-------------------
                                           P05                .EQU                5
                                           P04                .EQU                4
                                           P03                .EQU                3
                                           P01                .EQU                1
                                           P00                .EQU                0
                                           _P05               .EQU                5
                                           _P04               .EQU                4
                                           _P03               .EQU                3
                                           _P01               .EQU                1
                                           _P00               .EQU                0
                                           
                                           ;Address:0x06 P2 Bits-------------------
                                           P21                .EQU                1
                                           P20                .EQU                0
                                           _P21               .EQU                1
                                           _P20               .EQU                0
                                           
                                           ;Address:0x07 P1 Bits-------------------
                                           P17                .EQU                7
                                           P16                .EQU                6
                                           P12                .EQU                2
                                           _P17               .EQU                7
                                           _P16               .EQU                6
                                           _P12               .EQU                2
                                           
                                           ;Address:0x08 P3 Bits-------------------
                                           P33                .EQU                3
                                           P32                .EQU                2
                                           P31                .EQU                1
                                           P30                .EQU                0
                                           _P33               .EQU                3
                                           _P32               .EQU                2
                                           _P31               .EQU                1
                                           _P30               .EQU                0
                                           
                                           ;Address:0x0B INTCTL Bits---------------
                                           AIE                .EQU                7
                                           PUIE               .EQU                6
                                           T0IE               .EQU                5
                                           P0IE               .EQU                3
                                           T0IF               .EQU                2
                                           P0IF               .EQU                0
                                           _AIE               .EQU                7
                                           _PUIE              .EQU                6
                                           _T0IE              .EQU                5
                                           _P0IE              .EQU                3
                                           _T0IF              .EQU                2
                                           _P0IF              .EQU                0
                                           
                                           ;Address:0x0C EIF1 Bits-----------------
                                           CTIF               .EQU                7
                                           ADIF               .EQU                6
                                           INT2IF             .EQU                5
                                           INT1IF             .EQU                4
                                           C1IF               .EQU                3
                                           PWM2IF             .EQU                2
                                           T2IF               .EQU                1
                                           T1IF               .EQU                0
                                           _CTIF              .EQU                7
                                           _ADIF              .EQU                6
                                           _INT2IF            .EQU                5
                                           _INT1IF            .EQU                4
                                           _C1IF              .EQU                3
                                           _PWM2IF            .EQU                2
                                           _T2IF              .EQU                1
                                           _T1IF              .EQU                0
                                           
                                           ;Address:0x10 T1CTL Bits----------------
                                           T1GC               .EQU                6
                                           T1CKS1             .EQU                5
                                           T1CKS0             .EQU                4
                                           T1SY               .EQU                2
                                           T1CS               .EQU                1
                                           T1ON               .EQU                0
                                           _T1GC              .EQU                6
                                           _T1CKS1            .EQU                5
                                           _T1CKS0            .EQU                4
                                           _T1SY              .EQU                2
                                           _T1CS              .EQU                1
                                           _T1ON              .EQU                0
                                           
                                           ;Address:0x12 T2CTL Bits----------------
                                           T2CKBS3            .EQU                6
                                           T2CKBS2            .EQU                5
                                           T2CKBS1            .EQU                4
                                           T2CKBS0            .EQU                3
                                           T2ON               .EQU                2
                                           T2CKPS1            .EQU                1
                                           T2CKPS0            .EQU                0
                                           _T2CKBS3           .EQU                6
                                           _T2CKBS2           .EQU                5
                                           _T2CKBS1           .EQU                4
                                           _T2CKBS0           .EQU                3
                                           _T2ON              .EQU                2
                                           _T2CKPS1           .EQU                1
                                           _T2CKPS0           .EQU                0
                                           
                                           ;Address:0x15 PWMCTL Bits---------------
                                           INT1SE             .EQU                6
                                           _INT1SE            .EQU                6
                                           
                                           ;Address:0x1A CMCTL1 Bits---------------
                                           CTCLKSEL1          .EQU                7
                                           CTCLKSEL0          .EQU                6
                                           CTVREFSEL1         .EQU                5
                                           CTVREFSEL0         .EQU                4
                                           _CTCLKSEL1         .EQU                7
                                           _CTCLKSEL0         .EQU                6
                                           _CTVREFSEL1        .EQU                5
                                           _CTVREFSEL0        .EQU                4
                                           
                                           ;Address:0x1F ADCCTL0 Bits--------------
                                           ADLR               .EQU                7
                                           CHS3               .EQU                5
                                           CHS2               .EQU                4
                                           CHS1               .EQU                3
                                           CHS0               .EQU                2
                                           START              .EQU                1
                                           ADEN               .EQU                0
                                           _ADLR              .EQU                7
                                           _CHS3              .EQU                5
                                           _CHS2              .EQU                4
                                           _CHS1              .EQU                3
                                           _CHS0              .EQU                2
                                           _START             .EQU                1
                                           _ADEN              .EQU                0
                                           
                                           ;Address:0x21 OPTR Bits-----------------
                                           PUPH               .EQU                7
                                           T0CS               .EQU                5
                                           T0SE               .EQU                4
                                           PSA                .EQU                3
                                           PS2                .EQU                2
                                           PS1                .EQU                1
                                           PS0                .EQU                0
                                           _PUPH              .EQU                7
                                           _T0CS              .EQU                5
                                           _T0SE              .EQU                4
                                           _PSA               .EQU                3
                                           _PS2               .EQU                2
                                           _PS1               .EQU                1
                                           _PS0               .EQU                0
                                           
                                           ;Address:0x25 TR0 Bits------------------
                                           TR05               .EQU                5
                                           TR04               .EQU                4
                                           TR03               .EQU                3
                                           TR01               .EQU                1
                                           TR00               .EQU                0
                                           _TR05              .EQU                5
                                           _TR04              .EQU                4
                                           _TR03              .EQU                3
                                           _TR01              .EQU                1
                                           _TR00              .EQU                0
                                           
                                           ;Address:0x26 TR2 Bits------------------
                                           TR21               .EQU                1
                                           TR20               .EQU                0
                                           _TR21              .EQU                1
                                           _TR20              .EQU                0
                                           
                                           ;Address:0x27 TR1 Bits------------------
                                           TR17               .EQU                7
                                           TR16               .EQU                6
                                           TR12               .EQU                2
                                           _TR17              .EQU                7
                                           _TR16              .EQU                6
                                           _TR12              .EQU                2
                                           
                                           ;Address:0x28 TR3 Bits------------------
                                           TR33               .EQU                3
                                           TR32               .EQU                2
                                           TR31               .EQU                1
                                           TR30               .EQU                0
                                           _TR33              .EQU                3
                                           _TR32              .EQU                2
                                           _TR31              .EQU                1
                                           _TR30              .EQU                0
                                           
                                           ;Address:0x2C EIE1 Bits-----------------
                                           CTIE               .EQU                7
                                           ADIE               .EQU                6
                                           INT2IE             .EQU                5
                                           INT1IE             .EQU                4
                                           C1IE               .EQU                3
                                           PWM2IE             .EQU                2
                                           T2IE               .EQU                1
                                           T1IE               .EQU                0
                                           _CTIE              .EQU                7
                                           _ADIE              .EQU                6
                                           _INT2IE            .EQU                5
                                           _INT1IE            .EQU                4
                                           _C1IE              .EQU                3
                                           _PWM2IE            .EQU                2
                                           _T2IE              .EQU                1
                                           _T1IE              .EQU                0
                                           
                                           ;Address:0x2E PCTL Bits-----------------
                                           VREEN              .EQU                7
                                           VREOE              .EQU                6
                                           SLVREN             .EQU                4
                                           POR                .EQU                1
                                           LVR                .EQU                0
                                           _VREEN             .EQU                7
                                           _VREOE             .EQU                6
                                           _SLVREN            .EQU                4
                                           _POR               .EQU                1
                                           _LVR               .EQU                0
                                           
                                           ;Address:0x2F OSCCTL Bits---------------
                                           CKOEN              .EQU                7
                                           IRCS2              .EQU                6
                                           IRCS1              .EQU                5
                                           IRCS0              .EQU                4
                                           _CKOEN             .EQU                7
                                           _IRCS2             .EQU                6
                                           _IRCS1             .EQU                5
                                           _IRCS0             .EQU                4
                                           
                                           ;Address:0x31 ANSEL Bits----------------
                                           ANS6               .EQU                6
                                           ANS3               .EQU                3
                                           ANS1               .EQU                1
                                           _ANS6              .EQU                6
                                           _ANS3              .EQU                3
                                           _ANS1              .EQU                1
                                           
                                           ;Address:0x35 PUR Bits------------------
                                           PUR5               .EQU                5
                                           PUR4               .EQU                4
                                           PUR2               .EQU                2
                                           PUR1               .EQU                1
                                           PUR0               .EQU                0
                                           _PUR5              .EQU                5
                                           _PUR4              .EQU                4
                                           _PUR2              .EQU                2
                                           _PUR1              .EQU                1
                                           _PUR0              .EQU                0
                                           
                                           ;Address:0x36 IOCL Bits-----------------
                                           IOCL5              .EQU                5
                                           IOCL4              .EQU                4
                                           IOCL3              .EQU                3
                                           IOCL2              .EQU                2
                                           IOCL1              .EQU                1
                                           IOCL0              .EQU                0
                                           _IOCL5             .EQU                5
                                           _IOCL4             .EQU                4
                                           _IOCL3             .EQU                3
                                           _IOCL2             .EQU                2
                                           _IOCL1             .EQU                1
                                           _IOCL0             .EQU                0
                                           
                                           ;Address:0x3F ADCCTL1 Bits--------------
                                           ADCS2              .EQU                6
                                           ADCS1              .EQU                5
                                           ADCS0              .EQU                4
                                           VCFG1              .EQU                3
                                           VCFG0              .EQU                2
                                           _ADCS2             .EQU                6
                                           _ADCS1             .EQU                5
                                           _ADCS0             .EQU                4
                                           _VCFG1             .EQU                3
                                           _VCFG0             .EQU                2
                                           
                                           ;Address:0x50 T3L Bits------------------
                                           T3L7               .EQU                7
                                           T3L6               .EQU                6
                                           T3L5               .EQU                5
                                           T3L4               .EQU                4
                                           T3L3               .EQU                3
                                           T3L2               .EQU                2
                                           T3L1               .EQU                1
                                           T3L0               .EQU                0
                                           _T3L7              .EQU                7
                                           _T3L6              .EQU                6
                                           _T3L5              .EQU                5
                                           _T3L4              .EQU                4
                                           _T3L3              .EQU                3
                                           _T3L2              .EQU                2
                                           _T3L1              .EQU                1
                                           _T3L0              .EQU                0
                                           
                                           ;Address:0x53 CTCTL Bits----------------
                                           CTEN               .EQU                7
                                           CTSTART            .EQU                6
                                           CTCAPS             .EQU                5
                                           CTCMS              .EQU                4
                                           CTCHSEL4           .EQU                4
                                           CTCHSEL3           .EQU                3
                                           CTCHSEL2           .EQU                2
                                           CTCHSEL1           .EQU                1
                                           CTCHSEL0           .EQU                0
                                           _CTEN              .EQU                7
                                           _CTSTART           .EQU                6
                                           _CTCAPS            .EQU                5
                                           _CTCMS             .EQU                4
                                           _CTCHSEL4          .EQU                4
                                           _CTCHSEL3          .EQU                3
                                           _CTCHSEL2          .EQU                2
                                           _CTCHSEL1          .EQU                1
                                           _CTCHSEL0          .EQU                0
                                           
                                           ;Address:0x5E OSCLDOCAL Bits------------
                                            
                                            
                                           ;--------------------------------------------------------
                                           ; external declarations
                                           ;--------------------------------------------------------
                                           	.extern	_PSW_bits
                                           	.extern	_P0_bits
                                           	.extern	_P2_bits
                                           	.extern	_P1_bits
                                           	.extern	_P3_bits
                                           	.extern	_INTCTL_bits
                                           	.extern	_EIF1_bits
                                           	.extern	_T1CTL_bits
                                           	.extern	_T2CTL_bits
                                           	.extern	_PWMCTL_bits
                                           	.extern	_CMCTL1_bits
                                           	.extern	_ADCCTL0_bits
                                           	.extern	_OPTR_bits
                                           	.extern	_TR0_bits
                                           	.extern	_TR2_bits
                                           	.extern	_TR1_bits
                                           	.extern	_TR3_bits
                                           	.extern	_EIE1_bits
                                           	.extern	_PCTL_bits
                                           	.extern	_OSCCTL_bits
                                           	.extern	_ANSEL_bits
                                           	.extern	_PUR_bits
                                           	.extern	_IOCL_bits
                                           	.extern	_ADCCTL1_bits
                                           	.extern	_T3L_bits
                                           	.extern	_CTCTL_bits
                                           	.extern	_OSCLDOCAL_bits
                                           	.extern	_T0
                                           	.extern	_PCL
                                           	.extern	_PSW
                                           	.extern	_P0
                                           	.extern	_P2
                                           	.extern	_P1
                                           	.extern	_P3
                                           	.extern	_PCH
                                           	.extern	_INTCTL
                                           	.extern	_EIF1
                                           	.extern	_T1L
                                           	.extern	_T1H
                                           	.extern	_T1CTL
                                           	.extern	_T2
                                           	.extern	_T2CTL
                                           	.extern	_PWMCTL
                                           	.extern	_CMCTL1
                                           	.extern	_VRECAL
                                           	.extern	_ADCDATAH
                                           	.extern	_ADCCTL0
                                           	.extern	_OPTR
                                           	.extern	_TR0
                                           	.extern	_TR2
                                           	.extern	_TR1
                                           	.extern	_TR3
                                           	.extern	_EIE1
                                           	.extern	_PCTL
                                           	.extern	_OSCCTL
                                           	.extern	_OSCCAL0
                                           	.extern	_ANSEL
                                           	.extern	_PUR
                                           	.extern	_IOCL
                                           	.extern	_OSCCAL1
                                           	.extern	_ADCDATAL
                                           	.extern	_ADCCTL1
                                           	.extern	_T3L
                                           	.extern	_CTCTL
                                           	.extern	_T2CCR
                                           	.extern	_OSCLDOCAL
                                           	.extern	_T1U
                                           
                                           	.extern STK12
                                           	.extern STK11
                                           	.extern STK10
                                           	.extern STK09
                                           	.extern STK08
                                           	.extern STK07
                                           	.extern STK06
                                           	.extern STK05
                                           	.extern STK04
                                           	.extern STK03
                                           	.extern STK02
                                           	.extern STK01
                                           	.extern STK00
                                           ;--------------------------------------------------------
                                           ; global declarations
                                           ;--------------------------------------------------------
                                           	.global	_init_mcu
                                           
                                           ;--------------------------------------------------------
                                           ; global definitions
                                           ;--------------------------------------------------------
                                           ;--------------------------------------------------------
                                           ; absolute symbol definitions
                                           ;--------------------------------------------------------
                                           ;--------------------------------------------------------
                                           ; compiler-defined variables
                                           ;--------------------------------------------------------
                                           ;--------------------------------------------------------
                                           ; initialized data
                                           ;--------------------------------------------------------
                                           ;--------------------------------------------------------
                                           ; overlayable items in internal ram 
                                           ;--------------------------------------------------------
                                           ;	.udata_ovr
                                           
                                           
                                           func._init_mcu	.code
                                           ;***
                                           ;  PostBlock Stats: dbName = C
                                           ;***
                                           ;entry:  _init_mcu	;Function start
                                           ; 2 exit points
                                           ;has an exit
                                           ;; Starting PostCode block
                                           ;	op : LABEL
                                           ;	op : FUNCTION
                                           _init_mcu	;Function start
                                           ; 2 exit points
                                           ;	op : =
                                           ;	.line	17; "../init_mcu.c"	OSCCTL = 0x60;           //8M
0006ae   9860     MOV	R0, #0x60            	MOV	R0,# 0x60
0006af   512f     MOV	0x2f, R0             	MOV	_OSCCTL, R0
                                           ;	op : =
                                           ;	.line	20; "../init_mcu.c"	TR0 = 0XEF;              //1111 1111		£¡£¡¡¶¡¶×¢Òâµã:TR0.7ÕâÒ»Î»±ØÐëÉèÖÃÎª1£¬ÊäÈëÌ¬¡·¡·£¡£¡
0006b0   98ef     MOV	R0, #0xef            	MOV	R0,# 0xef
0006b1   5125     MOV	0x25, R0             	MOV	_TR0, R0
                                           ;	op : =
                                           ;	.line	21; "../init_mcu.c"	TR1 = 0XFF;              //1111 1111		P16,P17´¥ÃþÍ¨µÀ2,3  ÉèÖÃIO¿ÚÎªÊäÈë
0006b2   98ff     MOV	R0, #0xff            	MOV	R0,# 0xff
0006b3   5127     MOV	0x27, R0             	MOV	_TR1, R0
                                           ;	op : =
                                           ;	.line	22; "../init_mcu.c"	TR2 = 0XFF;              //1111 1111		P20,P21´¥ÃþÍ¨µÀ4,5  ÉèÖÃIO¿ÚÎªÊäÈë
0006b4   98ff     MOV	R0, #0xff            	MOV	R0,# 0xff
0006b5   5126     MOV	0x26, R0             	MOV	_TR2, R0
                                           ;	op : =
                                           ;	.line	24; "../init_mcu.c"	P0 = 0X00;               //0000 0000
0006b6   0305     CLR	0x5                  	CLR	_P0
                                           ;	op : =
                                           ;	.line	25; "../init_mcu.c"	P1 = 0X00;               //0000 0000
0006b7   0307     CLR	0x7                  	CLR	_P1
                                           ;	op : =
                                           ;	.line	26; "../init_mcu.c"	P2 = 0x00;               //0000 0000
0006b8   0306     CLR	0x6                  	CLR	_P2
                                           ;	op : |
                                           ;	.line	28; "../init_mcu.c"	ANSEL |= 1<<6;			 //ÉèÖÃAN6ÎªÄ£Äâ¿Ú,Íâ¹ÒµçÈÝ½ÅÉèÖÃÎªÄ£Äâ¿Ú
0006b9   6e31     SET	0x31, 6              	SET	_ANSEL, 6
                                           ;	op : =
                                           ;	.line	31; "../init_mcu.c"	T1CTL = 0X00;    		 //1£º1·ÖÆµ£¬²»¿ªÆô¼ÆÊýÆ÷T1
0006ba   0310     CLR	0x10                 	CLR	_T1CTL
                                           ;	op : =
                                           ;	.line	32; "../init_mcu.c"	T1L = 0;
0006bb   030e     CLR	0xe                  	CLR	_T1L
                                           ;	op : =
                                           ;	.line	33; "../init_mcu.c"	T1H = 0;
0006bc   030f     CLR	0xf                  	CLR	_T1H
                                           ;	op : =
                                           ;	.line	34; "../init_mcu.c"	T1IF = 0;
0006bd   600c     CLR	0xc, 0               	CLR	_EIF1_bits, 0
                                           ;	op : =
                                           ;	.line	35; "../init_mcu.c"	AIE = 0;
0006be   670b     CLR	0xb, 7               	CLR	_INTCTL_bits, 7
                                           ;	op : LABEL
                                           ;	op : ENDFUNCTION
0006bf   0008     CRET                     	CRET	
                                           ; exit point of _init_mcu
                                           
                                           
                                           ;	code size estimation:
                                           ;	   18+    0 =    18 instructions (   36 byte)
                                           
                                           
                                           	.end
                                           ;--------------------------------------------------------
                                           ; File Created by ChiponCC : aolisn inc.
                                           ; Version 3.0.4#6752 (Jul  6 2017 15:09:47) (MSVC)
                                           ; This file was generated Wed Apr 04 14:53:43 2018
                                           ;--------------------------------------------------------
                                           ; chipon port for the 16-bit core
                                           ;--------------------------------------------------------
                                           ;	.file	"../kf8s_touch_g.c"
                                           	.radix dec
                                           	.include "KF8S1024.inc"
                                           
                                           ;************************************************************ 
                                           ;       Header file for the KungFu8 
                                           ;       KF8S1024 
                                           ;       Microcontroller
                                           ; 
                                           ;       Copyright 2012-2013 ChipON, All rights reserved
                                           ;************************************************************ 
                                            
                                           T0                .EQU                0x01
                                           PCL               .EQU                0x02
                                           PSW               .EQU                0x03
                                           P0                .EQU                0x05
                                           P2                .EQU                0x06
                                           P1                .EQU                0x07
                                           P3                .EQU                0x08
                                           PCH               .EQU                0x0A
                                           INTCTL            .EQU                0x0B
                                           EIF1              .EQU                0x0C
                                           T1L               .EQU                0x0E
                                           T1H               .EQU                0x0F
                                           T1CTL             .EQU                0x10
                                           T2                .EQU                0x11
                                           T2CTL             .EQU                0x12
                                           PWMCTL            .EQU                0x15
                                           CMCTL1            .EQU                0x1A
                                           VRECAL            .EQU                0x1C
                                           ADCDATAH          .EQU                0x1E
                                           ADCCTL0           .EQU                0x1F
                                           OPTR              .EQU                0x21
                                           TR0               .EQU                0x25
                                           TR2               .EQU                0x26
                                           TR1               .EQU                0x27
                                           TR3               .EQU                0x28
                                           EIE1              .EQU                0x2C
                                           PCTL              .EQU                0x2E
                                           OSCCTL            .EQU                0x2F
                                           OSCCAL0           .EQU                0x30
                                           ANSEL             .EQU                0x31
                                           PUR               .EQU                0x35
                                           IOCL              .EQU                0x36
                                           OSCCAL1           .EQU                0x37
                                           ADCDATAL          .EQU                0x3E
                                           ADCCTL1           .EQU                0x3F
                                           T3L               .EQU                0x50
                                           CTCTL             .EQU                0x53
                                           T2CCR             .EQU                0x54
                                           OSCLDOCAL         .EQU                0x5E
                                           T1U               .EQU                0x5F
                                            
                                            
                                           
                                           ;Address:0x03 PSW Bits------------------
                                           RP0                .EQU                5
                                           TO                 .EQU                4
                                           PD                 .EQU                3
                                           Z                  .EQU                2
                                           DC                 .EQU                1
                                           CY                 .EQU                0
                                           _RP0               .EQU                5
                                           _TO                .EQU                4
                                           _PD                .EQU                3
                                           _Z                 .EQU                2
                                           _DC                .EQU                1
                                           _CY                .EQU                0
                                           
                                           ;Address:0x05 P0 Bits-------------------
                                           P05                .EQU                5
                                           P04                .EQU                4
                                           P03                .EQU                3
                                           P01                .EQU                1
                                           P00                .EQU                0
                                           _P05               .EQU                5
                                           _P04               .EQU                4
                                           _P03               .EQU                3
                                           _P01               .EQU                1
                                           _P00               .EQU                0
                                           
                                           ;Address:0x06 P2 Bits-------------------
                                           P21                .EQU                1
                                           P20                .EQU                0
                                           _P21               .EQU                1
                                           _P20               .EQU                0
                                           
                                           ;Address:0x07 P1 Bits-------------------
                                           P17                .EQU                7
                                           P16                .EQU                6
                                           P12                .EQU                2
                                           _P17               .EQU                7
                                           _P16               .EQU                6
                                           _P12               .EQU                2
                                           
                                           ;Address:0x08 P3 Bits-------------------
                                           P33                .EQU                3
                                           P32                .EQU                2
                                           P31                .EQU                1
                                           P30                .EQU                0
                                           _P33               .EQU                3
                                           _P32               .EQU                2
                                           _P31               .EQU                1
                                           _P30               .EQU                0
                                           
                                           ;Address:0x0B INTCTL Bits---------------
                                           AIE                .EQU                7
                                           PUIE               .EQU                6
                                           T0IE               .EQU                5
                                           P0IE               .EQU                3
                                           T0IF               .EQU                2
                                           P0IF               .EQU                0
                                           _AIE               .EQU                7
                                           _PUIE              .EQU                6
                                           _T0IE              .EQU                5
                                           _P0IE              .EQU                3
                                           _T0IF              .EQU                2
                                           _P0IF              .EQU                0
                                           
                                           ;Address:0x0C EIF1 Bits-----------------
                                           CTIF               .EQU                7
                                           ADIF               .EQU                6
                                           INT2IF             .EQU                5
                                           INT1IF             .EQU                4
                                           C1IF               .EQU                3
                                           PWM2IF             .EQU                2
                                           T2IF               .EQU                1
                                           T1IF               .EQU                0
                                           _CTIF              .EQU                7
                                           _ADIF              .EQU                6
                                           _INT2IF            .EQU                5
                                           _INT1IF            .EQU                4
                                           _C1IF              .EQU                3
                                           _PWM2IF            .EQU                2
                                           _T2IF              .EQU                1
                                           _T1IF              .EQU                0
                                           
                                           ;Address:0x10 T1CTL Bits----------------
                                           T1GC               .EQU                6
                                           T1CKS1             .EQU                5
                                           T1CKS0             .EQU                4
                                           T1SY               .EQU                2
                                           T1CS               .EQU                1
                                           T1ON               .EQU                0
                                           _T1GC              .EQU                6
                                           _T1CKS1            .EQU                5
                                           _T1CKS0            .EQU                4
                                           _T1SY              .EQU                2
                                           _T1CS              .EQU                1
                                           _T1ON              .EQU                0
                                           
                                           ;Address:0x12 T2CTL Bits----------------
                                           T2CKBS3            .EQU                6
                                           T2CKBS2            .EQU                5
                                           T2CKBS1            .EQU                4
                                           T2CKBS0            .EQU                3
                                           T2ON               .EQU                2
                                           T2CKPS1            .EQU                1
                                           T2CKPS0            .EQU                0
                                           _T2CKBS3           .EQU                6
                                           _T2CKBS2           .EQU                5
                                           _T2CKBS1           .EQU                4
                                           _T2CKBS0           .EQU                3
                                           _T2ON              .EQU                2
                                           _T2CKPS1           .EQU                1
                                           _T2CKPS0           .EQU                0
                                           
                                           ;Address:0x15 PWMCTL Bits---------------
                                           INT1SE             .EQU                6
                                           _INT1SE            .EQU                6
                                           
                                           ;Address:0x1A CMCTL1 Bits---------------
                                           CTCLKSEL1          .EQU                7
                                           CTCLKSEL0          .EQU                6
                                           CTVREFSEL1         .EQU                5
                                           CTVREFSEL0         .EQU                4
                                           _CTCLKSEL1         .EQU                7
                                           _CTCLKSEL0         .EQU                6
                                           _CTVREFSEL1        .EQU                5
                                           _CTVREFSEL0        .EQU                4
                                           
                                           ;Address:0x1F ADCCTL0 Bits--------------
                                           ADLR               .EQU                7
                                           CHS3               .EQU                5
                                           CHS2               .EQU                4
                                           CHS1               .EQU                3
                                           CHS0               .EQU                2
                                           START              .EQU                1
                                           ADEN               .EQU                0
                                           _ADLR              .EQU                7
                                           _CHS3              .EQU                5
                                           _CHS2              .EQU                4
                                           _CHS1              .EQU                3
                                           _CHS0              .EQU                2
                                           _START             .EQU                1
                                           _ADEN              .EQU                0
                                           
                                           ;Address:0x21 OPTR Bits-----------------
                                           PUPH               .EQU                7
                                           T0CS               .EQU                5
                                           T0SE               .EQU                4
                                           PSA                .EQU                3
                                           PS2                .EQU                2
                                           PS1                .EQU                1
                                           PS0                .EQU                0
                                           _PUPH              .EQU                7
                                           _T0CS              .EQU                5
                                           _T0SE              .EQU                4
                                           _PSA               .EQU                3
                                           _PS2               .EQU                2
                                           _PS1               .EQU                1
                                           _PS0               .EQU                0
                                           
                                           ;Address:0x25 TR0 Bits------------------
                                           TR05               .EQU                5
                                           TR04               .EQU                4
                                           TR03               .EQU                3
                                           TR01               .EQU                1
                                           TR00               .EQU                0
                                           _TR05              .EQU                5
                                           _TR04              .EQU                4
                                           _TR03              .EQU                3
                                           _TR01              .EQU                1
                                           _TR00              .EQU                0
                                           
                                           ;Address:0x26 TR2 Bits------------------
                                           TR21               .EQU                1
                                           TR20               .EQU                0
                                           _TR21              .EQU                1
                                           _TR20              .EQU                0
                                           
                                           ;Address:0x27 TR1 Bits------------------
                                           TR17               .EQU                7
                                           TR16               .EQU                6
                                           TR12               .EQU                2
                                           _TR17              .EQU                7
                                           _TR16              .EQU                6
                                           _TR12              .EQU                2
                                           
                                           ;Address:0x28 TR3 Bits------------------
                                           TR33               .EQU                3
                                           TR32               .EQU                2
                                           TR31               .EQU                1
                                           TR30               .EQU                0
                                           _TR33              .EQU                3
                                           _TR32              .EQU                2
                                           _TR31              .EQU                1
                                           _TR30              .EQU                0
                                           
                                           ;Address:0x2C EIE1 Bits-----------------
                                           CTIE               .EQU                7
                                           ADIE               .EQU                6
                                           INT2IE             .EQU                5
                                           INT1IE             .EQU                4
                                           C1IE               .EQU                3
                                           PWM2IE             .EQU                2
                                           T2IE               .EQU                1
                                           T1IE               .EQU                0
                                           _CTIE              .EQU                7
                                           _ADIE              .EQU                6
                                           _INT2IE            .EQU                5
                                           _INT1IE            .EQU                4
                                           _C1IE              .EQU                3
                                           _PWM2IE            .EQU                2
                                           _T2IE              .EQU                1
                                           _T1IE              .EQU                0
                                           
                                           ;Address:0x2E PCTL Bits-----------------
                                           VREEN              .EQU                7
                                           VREOE              .EQU                6
                                           SLVREN             .EQU                4
                                           POR                .EQU                1
                                           LVR                .EQU                0
                                           _VREEN             .EQU                7
                                           _VREOE             .EQU                6
                                           _SLVREN            .EQU                4
                                           _POR               .EQU                1
                                           _LVR               .EQU                0
                                           
                                           ;Address:0x2F OSCCTL Bits---------------
                                           CKOEN              .EQU                7
                                           IRCS2              .EQU                6
                                           IRCS1              .EQU                5
                                           IRCS0              .EQU                4
                                           _CKOEN             .EQU                7
                                           _IRCS2             .EQU                6
                                           _IRCS1             .EQU                5
                                           _IRCS0             .EQU                4
                                           
                                           ;Address:0x31 ANSEL Bits----------------
                                           ANS6               .EQU                6
                                           ANS3               .EQU                3
                                           ANS1               .EQU                1
                                           _ANS6              .EQU                6
                                           _ANS3              .EQU                3
                                           _ANS1              .EQU                1
                                           
                                           ;Address:0x35 PUR Bits------------------
                                           PUR5               .EQU                5
                                           PUR4               .EQU                4
                                           PUR2               .EQU                2
                                           PUR1               .EQU                1
                                           PUR0               .EQU                0
                                           _PUR5              .EQU                5
                                           _PUR4              .EQU                4
                                           _PUR2              .EQU                2
                                           _PUR1              .EQU                1
                                           _PUR0              .EQU                0
                                           
                                           ;Address:0x36 IOCL Bits-----------------
                                           IOCL5              .EQU                5
                                           IOCL4              .EQU                4
                                           IOCL3              .EQU                3
                                           IOCL2              .EQU                2
                                           IOCL1              .EQU                1
                                           IOCL0              .EQU                0
                                           _IOCL5             .EQU                5
                                           _IOCL4             .EQU                4
                                           _IOCL3             .EQU                3
                                           _IOCL2             .EQU                2
                                           _IOCL1             .EQU                1
                                           _IOCL0             .EQU                0
                                           
                                           ;Address:0x3F ADCCTL1 Bits--------------
                                           ADCS2              .EQU                6
                                           ADCS1              .EQU                5
                                           ADCS0              .EQU                4
                                           VCFG1              .EQU                3
                                           VCFG0              .EQU                2
                                           _ADCS2             .EQU                6
                                           _ADCS1             .EQU                5
                                           _ADCS0             .EQU                4
                                           _VCFG1             .EQU                3
                                           _VCFG0             .EQU                2
                                           
                                           ;Address:0x50 T3L Bits------------------
                                           T3L7               .EQU                7
                                           T3L6               .EQU                6
                                           T3L5               .EQU                5
                                           T3L4               .EQU                4
                                           T3L3               .EQU                3
                                           T3L2               .EQU                2
                                           T3L1               .EQU                1
                                           T3L0               .EQU                0
                                           _T3L7              .EQU                7
                                           _T3L6              .EQU                6
                                           _T3L5              .EQU                5
                                           _T3L4              .EQU                4
                                           _T3L3              .EQU                3
                                           _T3L2              .EQU                2
                                           _T3L1              .EQU                1
                                           _T3L0              .EQU                0
                                           
                                           ;Address:0x53 CTCTL Bits----------------
                                           CTEN               .EQU                7
                                           CTSTART            .EQU                6
                                           CTCAPS             .EQU                5
                                           CTCMS              .EQU                4
                                           CTCHSEL4           .EQU                4
                                           CTCHSEL3           .EQU                3
                                           CTCHSEL2           .EQU                2
                                           CTCHSEL1           .EQU                1
                                           CTCHSEL0           .EQU                0
                                           _CTEN              .EQU                7
                                           _CTSTART           .EQU                6
                                           _CTCAPS            .EQU                5
                                           _CTCMS             .EQU                4
                                           _CTCHSEL4          .EQU                4
                                           _CTCHSEL3          .EQU                3
                                           _CTCHSEL2          .EQU                2
                                           _CTCHSEL1          .EQU                1
                                           _CTCHSEL0          .EQU                0
                                           
                                           ;Address:0x5E OSCLDOCAL Bits------------
                                            
                                            
                                           ;--------------------------------------------------------
                                           ; external declarations
                                           ;--------------------------------------------------------
                                           	.extern	_init_mcu
                                           	.extern	__KF8S_Get_Ver_General_
                                           	.extern	__KF8S_Lib_Set_General_Parameter
                                           	.extern	__KF8S_Init_Touch_General_
                                           	.extern	__KF8S_Touch_Process_General_
                                           	.extern	__KF8S_Touch_TEST_General_
                                           	.extern	__R2PCL
                                           	.extern	_TOUCH_DEBUG_TRS_DEAL
                                           	.extern	_TOUCH_DEBUG_SEND_OUT
                                           	.extern	_delay_ms
                                           	.extern	_delay_us
                                           	.extern	_PSW_bits
                                           	.extern	_P0_bits
                                           	.extern	_P2_bits
                                           	.extern	_P1_bits
                                           	.extern	_P3_bits
                                           	.extern	_INTCTL_bits
                                           	.extern	_EIF1_bits
                                           	.extern	_T1CTL_bits
                                           	.extern	_T2CTL_bits
                                           	.extern	_PWMCTL_bits
                                           	.extern	_CMCTL1_bits
                                           	.extern	_ADCCTL0_bits
                                           	.extern	_OPTR_bits
                                           	.extern	_TR0_bits
                                           	.extern	_TR2_bits
                                           	.extern	_TR1_bits
                                           	.extern	_TR3_bits
                                           	.extern	_EIE1_bits
                                           	.extern	_PCTL_bits
                                           	.extern	_OSCCTL_bits
                                           	.extern	_ANSEL_bits
                                           	.extern	_PUR_bits
                                           	.extern	_IOCL_bits
                                           	.extern	_ADCCTL1_bits
                                           	.extern	_T3L_bits
                                           	.extern	_CTCTL_bits
                                           	.extern	_OSCLDOCAL_bits
                                           	.extern	__KF8_LIBc_channel_Buf
                                           	.extern	_sentbuf1
                                           	.extern	_sentbuf2
                                           	.extern	_sentbuf3
                                           	.extern	_sentbuf4
                                           	.extern	_T0
                                           	.extern	_PCL
                                           	.extern	_PSW
                                           	.extern	_P0
                                           	.extern	_P2
                                           	.extern	_P1
                                           	.extern	_P3
                                           	.extern	_PCH
                                           	.extern	_INTCTL
                                           	.extern	_EIF1
                                           	.extern	_T1L
                                           	.extern	_T1H
                                           	.extern	_T1CTL
                                           	.extern	_T2
                                           	.extern	_T2CTL
                                           	.extern	_PWMCTL
                                           	.extern	_CMCTL1
                                           	.extern	_VRECAL
                                           	.extern	_ADCDATAH
                                           	.extern	_ADCCTL0
                                           	.extern	_OPTR
                                           	.extern	_TR0
                                           	.extern	_TR2
                                           	.extern	_TR1
                                           	.extern	_TR3
                                           	.extern	_EIE1
                                           	.extern	_PCTL
                                           	.extern	_OSCCTL
                                           	.extern	_OSCCAL0
                                           	.extern	_ANSEL
                                           	.extern	_PUR
                                           	.extern	_IOCL
                                           	.extern	_OSCCAL1
                                           	.extern	_ADCDATAL
                                           	.extern	_ADCCTL1
                                           	.extern	_T3L
                                           	.extern	_CTCTL
                                           	.extern	_T2CCR
                                           	.extern	_OSCLDOCAL
                                           	.extern	_T1U
                                           
                                           	.extern STK12
                                           	.extern STK11
                                           	.extern STK10
                                           	.extern STK09
                                           	.extern STK08
                                           	.extern STK07
                                           	.extern STK06
                                           	.extern STK05
                                           	.extern STK04
                                           	.extern STK03
                                           	.extern STK02
                                           	.extern STK01
                                           	.extern STK00
                                           ;--------------------------------------------------------
                                           ; global declarations
                                           ;--------------------------------------------------------
                                           	.global	__KF8_LIBc_baseline_count_
                                           	.global	__KF8_LIBi_buff_hit_
                                           	.global	__KF8_LIBi_buff_baseline_
                                           	.global	__KF8_LIBc_touch_count_
                                           	.global	__KF8_LIBi_Date_Change_
                                           	.global	__KF8_LIBc_channel_
                                           	.global	__KF8_LIBi_channel_flag_
                                           	.global	_CHS_AMOUNT
                                           	.global	_TCS_AMOUNT
                                           	.global	__KF8_Disturb_Protect_Circle_
                                           	.global	__KF8_DoubleKey_Compages_Limitable_Circle_
                                           	.global	__KF8_Key_Max_Pressed_Limitable_Circle_
                                           	.global	__KF8_BaseLine_Update_Circle_Count_For_UP_
                                           	.global	__KF8_BaseLine_Update_Circle_Count_For_Down_
                                           	.global	__KF8_Define_Disturb_Channels_Amount_
                                           	.global	__KF8_BasicLine_UP_Noise_Threshold_
                                           	.global	__KF8_BasicLine_Down_Noise_Threshold_
                                           	.global	__KF8_Data_Steady_Threshold_Set_
                                           	.global	__KF8_Inside_Reference_Channel_Disturb_Threshold_Set_
                                           	.global	__KF8_TOUCH_CH_EN
                                           	.global	__KF8_Inside_Reference_Channel_Declare_
                                           	.global	__KF8_Config_Finger_Threshold
                                           
                                           ;--------------------------------------------------------
                                           ; global definitions
                                           ;--------------------------------------------------------
                                           UD_kf8s_touch_g_0	.udata
                                           __KF8_LIBc_baseline_count_	.res	8
                                           
                                           UD_kf8s_touch_g_1	.udata
                                           __KF8_LIBi_buff_hit_	.res	16
                                           
                                           UD_kf8s_touch_g_2	.udata
                                           __KF8_LIBi_buff_baseline_	.res	16
                                           
                                           UD_kf8s_touch_g_3	.udata
                                           __KF8_LIBc_touch_count_	.res	8
                                           
                                           UD_kf8s_touch_g_4	.udata
                                           __KF8_LIBi_Date_Change_	.res	8
                                           
                                           UD_kf8s_touch_g_5	.udata
                                           __KF8_LIBc_channel_	.res	1
                                           
                                           UD_kf8s_touch_g_6	.udata
                                           __KF8_LIBi_channel_flag_	.res	2
                                           
                                           ;--------------------------------------------------------
                                           ; absolute symbol definitions
                                           ;--------------------------------------------------------
                                           ;--------------------------------------------------------
                                           ; compiler-defined variables
                                           ;--------------------------------------------------------
                                           ;--------------------------------------------------------
                                           ; initialized data
                                           ;--------------------------------------------------------
                                           
                                           ID_kf8s_touch_g_0	.code
                                           _CHS_AMOUNT
000711   b008     RRET	R0, #0x8            	RRET R0, #0x08
                                           
                                           
                                           ID_kf8s_touch_g_1	.code
                                           _TCS_AMOUNT
000712   b005     RRET	R0, #0x5            	RRET R0, #0x05
                                           
                                           
                                           ID_kf8s_touch_g_2	.code
                                           __KF8_Disturb_Protect_Circle_
000713   b064     RRET	R0, #0x64           	RRET R0, #0x64
                                           
                                           
                                           ID_kf8s_touch_g_3	.code
                                           __KF8_DoubleKey_Compages_Limitable_Circle_
000002   b02c     RRET	R0, #0x2c           	RRET R0, #0x2c
000003   b001     RRET	R0, #0x1            	RRET R0, #0x01
                                           
                                           
                                           ID_kf8s_touch_g_4	.code
                                           __KF8_Key_Max_Pressed_Limitable_Circle_
00070b   b040     RRET	R0, #0x40           	RRET R0, #0x40
00070c   b01f     RRET	R0, #0x1f           	RRET R0, #0x1f
                                           
                                           
                                           ID_kf8s_touch_g_5	.code
                                           __KF8_BaseLine_Update_Circle_Count_For_UP_
000714   b040     RRET	R0, #0x40           	RRET R0, #0x40
                                           
                                           
                                           ID_kf8s_touch_g_6	.code
                                           __KF8_BaseLine_Update_Circle_Count_For_Down_
000715   b0c0     RRET	R0, #0xc0           	RRET R0, #0xc0
                                           
                                           
                                           ID_kf8s_touch_g_7	.code
                                           __KF8_Define_Disturb_Channels_Amount_
000716   b003     RRET	R0, #0x3            	RRET R0, #0x03
                                           
                                           
                                           ID_kf8s_touch_g_8	.code
                                           __KF8_BasicLine_UP_Noise_Threshold_
000717   b0ec     RRET	R0, #0xec           	RRET R0, #0xec
                                           
                                           
                                           ID_kf8s_touch_g_9	.code
                                           __KF8_BasicLine_Down_Noise_Threshold_
000718   b014     RRET	R0, #0x14           	RRET R0, #0x14
                                           
                                           
                                           ID_kf8s_touch_g_10	.code
                                           __KF8_Data_Steady_Threshold_Set_
000719   b00c     RRET	R0, #0xc            	RRET R0, #0x0c
                                           
                                           
                                           ID_kf8s_touch_g_11	.code
                                           __KF8_Inside_Reference_Channel_Disturb_Threshold_Set_
00071a   b00f     RRET	R0, #0xf            	RRET R0, #0x0f
                                           
                                           
                                           ID_kf8s_touch_g_12	.code
                                           __KF8_TOUCH_CH_EN
0006f5   b002     RRET	R0, #0x2            	RRET R0, #0x02
0006f6   b003     RRET	R0, #0x3            	RRET R0, #0x03
0006f7   b004     RRET	R0, #0x4            	RRET R0, #0x04
0006f8   b005     RRET	R0, #0x5            	RRET R0, #0x05
0006f9   b008     RRET	R0, #0x8            	RRET R0, #0x08
0006fa   b009     RRET	R0, #0x9            	RRET R0, #0x09
0006fb   b00a     RRET	R0, #0xa            	RRET R0, #0x0a
0006fc   b00b     RRET	R0, #0xb            	RRET R0, #0x0b
                                           
                                           
                                           ID_kf8s_touch_g_13	.code
                                           __KF8_Inside_Reference_Channel_Declare_
00071b   b014     RRET	R0, #0x14           	RRET R0, #0x14
                                           
                                           
                                           ID_kf8s_touch_g_14	.code
                                           __KF8_Config_Finger_Threshold
0006fd   b032     RRET	R0, #0x32           	RRET R0, #0x32
0006fe   b032     RRET	R0, #0x32           	RRET R0, #0x32
0006ff   b032     RRET	R0, #0x32           	RRET R0, #0x32
000700   b032     RRET	R0, #0x32           	RRET R0, #0x32
000701   b032     RRET	R0, #0x32           	RRET R0, #0x32
000702   b032     RRET	R0, #0x32           	RRET R0, #0x32
000703   b032     RRET	R0, #0x32           	RRET R0, #0x32
000704   b032     RRET	R0, #0x32           	RRET R0, #0x32
                                           
                                           ;--------------------------------------------------------
                                           ; overlayable items in internal ram 
                                           ;--------------------------------------------------------
                                           ;	.udata_ovr
                                           
                                           ;	code size estimation:
                                           ;	    0+    0 =     0 instructions (    0 byte)
                                           
                                           
                                           	.end
                                           ;--------------------------------------------------------
                                           ; File Created by ChiponCC : aolisn inc.
                                           ; Version 3.0.4#6752 (Jul  6 2017 15:09:47) (MSVC)
                                           ; This file was generated Wed Apr 04 14:53:45 2018
                                           ;--------------------------------------------------------
                                           ; chipon port for the 16-bit core
                                           ;--------------------------------------------------------
                                           ;	.file	"../main.c"
                                           	.radix dec
                                           	.include "KF8S1024.inc"
                                           
                                           ;************************************************************ 
                                           ;       Header file for the KungFu8 
                                           ;       KF8S1024 
                                           ;       Microcontroller
                                           ; 
                                           ;       Copyright 2012-2013 ChipON, All rights reserved
                                           ;************************************************************ 
                                            
                                           T0                .EQU                0x01
                                           PCL               .EQU                0x02
                                           PSW               .EQU                0x03
                                           P0                .EQU                0x05
                                           P2                .EQU                0x06
                                           P1                .EQU                0x07
                                           P3                .EQU                0x08
                                           PCH               .EQU                0x0A
                                           INTCTL            .EQU                0x0B
                                           EIF1              .EQU                0x0C
                                           T1L               .EQU                0x0E
                                           T1H               .EQU                0x0F
                                           T1CTL             .EQU                0x10
                                           T2                .EQU                0x11
                                           T2CTL             .EQU                0x12
                                           PWMCTL            .EQU                0x15
                                           CMCTL1            .EQU                0x1A
                                           VRECAL            .EQU                0x1C
                                           ADCDATAH          .EQU                0x1E
                                           ADCCTL0           .EQU                0x1F
                                           OPTR              .EQU                0x21
                                           TR0               .EQU                0x25
                                           TR2               .EQU                0x26
                                           TR1               .EQU                0x27
                                           TR3               .EQU                0x28
                                           EIE1              .EQU                0x2C
                                           PCTL              .EQU                0x2E
                                           OSCCTL            .EQU                0x2F
                                           OSCCAL0           .EQU                0x30
                                           ANSEL             .EQU                0x31
                                           PUR               .EQU                0x35
                                           IOCL              .EQU                0x36
                                           OSCCAL1           .EQU                0x37
                                           ADCDATAL          .EQU                0x3E
                                           ADCCTL1           .EQU                0x3F
                                           T3L               .EQU                0x50
                                           CTCTL             .EQU                0x53
                                           T2CCR             .EQU                0x54
                                           OSCLDOCAL         .EQU                0x5E
                                           T1U               .EQU                0x5F
                                            
                                            
                                           
                                           ;Address:0x03 PSW Bits------------------
                                           RP0                .EQU                5
                                           TO                 .EQU                4
                                           PD                 .EQU                3
                                           Z                  .EQU                2
                                           DC                 .EQU                1
                                           CY                 .EQU                0
                                           _RP0               .EQU                5
                                           _TO                .EQU                4
                                           _PD                .EQU                3
                                           _Z                 .EQU                2
                                           _DC                .EQU                1
                                           _CY                .EQU                0
                                           
                                           ;Address:0x05 P0 Bits-------------------
                                           P05                .EQU                5
                                           P04                .EQU                4
                                           P03                .EQU                3
                                           P01                .EQU                1
                                           P00                .EQU                0
                                           _P05               .EQU                5
                                           _P04               .EQU                4
                                           _P03               .EQU                3
                                           _P01               .EQU                1
                                           _P00               .EQU                0
                                           
                                           ;Address:0x06 P2 Bits-------------------
                                           P21                .EQU                1
                                           P20                .EQU                0
                                           _P21               .EQU                1
                                           _P20               .EQU                0
                                           
                                           ;Address:0x07 P1 Bits-------------------
                                           P17                .EQU                7
                                           P16                .EQU                6
                                           P12                .EQU                2
                                           _P17               .EQU                7
                                           _P16               .EQU                6
                                           _P12               .EQU                2
                                           
                                           ;Address:0x08 P3 Bits-------------------
                                           P33                .EQU                3
                                           P32                .EQU                2
                                           P31                .EQU                1
                                           P30                .EQU                0
                                           _P33               .EQU                3
                                           _P32               .EQU                2
                                           _P31               .EQU                1
                                           _P30               .EQU                0
                                           
                                           ;Address:0x0B INTCTL Bits---------------
                                           AIE                .EQU                7
                                           PUIE               .EQU                6
                                           T0IE               .EQU                5
                                           P0IE               .EQU                3
                                           T0IF               .EQU                2
                                           P0IF               .EQU                0
                                           _AIE               .EQU                7
                                           _PUIE              .EQU                6
                                           _T0IE              .EQU                5
                                           _P0IE              .EQU                3
                                           _T0IF              .EQU                2
                                           _P0IF              .EQU                0
                                           
                                           ;Address:0x0C EIF1 Bits-----------------
                                           CTIF               .EQU                7
                                           ADIF               .EQU                6
                                           INT2IF             .EQU                5
                                           INT1IF             .EQU                4
                                           C1IF               .EQU                3
                                           PWM2IF             .EQU                2
                                           T2IF               .EQU                1
                                           T1IF               .EQU                0
                                           _CTIF              .EQU                7
                                           _ADIF              .EQU                6
                                           _INT2IF            .EQU                5
                                           _INT1IF            .EQU                4
                                           _C1IF              .EQU                3
                                           _PWM2IF            .EQU                2
                                           _T2IF              .EQU                1
                                           _T1IF              .EQU                0
                                           
                                           ;Address:0x10 T1CTL Bits----------------
                                           T1GC               .EQU                6
                                           T1CKS1             .EQU                5
                                           T1CKS0             .EQU                4
                                           T1SY               .EQU                2
                                           T1CS               .EQU                1
                                           T1ON               .EQU                0
                                           _T1GC              .EQU                6
                                           _T1CKS1            .EQU                5
                                           _T1CKS0            .EQU                4
                                           _T1SY              .EQU                2
                                           _T1CS              .EQU                1
                                           _T1ON              .EQU                0
                                           
                                           ;Address:0x12 T2CTL Bits----------------
                                           T2CKBS3            .EQU                6
                                           T2CKBS2            .EQU                5
                                           T2CKBS1            .EQU                4
                                           T2CKBS0            .EQU                3
                                           T2ON               .EQU                2
                                           T2CKPS1            .EQU                1
                                           T2CKPS0            .EQU                0
                                           _T2CKBS3           .EQU                6
                                           _T2CKBS2           .EQU                5
                                           _T2CKBS1           .EQU                4
                                           _T2CKBS0           .EQU                3
                                           _T2ON              .EQU                2
                                           _T2CKPS1           .EQU                1
                                           _T2CKPS0           .EQU                0
                                           
                                           ;Address:0x15 PWMCTL Bits---------------
                                           INT1SE             .EQU                6
                                           _INT1SE            .EQU                6
                                           
                                           ;Address:0x1A CMCTL1 Bits---------------
                                           CTCLKSEL1          .EQU                7
                                           CTCLKSEL0          .EQU                6
                                           CTVREFSEL1         .EQU                5
                                           CTVREFSEL0         .EQU                4
                                           _CTCLKSEL1         .EQU                7
                                           _CTCLKSEL0         .EQU                6
                                           _CTVREFSEL1        .EQU                5
                                           _CTVREFSEL0        .EQU                4
                                           
                                           ;Address:0x1F ADCCTL0 Bits--------------
                                           ADLR               .EQU                7
                                           CHS3               .EQU                5
                                           CHS2               .EQU                4
                                           CHS1               .EQU                3
                                           CHS0               .EQU                2
                                           START              .EQU                1
                                           ADEN               .EQU                0
                                           _ADLR              .EQU                7
                                           _CHS3              .EQU                5
                                           _CHS2              .EQU                4
                                           _CHS1              .EQU                3
                                           _CHS0              .EQU                2
                                           _START             .EQU                1
                                           _ADEN              .EQU                0
                                           
                                           ;Address:0x21 OPTR Bits-----------------
                                           PUPH               .EQU                7
                                           T0CS               .EQU                5
                                           T0SE               .EQU                4
                                           PSA                .EQU                3
                                           PS2                .EQU                2
                                           PS1                .EQU                1
                                           PS0                .EQU                0
                                           _PUPH              .EQU                7
                                           _T0CS              .EQU                5
                                           _T0SE              .EQU                4
                                           _PSA               .EQU                3
                                           _PS2               .EQU                2
                                           _PS1               .EQU                1
                                           _PS0               .EQU                0
                                           
                                           ;Address:0x25 TR0 Bits------------------
                                           TR05               .EQU                5
                                           TR04               .EQU                4
                                           TR03               .EQU                3
                                           TR01               .EQU                1
                                           TR00               .EQU                0
                                           _TR05              .EQU                5
                                           _TR04              .EQU                4
                                           _TR03              .EQU                3
                                           _TR01              .EQU                1
                                           _TR00              .EQU                0
                                           
                                           ;Address:0x26 TR2 Bits------------------
                                           TR21               .EQU                1
                                           TR20               .EQU                0
                                           _TR21              .EQU                1
                                           _TR20              .EQU                0
                                           
                                           ;Address:0x27 TR1 Bits------------------
                                           TR17               .EQU                7
                                           TR16               .EQU                6
                                           TR12               .EQU                2
                                           _TR17              .EQU                7
                                           _TR16              .EQU                6
                                           _TR12              .EQU                2
                                           
                                           ;Address:0x28 TR3 Bits------------------
                                           TR33               .EQU                3
                                           TR32               .EQU                2
                                           TR31               .EQU                1
                                           TR30               .EQU                0
                                           _TR33              .EQU                3
                                           _TR32              .EQU                2
                                           _TR31              .EQU                1
                                           _TR30              .EQU                0
                                           
                                           ;Address:0x2C EIE1 Bits-----------------
                                           CTIE               .EQU                7
                                           ADIE               .EQU                6
                                           INT2IE             .EQU                5
                                           INT1IE             .EQU                4
                                           C1IE               .EQU                3
                                           PWM2IE             .EQU                2
                                           T2IE               .EQU                1
                                           T1IE               .EQU                0
                                           _CTIE              .EQU                7
                                           _ADIE              .EQU                6
                                           _INT2IE            .EQU                5
                                           _INT1IE            .EQU                4
                                           _C1IE              .EQU                3
                                           _PWM2IE            .EQU                2
                                           _T2IE              .EQU                1
                                           _T1IE              .EQU                0
                                           
                                           ;Address:0x2E PCTL Bits-----------------
                                           VREEN              .EQU                7
                                           VREOE              .EQU                6
                                           SLVREN             .EQU                4
                                           POR                .EQU                1
                                           LVR                .EQU                0
                                           _VREEN             .EQU                7
                                           _VREOE             .EQU                6
                                           _SLVREN            .EQU                4
                                           _POR               .EQU                1
                                           _LVR               .EQU                0
                                           
                                           ;Address:0x2F OSCCTL Bits---------------
                                           CKOEN              .EQU                7
                                           IRCS2              .EQU                6
                                           IRCS1              .EQU                5
                                           IRCS0              .EQU                4
                                           _CKOEN             .EQU                7
                                           _IRCS2             .EQU                6
                                           _IRCS1             .EQU                5
                                           _IRCS0             .EQU                4
                                           
                                           ;Address:0x31 ANSEL Bits----------------
                                           ANS6               .EQU                6
                                           ANS3               .EQU                3
                                           ANS1               .EQU                1
                                           _ANS6              .EQU                6
                                           _ANS3              .EQU                3
                                           _ANS1              .EQU                1
                                           
                                           ;Address:0x35 PUR Bits------------------
                                           PUR5               .EQU                5
                                           PUR4               .EQU                4
                                           PUR2               .EQU                2
                                           PUR1               .EQU                1
                                           PUR0               .EQU                0
                                           _PUR5              .EQU                5
                                           _PUR4              .EQU                4
                                           _PUR2              .EQU                2
                                           _PUR1              .EQU                1
                                           _PUR0              .EQU                0
                                           
                                           ;Address:0x36 IOCL Bits-----------------
                                           IOCL5              .EQU                5
                                           IOCL4              .EQU                4
                                           IOCL3              .EQU                3
                                           IOCL2              .EQU                2
                                           IOCL1              .EQU                1
                                           IOCL0              .EQU                0
                                           _IOCL5             .EQU                5
                                           _IOCL4             .EQU                4
                                           _IOCL3             .EQU                3
                                           _IOCL2             .EQU                2
                                           _IOCL1             .EQU                1
                                           _IOCL0             .EQU                0
                                           
                                           ;Address:0x3F ADCCTL1 Bits--------------
                                           ADCS2              .EQU                6
                                           ADCS1              .EQU                5
                                           ADCS0              .EQU                4
                                           VCFG1              .EQU                3
                                           VCFG0              .EQU                2
                                           _ADCS2             .EQU                6
                                           _ADCS1             .EQU                5
                                           _ADCS0             .EQU                4
                                           _VCFG1             .EQU                3
                                           _VCFG0             .EQU                2
                                           
                                           ;Address:0x50 T3L Bits------------------
                                           T3L7               .EQU                7
                                           T3L6               .EQU                6
                                           T3L5               .EQU                5
                                           T3L4               .EQU                4
                                           T3L3               .EQU                3
                                           T3L2               .EQU                2
                                           T3L1               .EQU                1
                                           T3L0               .EQU                0
                                           _T3L7              .EQU                7
                                           _T3L6              .EQU                6
                                           _T3L5              .EQU                5
                                           _T3L4              .EQU                4
                                           _T3L3              .EQU                3
                                           _T3L2              .EQU                2
                                           _T3L1              .EQU                1
                                           _T3L0              .EQU                0
                                           
                                           ;Address:0x53 CTCTL Bits----------------
                                           CTEN               .EQU                7
                                           CTSTART            .EQU                6
                                           CTCAPS             .EQU                5
                                           CTCMS              .EQU                4
                                           CTCHSEL4           .EQU                4
                                           CTCHSEL3           .EQU                3
                                           CTCHSEL2           .EQU                2
                                           CTCHSEL1           .EQU                1
                                           CTCHSEL0           .EQU                0
                                           _CTEN              .EQU                7
                                           _CTSTART           .EQU                6
                                           _CTCAPS            .EQU                5
                                           _CTCMS             .EQU                4
                                           _CTCHSEL4          .EQU                4
                                           _CTCHSEL3          .EQU                3
                                           _CTCHSEL2          .EQU                2
                                           _CTCHSEL1          .EQU                1
                                           _CTCHSEL0          .EQU                0
                                           
                                           ;Address:0x5E OSCLDOCAL Bits------------
                                            
                                            
                                           ;--------------------------------------------------------
                                           ; external declarations
                                           ;--------------------------------------------------------
                                           	.extern	_init_mcu
                                           	.extern	__KF8S_Get_Ver_General_
                                           	.extern	__KF8S_Lib_Set_General_Parameter
                                           	.extern	__KF8S_Init_Touch_General_
                                           	.extern	__KF8S_Touch_Process_General_
                                           	.extern	__KF8S_Touch_TEST_General_
                                           	.extern	__R2PCL
                                           	.extern	_TOUCH_DEBUG_TRS_DEAL
                                           	.extern	_TOUCH_DEBUG_SEND_OUT
                                           	.extern	_PSW_bits
                                           	.extern	_P0_bits
                                           	.extern	_P2_bits
                                           	.extern	_P1_bits
                                           	.extern	_P3_bits
                                           	.extern	_INTCTL_bits
                                           	.extern	_EIF1_bits
                                           	.extern	_T1CTL_bits
                                           	.extern	_T2CTL_bits
                                           	.extern	_PWMCTL_bits
                                           	.extern	_CMCTL1_bits
                                           	.extern	_ADCCTL0_bits
                                           	.extern	_OPTR_bits
                                           	.extern	_TR0_bits
                                           	.extern	_TR2_bits
                                           	.extern	_TR1_bits
                                           	.extern	_TR3_bits
                                           	.extern	_EIE1_bits
                                           	.extern	_PCTL_bits
                                           	.extern	_OSCCTL_bits
                                           	.extern	_ANSEL_bits
                                           	.extern	_PUR_bits
                                           	.extern	_IOCL_bits
                                           	.extern	_ADCCTL1_bits
                                           	.extern	_T3L_bits
                                           	.extern	_CTCTL_bits
                                           	.extern	_OSCLDOCAL_bits
                                           	.extern	__KF8_LIBi_channel_flag_
                                           	.extern	__KF8_LIBc_channel_
                                           	.extern	__KF8_LIBc_channel_Buf
                                           	.extern	__KF8_LIBi_Date_Change_
                                           	.extern	__KF8_LIBc_baseline_count_
                                           	.extern	__KF8_LIBi_buff_hit_
                                           	.extern	__KF8_LIBi_buff_baseline_
                                           	.extern	__KF8_LIBc_touch_count_
                                           	.extern	_sentbuf1
                                           	.extern	_sentbuf2
                                           	.extern	_sentbuf3
                                           	.extern	_sentbuf4
                                           	.extern	_CHS_AMOUNT
                                           	.extern	_TCS_AMOUNT
                                           	.extern	__KF8_Disturb_Protect_Circle_
                                           	.extern	__KF8_DoubleKey_Compages_Limitable_Circle_
                                           	.extern	__KF8_Key_Max_Pressed_Limitable_Circle_
                                           	.extern	__KF8_BaseLine_Update_Circle_Count_For_UP_
                                           	.extern	__KF8_BaseLine_Update_Circle_Count_For_Down_
                                           	.extern	__KF8_Define_Disturb_Channels_Amount_
                                           	.extern	__KF8_BasicLine_UP_Noise_Threshold_
                                           	.extern	__KF8_BasicLine_Down_Noise_Threshold_
                                           	.extern	__KF8_Data_Steady_Threshold_Set_
                                           	.extern	__KF8_Inside_Reference_Channel_Disturb_Threshold_Set_
                                           	.extern	__KF8_Inside_Reference_Channel_Declare_
                                           	.extern	__KF8_Config_Finger_Threshold
                                           	.extern	__KF8_TOUCH_CH_EN
                                           	.extern	_T0
                                           	.extern	_PCL
                                           	.extern	_PSW
                                           	.extern	_P0
                                           	.extern	_P2
                                           	.extern	_P1
                                           	.extern	_P3
                                           	.extern	_PCH
                                           	.extern	_INTCTL
                                           	.extern	_EIF1
                                           	.extern	_T1L
                                           	.extern	_T1H
                                           	.extern	_T1CTL
                                           	.extern	_T2
                                           	.extern	_T2CTL
                                           	.extern	_PWMCTL
                                           	.extern	_CMCTL1
                                           	.extern	_VRECAL
                                           	.extern	_ADCDATAH
                                           	.extern	_ADCCTL0
                                           	.extern	_OPTR
                                           	.extern	_TR0
                                           	.extern	_TR2
                                           	.extern	_TR1
                                           	.extern	_TR3
                                           	.extern	_EIE1
                                           	.extern	_PCTL
                                           	.extern	_OSCCTL
                                           	.extern	_OSCCAL0
                                           	.extern	_ANSEL
                                           	.extern	_PUR
                                           	.extern	_IOCL
                                           	.extern	_OSCCAL1
                                           	.extern	_ADCDATAL
                                           	.extern	_ADCCTL1
                                           	.extern	_T3L
                                           	.extern	_CTCTL
                                           	.extern	_T2CCR
                                           	.extern	_OSCLDOCAL
                                           	.extern	_T1U
                                           	.extern	_startup
                                           	.extern	__gsinit_startup
                                           ;--------------------------------------------------------
                                           ; global declarations
                                           ;--------------------------------------------------------
                                           	.global	_delay_us
                                           	.global	_delay_ms
                                           	.global	_display
                                           	.global	_INT_FUN
                                           	.global	_main
                                           	.global	_Touch_Watch
                                           	.global	_flag
                                           
                                           	.global STK12
                                           	.global STK11
                                           	.global STK10
                                           	.global STK09
                                           	.global STK08
                                           	.global STK07
                                           	.global STK06
                                           	.global STK05
                                           	.global STK04
                                           	.global STK03
                                           	.global STK02
                                           	.global STK01
                                           	.global STK00
                                           
                                           sharebank .udata
                                           STK12	.res 1
                                           	.type STK12, 108
                                           STK11	.res 1
                                           	.type STK11, 108
                                           STK10	.res 1
                                           	.type STK10, 108
                                           STK09	.res 1
                                           	.type STK09, 108
                                           STK08	.res 1
                                           	.type STK08, 108
                                           STK07	.res 1
                                           	.type STK07, 108
                                           STK06	.res 1
                                           	.type STK06, 108
                                           STK05	.res 1
                                           	.type STK05, 108
                                           STK04	.res 1
                                           	.type STK04, 108
                                           STK03	.res 1
                                           	.type STK03, 108
                                           STK02	.res 1
                                           	.type STK02, 108
                                           STK01	.res 1
                                           	.type STK01, 108
                                           STK00	.res 1
                                           	.type STK00, 108
                                           
                                           ;--------------------------------------------------------
                                           ; global definitions
                                           ;--------------------------------------------------------
                                           UD_main_0	.udata
                                           _Touch_Watch	.res	2
                                           
                                           UD_main_1	.udata
                                           _flag	.res	1
                                           
                                           ;--------------------------------------------------------
                                           ; absolute symbol definitions
                                           ;--------------------------------------------------------
                                           ;--------------------------------------------------------
                                           ; compiler-defined variables
                                           ;--------------------------------------------------------
                                           UDL_main_0	.udata
                                           r0x1004	.res	1
                                           UDL_main_1	.udata
                                           r0x1003	.res	1
                                           UDL_main_2	.udata
                                           r0x1005	.res	1
                                           UDL_main_3	.udata
                                           r0x1006	.res	1
                                           UDL_main_4	.udata
                                           r0x1007	.res	1
                                           UDL_main_5	.udata
                                           r0x1008	.res	1
                                           UDL_main_6	.udata
                                           r0x100E	.res	1
                                           UDL_main_7	.udata
                                           r0x100D	.res	1
                                           UDL_main_8	.udata
                                           r0x100F	.res	1
                                           UDL_main_9	.udata
                                           r0x1010	.res	1
                                           UDL_main_10	.udata
                                           r0x1009	.res	1
                                           UDL_main_11	.udata
                                           r0x100A	.res	1
                                           UDL_main_12	.udata
                                           r0x100B	.res	1
                                           ;--------------------------------------------------------
                                           ; initialized data
                                           ;--------------------------------------------------------
                                           ;--------------------------------------------------------
                                           ; overlayable items in internal ram 
                                           ;--------------------------------------------------------
                                           ;	.udata_ovr
                                           ;--------------------------------------------------------
                                           ; reset vector 
                                           ;--------------------------------------------------------
                                           STARTUP	.code 0x0000
000000   0000     NOP                      	NOP
                                           	PAGESEL	init_imp
000001   c705     JMP	#0x705               	JMP		init_imp
                                           
                                           	.global	init_imp
                                           INIT_IMP	.code
                                           init_imp
                                           	PAGESEL	_startup
000705   d6e4     CALL	#0x6e4              	CALL	_startup
                                           	PAGESEL	__gsinit_startup
000706   d70f     CALL	#0x70f              	CALL	__gsinit_startup
                                           	PAGESEL	_main
000707   c5f4     JMP	#0x5f4               	JMP		_main
                                           ;--------------------------------------------------------
                                           ; interrupt and initialization code
                                           ;--------------------------------------------------------
                                           c_interrupt	.code	0x4
000004   f8c3     MOV	R3, R0               	MOV		R3,R0
000005   5803     MOV	R4, 0x3              	MOV		R4,PSW
000006   5a0a     MOV	R5, 0xa              	MOV		R5,PCH
000007   f8ca     MOV	R2, R1               	MOV		R2,R1
                                           	PAGESEL	interrupt_service_routine
000008   c6c0     JMP	#0x6c0               	JMP		interrupt_service_routine
                                           
                                           
                                           
                                           func._INT_FUN	.code
                                           ;***
                                           ;  PostBlock Stats: dbName = I
                                           ;***
                                           ;entry:  _INT_FUN	;Function start
                                           ; 0 exit points
                                           ;functions called:
                                           ;   _TOUCH_DEBUG_TRS_DEAL
                                           ;   __KF8S_Touch_Process_General_
                                           ;   _TOUCH_DEBUG_TRS_DEAL
                                           ;   __KF8S_Touch_Process_General_
                                           ;; Starting PostCode block
                                           ;	op : LABEL
                                           ;	op : FUNCTION
                                           _INT_FUN	;Function start
                                           ; 0 exit points
                                           ;	op : GET_VALUE_AT_ADDRESS
                                           ; R3 resprent for wsave,R4 resprent for ssave, R5 resprent for psave
                                           interrupt_service_routine
                                           ;	.line	160; "../main.c"	if(T1IF||CTIF)
0006c0   700c     JNB	0xc, 0               	JNB	_EIF1_bits, 0
0006c1   c6c4     JMP	#0x6c4               	JMP	_00023_DS_
                                           ;	op : GET_VALUE_AT_ADDRESS
0006c2   7f0c     JB	0xc, 7                	JB	_EIF1_bits, 7
0006c3   c6cd     JMP	#0x6cd               	JMP	_00026_DS_
                                           ;	op : LABEL
                                           ;	op : =
                                           _00023_DS_
                                           ;	.line	162; "../main.c"	T1IF=0;
0006c4   600c     CLR	0xc, 0               	CLR	_EIF1_bits, 0
                                           ;	op : =
                                           ;	.line	163; "../main.c"	CTIF=0;
0006c5   670c     CLR	0xc, 7               	CLR	_EIF1_bits, 7
                                           ;	op : =
                                           ;	.line	164; "../main.c"	Touch_Watch=0;
0006c6   6503     CLR	0x3, 5               	BANKSEL	_Touch_Watch
0006c7   03b5     CLR	0xb5                 	CLR	_Touch_Watch
                                           	BANKSEL	_Touch_Watch
0006c8   03b6     CLR	0xb6                 	CLR	(_Touch_Watch + 1)
                                           ;	op : =
                                           ;	.line	165; "../main.c"	flag = 1;
0006c9   9801     MOV	R0, #0x1             	MOV	R0,# 0x01
                                           	BANKSEL	_flag
0006ca   51a1     MOV	0xa1, R0             	MOV	_flag, R0
                                           ;	op : CALL
                                           ;	.line	167; "../main.c"	TOUCH_DEBUG_TRS_DEAL();		// µ÷ÊÔÇúÏßÊä³ö
                                           	PAGESEL	_TOUCH_DEBUG_TRS_DEAL
0006cb   d413     CALL	#0x413              	CALL	_TOUCH_DEBUG_TRS_DEAL
                                           	PAGESEL	$
                                           ;	op : CALL
                                           ;	.line	168; "../main.c"	_KF8S_Touch_Process_General_(); //¸üÐÂ°´¼ü±êÖ¾
                                           	PAGESEL	__KF8S_Touch_Process_General_
0006cc   d510     CALL	#0x510              	CALL	__KF8S_Touch_Process_General_
                                           	PAGESEL	$
                                           ;	op : LABEL
                                           ;	op : ENDFUNCTION
                                           _00026_DS_
0006cd   f8d1     MOV	R1, R2               	MOV	R1, R2
0006ce   5b0a     MOV	0xa, R5              	MOV	PCH, R5
0006cf   5903     MOV	0x3, R4              	MOV	PSW, R4
0006d0   f8d8     MOV	R0, R3               	MOV	R0, R3
0006d1   0009     IRET                     	IRET	
                                           
                                           
                                           
                                           func._main	.code
                                           ;***
                                           ;  PostBlock Stats: dbName = M
                                           ;***
                                           ;entry:  _main	;Function start
                                           ; 2 exit points
                                           ;has an exit
                                           ;functions called:
                                           ;   _init_mcu
                                           ;   _delay_ms
                                           ;   __KF8S_Init_Touch_General_
                                           ;   _display
                                           ;   __KF8S_Init_Touch_General_
                                           ;   _init_mcu
                                           ;   _delay_ms
                                           ;   __KF8S_Init_Touch_General_
                                           ;   _display
                                           ;   __KF8S_Init_Touch_General_
                                           ;5 compiler assigned registers:
                                           ;   STK00
                                           ;   r0x1009
                                           ;   r0x100A
                                           ;   r0x100B
                                           ;   r0x100C
                                           ;; Starting PostCode block
                                           ;	op : LABEL
                                           ;	op : FUNCTION
                                           _main	;Function start
                                           ; 2 exit points
                                           ;	op : CALL
                                           ;	.line	182; "../main.c"	init_mcu();						//³õÊ¼»¯MCU¼Ä´æÆ÷
                                           	PAGESEL	_init_mcu
0005f4   d6ae     CALL	#0x6ae              	CALL	_init_mcu
                                           	PAGESEL	$
                                           ;	op : SEND
                                           ;	op : CALL
                                           ;	.line	183; "../main.c"	delay_ms(500);					//ÑÓÊ±Ò»»á£¬·ÀÖ¹ÉÏµçÎó´¥·¢´¥ÃþÍ¨µÀ
0005f5   98f4     MOV	R0, #0xf4            	MOV	R0,# 0xf4
0005f6   6503     CLR	0x3, 5               	BANKSEL	STK00
0005f7   51dd     MOV	0xdd, R0             	MOV	STK00, R0
0005f8   9801     MOV	R0, #0x1             	MOV	R0,# 0x01
                                           	PAGESEL	_delay_ms
0005f9   d64c     CALL	#0x64c              	CALL	_delay_ms
                                           	PAGESEL	$
                                           ;	op : =
                                           ;	.line	184; "../main.c"	CMCTL1 = 0x90;    //ÉèÖÃ´¥Ãþ·ÖÆµºÍ»ù×¼µçÑ¹
0005fa   9890     MOV	R0, #0x90            	MOV	R0,# 0x90
0005fb   511a     MOV	0x1a, R0             	MOV	_CMCTL1, R0
                                           ;	op : INLINEASM
0005fc   0064     CWDT                     	CWDT 
                                           ;	op : CALL
                                           ;	.line	188; "../main.c"	_KF8S_Init_Touch_General_();		//µ÷ÓÃµçÈÝ´¥Ãþ¿âº¯ÊýµÄ³õÊ¼»¯
                                           	PAGESEL	__KF8S_Init_Touch_General_
0005fd   d621     CALL	#0x621              	CALL	__KF8S_Init_Touch_General_
                                           	PAGESEL	$
                                           ;	op : INLINEASM
0005fe   0064     CWDT                     	CWDT 
                                           ;	op : LABEL
                                           ;	op : INLINEASM
                                           _00032_DS_
0005ff   0064     CWDT                     	CWDT 
                                           ;	op : CALL
                                           ;	.line	195; "../main.c"	display();					//ÏÔÊ¾LEDµÆ
                                           	PAGESEL	_display
000600   d71c     CALL	#0x71c              	CALL	_display
                                           	PAGESEL	$
                                           ;	op : +
                                           ;	.line	208; "../main.c"	Touch_Watch++;
000601   6503     CLR	0x3, 5               	BANKSEL	_Touch_Watch
000602   0bb5     INC	0xb5                 	INC	_Touch_Watch
000603   7a03     JB	0x3, 2                	JB	PSW, 2
000604   c606     JMP	#0x606               	JMP	_00039_DS_
                                           	BANKSEL	_Touch_Watch
000605   0bb6     INC	0xb6                 	INC	(_Touch_Watch + 1)
                                           ;	op : CAST
                                           _00039_DS_
                                           ;	.line	209; "../main.c"	if(Touch_Watch>50000)
                                           	BANKSEL	_Touch_Watch
000606   0eb5     MOVZ	R0, 0xb5            	MOVZ	R0, _Touch_Watch
                                           	BANKSEL	r0x1009
000607   5196     MOV	0x96, R0             	MOV	r0x1009, R0
                                           	BANKSEL	_Touch_Watch
000608   0eb6     MOVZ	R0, 0xb6            	MOVZ	R0, (_Touch_Watch + 1)
                                           	BANKSEL	r0x100A
000609   5195     MOV	0x95, R0             	MOV	r0x100A, R0
                                           	BANKSEL	r0x100B
00060a   0394     CLR	0x94                 	CLR	r0x100B
                                           ;;1	CLR	r0x100C
                                           ;	op : >
                                           ;swapping arguments (AOP_TYPEs 1/2)
                                           ;signed compare: left >= lit(0xC351=50001), size=4, mask=ffffffff
00060b   9800     MOV	R0, #0               	MOV	R0,# 0x00
00060c   8080     ADD	R0, #0x80            	ADD	R0,# 0x80
00060d   8080     ADD	R0, #0x80            	ADD	R0,# 0x80
                                           ;comparing bytes at offset 3
00060e   7a03     JB	0x3, 2                	JB	PSW, 2
00060f   c61a     JMP	#0x61a               	JMP	_00038_DS_
000610   9800     MOV	R0, #0               	MOV	R0,# 0x00
                                           	BANKSEL	r0x100B
000611   3894     SUB	R0, 0x94             	SUB	R0, r0x100B
000612   7a03     JB	0x3, 2                	JB	PSW, 2
000613   c61a     JMP	#0x61a               	JMP	_00038_DS_
000614   98c3     MOV	R0, #0xc3            	MOV	R0,# 0xc3
                                           	BANKSEL	r0x100A
000615   3895     SUB	R0, 0x95             	SUB	R0, r0x100A
000616   7a03     JB	0x3, 2                	JB	PSW, 2
000617   c61a     JMP	#0x61a               	JMP	_00038_DS_
000618   9851     MOV	R0, #0x51            	MOV	R0,# 0x51
                                           	BANKSEL	r0x1009
000619   3896     SUB	R0, 0x96             	SUB	R0, r0x1009
                                           _00038_DS_
00061a   7803     JB	0x3, 0                	JB	PSW, 0
00061b   c5ff     JMP	#0x5ff               	JMP	_00032_DS_
                                           ;	op : =
                                           ;	.line	211; "../main.c"	Touch_Watch=0;
                                           	BANKSEL	_Touch_Watch
00061c   03b5     CLR	0xb5                 	CLR	_Touch_Watch
                                           	BANKSEL	_Touch_Watch
00061d   03b6     CLR	0xb6                 	CLR	(_Touch_Watch + 1)
                                           ;	op : CALL
                                           ;	.line	212; "../main.c"	_KF8S_Init_Touch_General_();
                                           	PAGESEL	__KF8S_Init_Touch_General_
00061e   d621     CALL	#0x621              	CALL	__KF8S_Init_Touch_General_
                                           	PAGESEL	$
                                           ;	op : GOTO
00061f   c5ff     JMP	#0x5ff               	JMP	_00032_DS_
                                           ;	op : LABEL
                                           ;	op : ENDFUNCTION
000620   0008     CRET                     	CRET	
                                           ; exit point of _main
                                           
                                           
                                           
                                           func._delay_us	.code
                                           ;***
                                           ;  PostBlock Stats: dbName = C
                                           ;***
                                           ;entry:  _delay_us	;Function start
                                           ; 2 exit points
                                           ;has an exit
                                           ;5 compiler assigned registers:
                                           ;   r0x100D
                                           ;   STK00
                                           ;   r0x100E
                                           ;   r0x100F
                                           ;   r0x1010
                                           ;; Starting PostCode block
                                           ;	op : LABEL
                                           ;	op : FUNCTION
                                           _delay_us	;Function start
                                           ; 2 exit points
                                           ;	op : RECEIVE
                                           ;	.line	121; "../main.c"	void delay_us(uint us_data)
0006d2   6503     CLR	0x3, 5               	BANKSEL	r0x100D
0006d3   5199     MOV	0x99, R0             	MOV	r0x100D, R0
                                           	BANKSEL	STK00
0006d4   0edd     MOVZ	R0, 0xdd            	MOVZ	R0, STK00
                                           	BANKSEL	r0x100E
0006d5   519a     MOV	0x9a, R0             	MOV	r0x100E, R0
                                           ;	op : =
                                           ;	op : LABEL
                                           ;	op : =
                                           _00016_DS_
                                           ;	.line	123; "../main.c"	while(us_data--);
                                           	BANKSEL	r0x100E
0006d6   0e9a     MOVZ	R0, 0x9a            	MOVZ	R0, r0x100E
                                           	BANKSEL	r0x100F
0006d7   5198     MOV	0x98, R0             	MOV	r0x100F, R0
                                           	BANKSEL	r0x100D
0006d8   0e99     MOVZ	R0, 0x99            	MOVZ	R0, r0x100D
                                           	BANKSEL	r0x1010
0006d9   5197     MOV	0x97, R0             	MOV	r0x1010, R0
                                           ;	op : -
0006da   98ff     MOV	R0, #0xff            	MOV	R0,# 0xff
                                           	BANKSEL	r0x100E
0006db   219a     ADD	0x9a, R0             	ADD	r0x100E, R0
0006dc   7003     JNB	0x3, 0               	JNB	PSW, 0
0006dd   c6df     JMP	#0x6df               	JMP	_00040_DS_
                                           	BANKSEL	r0x100D
0006de   0799     DEC	0x99                 	DEC	r0x100D
                                           ;	op : IFX
                                           _00040_DS_
                                           	BANKSEL	r0x100F
0006df   0e98     MOVZ	R0, 0x98            	MOVZ	R0, r0x100F
                                           	BANKSEL	r0x1010
0006e0   3097     ORL	R0, 0x97             	ORL	R0, r0x1010
0006e1   7a03     JB	0x3, 2                	JB	PSW, 2
0006e2   c6d6     JMP	#0x6d6               	JMP	_00016_DS_
                                           ;	op : LABEL
                                           ;	op : ENDFUNCTION
0006e3   0008     CRET                     	CRET	
                                           ; exit point of _delay_us
                                           
                                           
                                           
                                           func._delay_ms	.code
                                           ;***
                                           ;  PostBlock Stats: dbName = C
                                           ;***
                                           ;entry:  _delay_ms	;Function start
                                           ; 2 exit points
                                           ;has an exit
                                           ;7 compiler assigned registers:
                                           ;   r0x1003
                                           ;   STK00
                                           ;   r0x1004
                                           ;   r0x1005
                                           ;   r0x1006
                                           ;   r0x1007
                                           ;   r0x1008
                                           ;; Starting PostCode block
                                           ;	op : LABEL
                                           ;	op : FUNCTION
                                           _delay_ms	;Function start
                                           ; 2 exit points
                                           ;	op : RECEIVE
                                           ;	.line	101; "../main.c"	void delay_ms(uint ms_data)
00064c   6503     CLR	0x3, 5               	BANKSEL	r0x1003
00064d   519f     MOV	0x9f, R0             	MOV	r0x1003, R0
                                           	BANKSEL	STK00
00064e   0edd     MOVZ	R0, 0xdd            	MOVZ	R0, STK00
                                           	BANKSEL	r0x1004
00064f   51a0     MOV	0xa0, R0             	MOV	r0x1004, R0
                                           ;	op : =
                                           ;	op : LABEL
                                           ;	op : =
                                           _00006_DS_
                                           ;	.line	104; "../main.c"	while(ms_data--)
                                           	BANKSEL	r0x1004
000650   0ea0     MOVZ	R0, 0xa0            	MOVZ	R0, r0x1004
                                           	BANKSEL	r0x1005
000651   519e     MOV	0x9e, R0             	MOV	r0x1005, R0
                                           	BANKSEL	r0x1003
000652   0e9f     MOVZ	R0, 0x9f            	MOVZ	R0, r0x1003
                                           	BANKSEL	r0x1006
000653   519d     MOV	0x9d, R0             	MOV	r0x1006, R0
                                           ;	op : -
000654   98ff     MOV	R0, #0xff            	MOV	R0,# 0xff
                                           	BANKSEL	r0x1004
000655   21a0     ADD	0xa0, R0             	ADD	r0x1004, R0
000656   7003     JNB	0x3, 0               	JNB	PSW, 0
000657   c659     JMP	#0x659               	JMP	_00041_DS_
                                           	BANKSEL	r0x1003
000658   079f     DEC	0x9f                 	DEC	r0x1003
                                           ;	op : IFX
                                           _00041_DS_
                                           	BANKSEL	r0x1005
000659   0e9e     MOVZ	R0, 0x9e            	MOVZ	R0, r0x1005
                                           	BANKSEL	r0x1006
00065a   309d     ORL	R0, 0x9d             	ORL	R0, r0x1006
00065b   7203     JNB	0x3, 2               	JNB	PSW, 2
00065c   c670     JMP	#0x670               	JMP	_00009_DS_
                                           ;	op : INLINEASM
00065d   0064     CWDT                     	CWDT 
                                           ;	op : =
                                           ;	.line	108; "../main.c"	while(j--)
00065e   98c8     MOV	R0, #0xc8            	MOV	R0,# 0xc8
                                           	BANKSEL	r0x1005
00065f   519e     MOV	0x9e, R0             	MOV	r0x1005, R0
                                           	BANKSEL	r0x1006
000660   039d     CLR	0x9d                 	CLR	r0x1006
                                           ;	op : LABEL
                                           ;	op : =
                                           _00003_DS_
                                           	BANKSEL	r0x1005
000661   0e9e     MOVZ	R0, 0x9e            	MOVZ	R0, r0x1005
                                           	BANKSEL	r0x1007
000662   519c     MOV	0x9c, R0             	MOV	r0x1007, R0
                                           	BANKSEL	r0x1006
000663   0e9d     MOVZ	R0, 0x9d            	MOVZ	R0, r0x1006
                                           	BANKSEL	r0x1008
000664   519b     MOV	0x9b, R0             	MOV	r0x1008, R0
                                           ;	op : -
000665   98ff     MOV	R0, #0xff            	MOV	R0,# 0xff
                                           	BANKSEL	r0x1005
000666   219e     ADD	0x9e, R0             	ADD	r0x1005, R0
000667   7003     JNB	0x3, 0               	JNB	PSW, 0
000668   c66a     JMP	#0x66a               	JMP	_00042_DS_
                                           	BANKSEL	r0x1006
000669   079d     DEC	0x9d                 	DEC	r0x1006
                                           ;	op : IFX
                                           _00042_DS_
                                           	BANKSEL	r0x1007
00066a   0e9c     MOVZ	R0, 0x9c            	MOVZ	R0, r0x1007
                                           	BANKSEL	r0x1008
00066b   309b     ORL	R0, 0x9b             	ORL	R0, r0x1008
00066c   7203     JNB	0x3, 2               	JNB	PSW, 2
00066d   c650     JMP	#0x650               	JMP	_00006_DS_
                                           ;	op : INLINEASM
00066e   0064     CWDT                     	CWDT 
                                           ;	op : GOTO
00066f   c661     JMP	#0x661               	JMP	_00003_DS_
                                           ;	op : LABEL
                                           ;	op : ENDFUNCTION
                                           _00009_DS_
000670   0008     CRET                     	CRET	
                                           ; exit point of _delay_ms
                                           
                                           
                                           
                                           func._display	.code
                                           ;***
                                           ;  PostBlock Stats: dbName = C
                                           ;***
                                           ;entry:  _display	;Function start
                                           ; 2 exit points
                                           ;has an exit
                                           ;; Starting PostCode block
                                           ;	op : LABEL
                                           ;	op : FUNCTION
                                           _display	;Function start
                                           ; 2 exit points
                                           ;	op : LABEL
                                           ;	op : ENDFUNCTION
                                           ;	.line	85; "../main.c"	if(_KF8_LIBi_channel_flag_&0x0800)		//Í¨µÀ11
00071c   0008     CRET                     	CRET	
                                           ; exit point of _display
                                           
                                           
                                           ;	code size estimation:
                                           ;	  123+   48 =   171 instructions (  438 byte)
                                           
                                           
                                           	.end
                                           
                                           ;************************************************************ 
                                           ;       Header file for the KungFu8 
                                           ;       KF8S1011 
                                           ;       Microcontroller
                                           ; 
                                           ;       Copyright 2012-2013 ChipON, All rights reserved
                                           ;************************************************************ 
                                            
                                           T0                .EQU                0x01
                                           PCL               .EQU                0x02
                                           PSW               .EQU                0x03
                                           P0                .EQU                0x05
                                           P2                .EQU                0x06
                                           P1                .EQU                0x07
                                           P3                .EQU                0x08
                                           P4                .EQU                0x09
                                           PCH               .EQU                0x0A
                                           INTCTL            .EQU                0x0B
                                           EIF1              .EQU                0x0C
                                           EIF2              .EQU                0x0D
                                           T1L               .EQU                0x0E
                                           T1H               .EQU                0x0F
                                           T1CTL             .EQU                0x10
                                           PWMCTL            .EQU                0x15
                                           CMCTL1            .EQU                0x1A
                                           VRECAL            .EQU                0x1C
                                           ANSEH             .EQU                0x1D
                                           ADCDATAH          .EQU                0x1E
                                           ADCCTL0           .EQU                0x1F
                                           OPTR              .EQU                0x21
                                           TR0               .EQU                0x25
                                           TR2               .EQU                0x26
                                           TR1               .EQU                0x27
                                           TR3               .EQU                0x28
                                           TR4               .EQU                0x29
                                           EIE1              .EQU                0x2C
                                           EIE2              .EQU                0x2D
                                           PCTL              .EQU                0x2E
                                           OSCCTL            .EQU                0x2F
                                           OSCCAL0           .EQU                0x30
                                           ANSEL             .EQU                0x31
                                           PUR               .EQU                0x35
                                           IOCL              .EQU                0x36
                                           OSCCAL1           .EQU                0x37
                                           BADDRH            .EQU                0x3A
                                           BADDRL            .EQU                0x3B
                                           EECTL1            .EQU                0x3C
                                           EECTL2            .EQU                0x3D
                                           ADCDATAL          .EQU                0x3E
                                           ADCCTL1           .EQU                0x3F
                                           T3L               .EQU                0x50
                                           CTCTL             .EQU                0x53
                                           RSCTL             .EQU                0x58
                                           TXSDR             .EQU                0x59
                                           RXSDR             .EQU                0x5A
                                           OSCLDOCAL         .EQU                0x5E
                                           T1U               .EQU                0x5F
                                           BRCTL             .EQU                0x77
                                           TSCTL             .EQU                0x78
                                           EUBRGL            .EQU                0x79
                                           EUBRGH            .EQU                0x7A
                                            
                                            
                                           
                                           ;Address:0x03 PSW Bits------------------
                                           RP0                .EQU                5
                                           TO                 .EQU                4
                                           PD                 .EQU                3
                                           Z                  .EQU                2
                                           DC                 .EQU                1
                                           CY                 .EQU                0
                                           _RP0               .EQU                5
                                           _TO                .EQU                4
                                           _PD                .EQU                3
                                           _Z                 .EQU                2
                                           _DC                .EQU                1
                                           _CY                .EQU                0
                                           
                                           ;Address:0x05 P0 Bits-------------------
                                           P07                .EQU                7
                                           P06                .EQU                6
                                           P05                .EQU                5
                                           P04                .EQU                4
                                           P03                .EQU                3
                                           P01                .EQU                1
                                           P00                .EQU                0
                                           _P07               .EQU                7
                                           _P06               .EQU                6
                                           _P05               .EQU                5
                                           _P04               .EQU                4
                                           _P03               .EQU                3
                                           _P01               .EQU                1
                                           _P00               .EQU                0
                                           
                                           ;Address:0x06 P2 Bits-------------------
                                           P27                .EQU                7
                                           P26                .EQU                6
                                           P23                .EQU                3
                                           P22                .EQU                2
                                           P21                .EQU                1
                                           P20                .EQU                0
                                           _P27               .EQU                7
                                           _P26               .EQU                6
                                           _P23               .EQU                3
                                           _P22               .EQU                2
                                           _P21               .EQU                1
                                           _P20               .EQU                0
                                           
                                           ;Address:0x07 P1 Bits-------------------
                                           P17                .EQU                7
                                           P16                .EQU                6
                                           P15                .EQU                5
                                           P13                .EQU                3
                                           P12                .EQU                2
                                           _P17               .EQU                7
                                           _P16               .EQU                6
                                           _P15               .EQU                5
                                           _P13               .EQU                3
                                           _P12               .EQU                2
                                           
                                           ;Address:0x08 P3 Bits-------------------
                                           P37                .EQU                7
                                           P36                .EQU                6
                                           P35                .EQU                5
                                           P34                .EQU                4
                                           P33                .EQU                3
                                           P31                .EQU                1
                                           P30                .EQU                0
                                           _P37               .EQU                7
                                           _P36               .EQU                6
                                           _P35               .EQU                5
                                           _P34               .EQU                4
                                           _P33               .EQU                3
                                           _P31               .EQU                1
                                           _P30               .EQU                0
                                           
                                           ;Address:0x09 P4 Bits-------------------
                                           P43                .EQU                3
                                           _P43               .EQU                3
                                           
                                           ;Address:0x0B INTCTL Bits---------------
                                           AIE                .EQU                7
                                           PUIE               .EQU                6
                                           T0IE               .EQU                5
                                           P0IE               .EQU                3
                                           T0IF               .EQU                2
                                           P0IF               .EQU                0
                                           _AIE               .EQU                7
                                           _PUIE              .EQU                6
                                           _T0IE              .EQU                5
                                           _P0IE              .EQU                3
                                           _T0IF              .EQU                2
                                           _P0IF              .EQU                0
                                           
                                           ;Address:0x0C EIF1 Bits-----------------
                                           CTIF               .EQU                7
                                           ADIF               .EQU                6
                                           INT2IF             .EQU                5
                                           INT1IF             .EQU                4
                                           C1IF               .EQU                3
                                           PWM2IF             .EQU                2
                                           T2IF               .EQU                1
                                           T1IF               .EQU                0
                                           _CTIF              .EQU                7
                                           _ADIF              .EQU                6
                                           _INT2IF            .EQU                5
                                           _INT1IF            .EQU                4
                                           _C1IF              .EQU                3
                                           _PWM2IF            .EQU                2
                                           _T2IF              .EQU                1
                                           _T1IF              .EQU                0
                                           
                                           ;Address:0x0D EIF2 Bits-----------------
                                           RXIF               .EQU                5
                                           TXIF               .EQU                4
                                           _RXIF              .EQU                5
                                           _TXIF              .EQU                4
                                           
                                           ;Address:0x10 T1CTL Bits----------------
                                           T1GC               .EQU                6
                                           T1CKS1             .EQU                5
                                           T1CKS0             .EQU                4
                                           T1SY               .EQU                2
                                           T1CS               .EQU                1
                                           T1ON               .EQU                0
                                           _T1GC              .EQU                6
                                           _T1CKS1            .EQU                5
                                           _T1CKS0            .EQU                4
                                           _T1SY              .EQU                2
                                           _T1CS              .EQU                1
                                           _T1ON              .EQU                0
                                           
                                           ;Address:0x15 PWMCTL Bits---------------
                                           INT2SE             .EQU                7
                                           INT1SE             .EQU                6
                                           _INT2SE            .EQU                7
                                           _INT1SE            .EQU                6
                                           
                                           ;Address:0x1A CMCTL1 Bits---------------
                                           CTCLKSEL1          .EQU                7
                                           CTCLKSEL0          .EQU                6
                                           CTVREFSEL1         .EQU                5
                                           CTVREFSEL0         .EQU                4
                                           _CTCLKSEL1         .EQU                7
                                           _CTCLKSEL0         .EQU                6
                                           _CTVREFSEL1        .EQU                5
                                           _CTVREFSEL0        .EQU                4
                                           
                                           ;Address:0x1D ANSEH Bits----------------
                                           ANS11              .EQU                3
                                           ANS10              .EQU                2
                                           _ANS11             .EQU                3
                                           _ANS10             .EQU                2
                                           
                                           ;Address:0x1F ADCCTL0 Bits--------------
                                           ADLR               .EQU                7
                                           CHS3               .EQU                5
                                           CHS2               .EQU                4
                                           CHS1               .EQU                3
                                           CHS0               .EQU                2
                                           START              .EQU                1
                                           ADEN               .EQU                0
                                           _ADLR              .EQU                7
                                           _CHS3              .EQU                5
                                           _CHS2              .EQU                4
                                           _CHS1              .EQU                3
                                           _CHS0              .EQU                2
                                           _START             .EQU                1
                                           _ADEN              .EQU                0
                                           
                                           ;Address:0x21 OPTR Bits-----------------
                                           PUPH               .EQU                7
                                           T0CS               .EQU                5
                                           T0SE               .EQU                4
                                           PSA                .EQU                3
                                           PS2                .EQU                2
                                           PS1                .EQU                1
                                           PS0                .EQU                0
                                           _PUPH              .EQU                7
                                           _T0CS              .EQU                5
                                           _T0SE              .EQU                4
                                           _PSA               .EQU                3
                                           _PS2               .EQU                2
                                           _PS1               .EQU                1
                                           _PS0               .EQU                0
                                           
                                           ;Address:0x25 TR0 Bits------------------
                                           TR07               .EQU                7
                                           TR06               .EQU                6
                                           TR05               .EQU                5
                                           TR04               .EQU                4
                                           TR03               .EQU                3
                                           TR01               .EQU                1
                                           TR00               .EQU                0
                                           _TR07              .EQU                7
                                           _TR06              .EQU                6
                                           _TR05              .EQU                5
                                           _TR04              .EQU                4
                                           _TR03              .EQU                3
                                           _TR01              .EQU                1
                                           _TR00              .EQU                0
                                           
                                           ;Address:0x26 TR2 Bits------------------
                                           TR27               .EQU                7
                                           TR26               .EQU                6
                                           TR23               .EQU                3
                                           TR22               .EQU                2
                                           TR21               .EQU                1
                                           TR20               .EQU                0
                                           _TR27              .EQU                7
                                           _TR26              .EQU                6
                                           _TR23              .EQU                3
                                           _TR22              .EQU                2
                                           _TR21              .EQU                1
                                           _TR20              .EQU                0
                                           
                                           ;Address:0x27 TR1 Bits------------------
                                           TR17               .EQU                7
                                           TR16               .EQU                6
                                           TR15               .EQU                5
                                           TR13               .EQU                3
                                           TR12               .EQU                2
                                           _TR17              .EQU                7
                                           _TR16              .EQU                6
                                           _TR15              .EQU                5
                                           _TR13              .EQU                3
                                           _TR12              .EQU                2
                                           
                                           ;Address:0x28 TR3 Bits------------------
                                           TR37               .EQU                7
                                           TR36               .EQU                6
                                           TR35               .EQU                5
                                           TR34               .EQU                4
                                           TR33               .EQU                3
                                           TR31               .EQU                1
                                           TR30               .EQU                0
                                           _TR37              .EQU                7
                                           _TR36              .EQU                6
                                           _TR35              .EQU                5
                                           _TR34              .EQU                4
                                           _TR33              .EQU                3
                                           _TR31              .EQU                1
                                           _TR30              .EQU                0
                                           
                                           ;Address:0x29 TR4 Bits------------------
                                           TR43               .EQU                3
                                           _TR43              .EQU                3
                                           
                                           ;Address:0x2C EIE1 Bits-----------------
                                           CTIE               .EQU                7
                                           ADIE               .EQU                6
                                           INT2IE             .EQU                5
                                           INT1IE             .EQU                4
                                           C1IE               .EQU                3
                                           PWM2IE             .EQU                2
                                           T2IE               .EQU                1
                                           T1IE               .EQU                0
                                           _CTIE              .EQU                7
                                           _ADIE              .EQU                6
                                           _INT2IE            .EQU                5
                                           _INT1IE            .EQU                4
                                           _C1IE              .EQU                3
                                           _PWM2IE            .EQU                2
                                           _T2IE              .EQU                1
                                           _T1IE              .EQU                0
                                           
                                           ;Address:0x2D EIE2 Bits-----------------
                                           RXIE               .EQU                5
                                           TXIE               .EQU                4
                                           _RXIE              .EQU                5
                                           _TXIE              .EQU                4
                                           
                                           ;Address:0x2E PCTL Bits-----------------
                                           VREEN              .EQU                7
                                           VREOE              .EQU                6
                                           SLVREN             .EQU                4
                                           POR                .EQU                1
                                           LVR                .EQU                0
                                           _VREEN             .EQU                7
                                           _VREOE             .EQU                6
                                           _SLVREN            .EQU                4
                                           _POR               .EQU                1
                                           _LVR               .EQU                0
                                           
                                           ;Address:0x2F OSCCTL Bits---------------
                                           CKOEN              .EQU                7
                                           IRCS2              .EQU                6
                                           IRCS1              .EQU                5
                                           IRCS0              .EQU                4
                                           _CKOEN             .EQU                7
                                           _IRCS2             .EQU                6
                                           _IRCS1             .EQU                5
                                           _IRCS0             .EQU                4
                                           
                                           ;Address:0x31 ANSEL Bits----------------
                                           ANS7               .EQU                7
                                           ANS6               .EQU                6
                                           ANS4               .EQU                4
                                           ANS3               .EQU                3
                                           ANS1               .EQU                1
                                           ANS0               .EQU                0
                                           _ANS7              .EQU                7
                                           _ANS6              .EQU                6
                                           _ANS4              .EQU                4
                                           _ANS3              .EQU                3
                                           _ANS1              .EQU                1
                                           _ANS0              .EQU                0
                                           
                                           ;Address:0x35 PUR Bits------------------
                                           PUR7               .EQU                7
                                           PUR6               .EQU                6
                                           PUR5               .EQU                5
                                           PUR4               .EQU                4
                                           PUR1               .EQU                1
                                           PUR0               .EQU                0
                                           _PUR7              .EQU                7
                                           _PUR6              .EQU                6
                                           _PUR5              .EQU                5
                                           _PUR4              .EQU                4
                                           _PUR1              .EQU                1
                                           _PUR0              .EQU                0
                                           
                                           ;Address:0x36 IOCL Bits-----------------
                                           IOCL7              .EQU                7
                                           IOCL6              .EQU                6
                                           IOCL5              .EQU                5
                                           IOCL4              .EQU                4
                                           IOCL3              .EQU                3
                                           IOCL1              .EQU                1
                                           IOCL0              .EQU                0
                                           _IOCL7             .EQU                7
                                           _IOCL6             .EQU                6
                                           _IOCL5             .EQU                5
                                           _IOCL4             .EQU                4
                                           _IOCL3             .EQU                3
                                           _IOCL1             .EQU                1
                                           _IOCL0             .EQU                0
                                           
                                           ;Address:0x3F ADCCTL1 Bits--------------
                                           ADCS2              .EQU                6
                                           ADCS1              .EQU                5
                                           ADCS0              .EQU                4
                                           VCFG1              .EQU                3
                                           VCFG0              .EQU                2
                                           _ADCS2             .EQU                6
                                           _ADCS1             .EQU                5
                                           _ADCS0             .EQU                4
                                           _VCFG1             .EQU                3
                                           _VCFG0             .EQU                2
                                           
                                           ;Address:0x50 T3L Bits------------------
                                           T3L7               .EQU                7
                                           T3L6               .EQU                6
                                           T3L5               .EQU                5
                                           T3L4               .EQU                4
                                           T3L3               .EQU                3
                                           T3L2               .EQU                2
                                           T3L1               .EQU                1
                                           T3L0               .EQU                0
                                           _T3L7              .EQU                7
                                           _T3L6              .EQU                6
                                           _T3L5              .EQU                5
                                           _T3L4              .EQU                4
                                           _T3L3              .EQU                3
                                           _T3L2              .EQU                2
                                           _T3L1              .EQU                1
                                           _T3L0              .EQU                0
                                           
                                           ;Address:0x53 CTCTL Bits----------------
                                           CTEN               .EQU                7
                                           CTSTART            .EQU                6
                                           CTCAPS             .EQU                5
                                           CTCMS              .EQU                4
                                           CTCHSEL4           .EQU                4
                                           CTCHSEL3           .EQU                3
                                           CTCHSEL2           .EQU                2
                                           CTCHSEL1           .EQU                1
                                           CTCHSEL0           .EQU                0
                                           _CTEN              .EQU                7
                                           _CTSTART           .EQU                6
                                           _CTCAPS            .EQU                5
                                           _CTCMS             .EQU                4
                                           _CTCHSEL4          .EQU                4
                                           _CTCHSEL3          .EQU                3
                                           _CTCHSEL2          .EQU                2
                                           _CTCHSEL1          .EQU                1
                                           _CTCHSEL0          .EQU                0
                                           
                                           ;Address:0x58 RSCTL Bits----------------
                                           SPEN               .EQU                7
                                           RX9                .EQU                6
                                           SRXEN              .EQU                5
                                           CRXEN              .EQU                4
                                           ADREN              .EQU                3
                                           FRER               .EQU                2
                                           OVFER              .EQU                1
                                           RX9D               .EQU                0
                                           _SPEN              .EQU                7
                                           _RX9               .EQU                6
                                           _SRXEN             .EQU                5
                                           _CRXEN             .EQU                4
                                           _ADREN             .EQU                3
                                           _FRER              .EQU                2
                                           _OVFER             .EQU                1
                                           _RX9D              .EQU                0
                                           
                                           ;Address:0x5E OSCLDOCAL Bits------------
                                           
                                           ;Address:0x77 BRCTL Bits----------------
                                           ABRDOVF            .EQU                7
                                           RCIDLF             .EQU                6
                                           SCKPS              .EQU                4
                                           BRG16              .EQU                3
                                           WUEN               .EQU                1
                                           ADRBEN             .EQU                0
                                           _ABRDOVF           .EQU                7
                                           _RCIDLF            .EQU                6
                                           _SCKPS             .EQU                4
                                           _BRG16             .EQU                3
                                           _WUEN              .EQU                1
                                           _ADRBEN            .EQU                0
                                           
                                           ;Address:0x78 TSCTL Bits----------------
                                           CSRS               .EQU                7
                                           TX9                .EQU                6
                                           TXEN               .EQU                5
                                           SYNC               .EQU                4
                                           SENDB              .EQU                3
                                           HBRG               .EQU                2
                                           TXSRS              .EQU                1
                                           TX9D               .EQU                0
                                           _CSRS              .EQU                7
                                           _TX9               .EQU                6
                                           _TXEN              .EQU                5
                                           _SYNC              .EQU                4
                                           _SENDB             .EQU                3
                                           _HBRG              .EQU                2
                                           _TXSRS             .EQU                1
                                           _TX9D              .EQU                0
                                           
                                           ;Address:0x79 EUBRGL Bits---------------
                                           BRG7               .EQU                7
                                           BRG6               .EQU                6
                                           BRG5               .EQU                5
                                           BRG4               .EQU                4
                                           BRG3               .EQU                3
                                           BRG2               .EQU                2
                                           BRG1               .EQU                1
                                           BRG0               .EQU                0
                                           _BRG7              .EQU                7
                                           _BRG6              .EQU                6
                                           _BRG5              .EQU                5
                                           _BRG4              .EQU                4
                                           _BRG3              .EQU                3
                                           _BRG2              .EQU                2
                                           _BRG1              .EQU                1
                                           _BRG0              .EQU                0
                                           
                                           ;Address:0x7A EUBRGH Bits---------------
                                           BRG15              .EQU                7
                                           BRG14              .EQU                6
                                           BRG13              .EQU                5
                                           BRG12              .EQU                4
                                           BRG11              .EQU                3
                                           BRG10              .EQU                2
                                           BRG9               .EQU                1
                                           BRG8               .EQU                0
                                           _BRG15             .EQU                7
                                           _BRG14             .EQU                6
                                           _BRG13             .EQU                5
                                           _BRG12             .EQU                4
                                           _BRG11             .EQU                3
                                           _BRG10             .EQU                2
                                           _BRG9              .EQU                1
                                           _BRG8              .EQU                0
                                            
                                            
                                           .config
002007   04c0     CPLR	0xc0               
002008   ffff     NOPZ                    
                                           fun.__R2PCL
00070d   530a     MOV	0xa, R1             
00070e   5102     MOV	0x2, R0             
                                           func.__gsinit_startup
00070f   d691     CALL	#0x691             
000710   0008     CRET                    
                                           .code
0006e4   dfff     CALL	#0xfff             
0006e5   5130     MOV	0x30, R0            
0006e6   ffff     NOPZ                    
0006e7   ffff     NOPZ                    
0006e8   dffe     CALL	#0xffe             
0006e9   5137     MOV	0x37, R0            
0006ea   ffff     NOPZ                    
0006eb   ffff     NOPZ                    
0006ec   dffd     CALL	#0xffd             
0006ed   511c     MOV	0x1c, R0            
0006ee   ffff     NOPZ                    
0006ef   ffff     NOPZ                    
0006f0   dffc     CALL	#0xffc             
0006f1   515e     MOV	0x5e, R0            
0006f2   ffff     NOPZ                    
0006f3   ffff     NOPZ                    
0006f4   0008     CRET                    
                                           ID_kf8s_touch_g_lib_0
000671   b001     RRET	R0, #0x1           
000672   b000     RRET	R0, #0             
000673   b002     RRET	R0, #0x2           
000674   b000     RRET	R0, #0             
000675   b004     RRET	R0, #0x4           
000676   b000     RRET	R0, #0             
000677   b008     RRET	R0, #0x8           
000678   b000     RRET	R0, #0             
000679   b010     RRET	R0, #0x10          
00067a   b000     RRET	R0, #0             
00067b   b020     RRET	R0, #0x20          
00067c   b000     RRET	R0, #0             
00067d   b040     RRET	R0, #0x40          
00067e   b000     RRET	R0, #0             
00067f   b080     RRET	R0, #0x80          
000680   b000     RRET	R0, #0             
000681   b000     RRET	R0, #0             
000682   b001     RRET	R0, #0x1           
000683   b000     RRET	R0, #0             
000684   b002     RRET	R0, #0x2           
000685   b000     RRET	R0, #0             
000686   b004     RRET	R0, #0x4           
000687   b000     RRET	R0, #0             
000688   b008     RRET	R0, #0x8           
000689   b000     RRET	R0, #0             
00068a   b010     RRET	R0, #0x10          
00068b   b000     RRET	R0, #0             
00068c   b020     RRET	R0, #0x20          
00068d   b000     RRET	R0, #0             
00068e   b040     RRET	R0, #0x40          
00068f   b000     RRET	R0, #0             
000690   b080     RRET	R0, #0x80          
                                           func.__KF8S_Touch_Process_General_
000510   6003     CLR	0x3, 0              
000511   6503     CLR	0x3, 5              
000512   12a2     RLCR	0xa2               
000513   5187     MOV	0x87, R0            
000514   7c53     JB	0x53, 4              
000515   c51d     JMP	#0x51d              
000516   525f     MOV	R1, 0x5f            
000517   7792     JNB	0x92, 7             
000518   c51b     JMP	#0x51b              
000519   6003     CLR	0x3, 0              
00051a   ff21     RRC	R1                  
00051b   5050     MOV	R0, 0x50            
00051c   c51f     JMP	#0x51f              
00051d   520f     MOV	R1, 0xf             
00051e   500e     MOV	R0, 0xe             
00051f   53ae     MOV	0xae, R1            
000520   51ad     MOV	0xad, R0            
000521   9802     MOV	R0, #0x2            
000522   21ad     ADD	0xad, R0            
000523   7003     JNB	0x3, 0              
000524   0bae     INC	0xae                
000525   9802     MOV	R0, #0x2            
000526   ff10     INC	R0                  
000527   c52b     JMP	#0x52b              
000528   6003     CLR	0x3, 0              
000529   11ae     RRC	0xae                
00052a   11ad     RRC	0xad                
00052b   ff58     DECJZ	R0                
00052c   c528     JMP	#0x528              
00052d   5087     MOV	R0, 0x87            
00052e   80ee     ADD	R0, #0xee           
00052f   f701     LD	R1, [R0]             
000530   53ab     MOV	0xab, R1            
000531   ff10     INC	R0                  
000532   f701     LD	R1, [R0]             
000533   53ac     MOV	0xac, R1            
000534   50ab     MOV	R0, 0xab            
000535   51a9     MOV	0xa9, R0            
000536   53aa     MOV	0xaa, R1            
000537   9802     MOV	R0, #0x2            
000538   21a9     ADD	0xa9, R0            
000539   7003     JNB	0x3, 0              
00053a   0baa     INC	0xaa                
00053b   9802     MOV	R0, #0x2            
00053c   ff10     INC	R0                  
00053d   c541     JMP	#0x541              
00053e   6003     CLR	0x3, 0              
00053f   11aa     RRC	0xaa                
000540   11a9     RRC	0xa9                
000541   ff58     DECJZ	R0                
000542   c53e     JMP	#0x53e              
000543   50a9     MOV	R0, 0xa9            
000544   52aa     MOV	R1, 0xaa            
000545   39ab     SUB	0xab, R0            
000546   7803     JB	0x3, 0               
000547   07ac     DEC	0xac                
000548   3bac     SUB	0xac, R1            
000549   52ae     MOV	R1, 0xae            
00054a   50ad     MOV	R0, 0xad            
00054b   21ab     ADD	0xab, R0            
00054c   7003     JNB	0x3, 0              
00054d   ff11     INC	R1                  
00054e   23ac     ADD	0xac, R1            
00054f   52ab     MOV	R1, 0xab            
000550   5087     MOV	R0, 0x87            
000551   80ee     ADD	R0, #0xee           
000552   f748     ST	[R0], R1             
000553   52ac     MOV	R1, 0xac            
000554   ff10     INC	R0                  
000555   f748     ST	[R0], R1             
000556   7092     JNB	0x92, 0             
000557   c577     JMP	#0x577              
000558   5087     MOV	R0, 0x87            
000559   80ee     ADD	R0, #0xee           
00055a   f701     LD	R1, [R0]             
00055b   5087     MOV	R0, 0x87            
00055c   80de     ADD	R0, #0xde           
00055d   f748     ST	[R0], R1             
00055e   5087     MOV	R0, 0x87            
00055f   80ef     ADD	R0, #0xef           
000560   f701     LD	R1, [R0]             
000561   5087     MOV	R0, 0x87            
000562   80df     ADD	R0, #0xdf           
000563   f748     ST	[R0], R1             
000564   50a2     MOV	R0, 0xa2            
000565   80c1     ADD	R0, #0xc1           
000566   9900     MOV	R1, #0              
000567   f748     ST	[R0], R1             
000568   50a2     MOV	R0, 0xa2            
000569   80c9     ADD	R0, #0xc9           
00056a   9900     MOV	R1, #0              
00056b   f748     ST	[R0], R1             
00056c   9800     MOV	R0, #0              
00056d   30a2     ORL	R0, 0xa2            
00056e   7a03     JB	0x3, 2               
00056f   c57e     JMP	#0x57e              
000570   0b84     INC	0x84                
000571   9824     MOV	R0, #0x24           
000572   3884     SUB	R0, 0x84            
000573   7803     JB	0x3, 0               
000574   c576     JMP	#0x576              
000575   6892     SET	0x92, 0             
000576   c57e     JMP	#0x57e              
000577   d2d8     CALL	#0x2d8             
000578   9800     MOV	R0, #0              
000579   6503     CLR	0x3, 5              
00057a   30a2     ORL	R0, 0xa2            
00057b   7a03     JB	0x3, 2               
00057c   c57e     JMP	#0x57e              
00057d   d009     CALL	#0x9               
00057e   9907     MOV	R1, #0x7            
00057f   9811     MOV	R0, #0x11           
000580   d708     CALL	#0x708             
000581   6503     CLR	0x3, 5              
000582   0ba2     INC	0xa2                
000583   18a2     XOR	R0, 0xa2            
000584   7203     JNB	0x3, 2              
000585   03a2     CLR	0xa2                
000586   7453     JNB	0x53, 4             
000587   c58c     JMP	#0x58c              
000588   030e     CLR	0xe                 
000589   030f     CLR	0xf                 
00058a   600c     CLR	0xc, 0              
00058b   c58d     JMP	#0x58d              
00058c   0350     CLR	0x50                
00058d   6003     CLR	0x3, 0              
00058e   50a2     MOV	R0, 0xa2            
00058f   80f5     ADD	R0, #0xf5           
000590   9906     MOV	R1, #0x6            
000591   7003     JNB	0x3, 0              
000592   ff11     INC	R1                  
000593   d708     CALL	#0x708             
000594   99f0     MOV	R1, #0xf0           
000595   6503     CLR	0x3, 5              
000596   2b53     AND	0x53, R1            
000597   3153     ORL	0x53, R0            
000598   9801     MOV	R0, #0x1            
000599   ff58     DECJZ	R0                
00059a   c599     JMP	#0x599              
00059b   6e53     SET	0x53, 6             
00059c   0000     NOP                     
00059d   7e53     JB	0x53, 6              
00059e   c59b     JMP	#0x59b              
00059f   7453     JNB	0x53, 4             
0005a0   035f     CLR	0x5f                
0005a1   6f2c     SET	0x2c, 7             
0005a2   670c     CLR	0xc, 7              
0005a3   0008     CRET                    
                                           func.__KF8_LIBf_scan_channel_
0002d8   6003     CLR	0x3, 0              
0002d9   6503     CLR	0x3, 5              
0002da   12a2     RLCR	0xa2               
0002db   5187     MOV	0x87, R0            
0002dc   9801     MOV	R0, #0x1            
0002dd   51ad     MOV	0xad, R0            
0002de   03ae     CLR	0xae                
0002df   50a2     MOV	R0, 0xa2            
0002e0   ff10     INC	R0                  
0002e1   c2e6     JMP	#0x2e6              
0002e2   6003     CLR	0x3, 0              
0002e3   6503     CLR	0x3, 5              
0002e4   13ad     RLC	0xad                
0002e5   13ae     RLC	0xae                
0002e6   ff58     DECJZ	R0                
0002e7   c2e2     JMP	#0x2e2              
0002e8   5287     MOV	R1, 0x87            
0002e9   81ee     ADD	R1, #0xee           
0002ea   f708     LD	R0, [R1]             
0002eb   51ab     MOV	0xab, R0            
0002ec   ff11     INC	R1                  
0002ed   f708     LD	R0, [R1]             
0002ee   51ac     MOV	0xac, R0            
0002ef   5287     MOV	R1, 0x87            
0002f0   81de     ADD	R1, #0xde           
0002f1   f708     LD	R0, [R1]             
0002f2   51a9     MOV	0xa9, R0            
0002f3   ff11     INC	R1                  
0002f4   f708     LD	R0, [R1]             
0002f5   51aa     MOV	0xaa, R0            
0002f6   d5a4     CALL	#0x5a4             
0002f7   9907     MOV	R1, #0x7            
0002f8   9818     MOV	R0, #0x18           
0002f9   d708     CALL	#0x708             
0002fa   8080     ADD	R0, #0x80           
0002fb   6503     CLR	0x3, 5              
0002fc   9980     MOV	R1, #0x80           
0002fd   2283     ADD	R1, 0x83            
0002fe   f848     SUB	R0, R1              
0002ff   7803     JB	0x3, 0               
000300   c30a     JMP	#0x30a              
000301   50af     MOV	R0, 0xaf            
000302   28ad     AND	R0, 0xad            
000303   7a03     JB	0x3, 2               
000304   c30a     JMP	#0x30a              
000305   50b0     MOV	R0, 0xb0            
000306   28ae     AND	R0, 0xae            
000307   7a03     JB	0x3, 2               
000308   c30a     JMP	#0x30a              
000309   0b82     INC	0x82                
00030a   52a2     MOV	R1, 0xa2            
00030b   81b9     ADD	R1, #0xb9           
00030c   f708     LD	R0, [R1]             
00030d   5283     MOV	R1, 0x83            
00030e   5385     MOV	0x85, R1            
00030f   3985     SUB	0x85, R0            
000310   6803     SET	0x3, 0              
000311   7f85     JB	0x85, 7              
000312   6003     CLR	0x3, 0              
000313   7803     JB	0x3, 0               
000314   c317     JMP	#0x317              
000315   0585     CPL	0x85                
000316   0b85     INC	0x85                
000317   9907     MOV	R1, #0x7            
000318   9819     MOV	R0, #0x19           
000319   d70d     CALL	#0x70d             
00031a   6503     CLR	0x3, 5              
00031b   5188     MOV	0x88, R0            
00031c   0e88     MOVZ	R0, 0x88           
00031d   8080     ADD	R0, #0x80           
00031e   5189     MOV	0x89, R0            
00031f   0e85     MOVZ	R0, 0x85           
000320   8080     ADD	R0, #0x80           
000321   3889     SUB	R0, 0x89            
000322   7003     JNB	0x3, 0              
000323   c340     JMP	#0x340              
000324   50a2     MOV	R0, 0xa2            
000325   80c9     ADD	R0, #0xc9           
000326   5188     MOV	0x88, R0            
000327   9800     MOV	R0, #0              
000328   5288     MOV	R1, 0x88            
000329   f741     ST	[R1], R0             
00032a   9801     MOV	R0, #0x1            
00032b   5188     MOV	0x88, R0            
00032c   9800     MOV	R0, #0              
00032d   518e     MOV	0x8e, R0            
00032e   0ea2     MOVZ	R0, 0xa2           
00032f   ff10     INC	R0                  
000330   c335     JMP	#0x335              
000331   6003     CLR	0x3, 0              
000332   6503     CLR	0x3, 5              
000333   1388     RLC	0x88                
000334   138e     RLC	0x8e                
000335   ff58     DECJZ	R0                
000336   c331     JMP	#0x331              
000337   0588     CPL	0x88                
000338   058e     CPL	0x8e                
000339   0e88     MOVZ	R0, 0x88           
00033a   518a     MOV	0x8a, R0            
00033b   29a7     AND	0xa7, R0            
00033c   0e8e     MOVZ	R0, 0x8e           
00033d   518b     MOV	0x8b, R0            
00033e   29a8     AND	0xa8, R0            
00033f   c353     JMP	#0x353              
000340   9801     MOV	R0, #0x1            
000341   5188     MOV	0x88, R0            
000342   9800     MOV	R0, #0              
000343   518e     MOV	0x8e, R0            
000344   0ea2     MOVZ	R0, 0xa2           
000345   ff10     INC	R0                  
000346   c34b     JMP	#0x34b              
000347   6003     CLR	0x3, 0              
000348   6503     CLR	0x3, 5              
000349   1388     RLC	0x88                
00034a   138e     RLC	0x8e                
00034b   ff58     DECJZ	R0                
00034c   c347     JMP	#0x347              
00034d   0e88     MOVZ	R0, 0x88           
00034e   518a     MOV	0x8a, R0            
00034f   31a7     ORL	0xa7, R0            
000350   0e8e     MOVZ	R0, 0x8e           
000351   518b     MOV	0x8b, R0            
000352   31a8     ORL	0xa8, R0            
000353   50a2     MOV	R0, 0xa2            
000354   80b9     ADD	R0, #0xb9           
000355   5188     MOV	0x88, R0            
000356   0e83     MOVZ	R0, 0x83           
000357   5288     MOV	R1, 0x88            
000358   f741     ST	[R1], R0             
000359   50a2     MOV	R0, 0xa2            
00035a   a801     XOR	R0, #0x1            
00035b   7a03     JB	0x3, 2               
00035c   c36b     JMP	#0x36b              
00035d   50b9     MOV	R0, 0xb9            
00035e   52ba     MOV	R1, 0xba            
00035f   8080     ADD	R0, #0x80           
000360   8180     ADD	R1, #0x80           
000361   f841     SUB	R1, R0              
000362   7803     JB	0x3, 0               
000363   c368     JMP	#0x368              
000364   9801     MOV	R0, #0x1            
000365   5181     MOV	0x81, R0            
000366   0380     CLR	0x80                
000367   c36b     JMP	#0x36b              
000368   9801     MOV	R0, #0x1            
000369   5180     MOV	0x80, R0            
00036a   0381     CLR	0x81                
00036b   9802     MOV	R0, #0x2            
00036c   38a2     SUB	R0, 0xa2            
00036d   7803     JB	0x3, 0               
00036e   c389     JMP	#0x389              
00036f   52a2     MOV	R1, 0xa2            
000370   81b9     ADD	R1, #0xb9           
000371   f708     LD	R0, [R1]             
000372   8080     ADD	R0, #0x80           
000373   5183     MOV	0x83, R0            
000374   5281     MOV	R1, 0x81            
000375   81b9     ADD	R1, #0xb9           
000376   f708     LD	R0, [R1]             
000377   8080     ADD	R0, #0x80           
000378   3883     SUB	R0, 0x83            
000379   7803     JB	0x3, 0               
00037a   c389     JMP	#0x389              
00037b   5280     MOV	R1, 0x80            
00037c   81b9     ADD	R1, #0xb9           
00037d   f708     LD	R0, [R1]             
00037e   8080     ADD	R0, #0x80           
00037f   3883     SUB	R0, 0x83            
000380   7003     JNB	0x3, 0              
000381   c385     JMP	#0x385              
000382   50a2     MOV	R0, 0xa2            
000383   5181     MOV	0x81, R0            
000384   c389     JMP	#0x389              
000385   5080     MOV	R0, 0x80            
000386   5181     MOV	0x81, R0            
000387   50a2     MOV	R0, 0xa2            
000388   5180     MOV	0x80, R0            
000389   7192     JNB	0x92, 1             
00038a   c412     JMP	#0x412              
00038b   50a2     MOV	R0, 0xa2            
00038c   80fd     ADD	R0, #0xfd           
00038d   9906     MOV	R1, #0x6            
00038e   7003     JNB	0x3, 0              
00038f   ff11     INC	R1                  
000390   d708     CALL	#0x708             
000391   6503     CLR	0x3, 5              
000392   5183     MOV	0x83, R0            
000393   9806     MOV	R0, #0x6            
000394   3983     SUB	0x83, R0            
000395   50a2     MOV	R0, 0xa2            
000396   80b9     ADD	R0, #0xb9           
000397   5188     MOV	0x88, R0            
000398   5288     MOV	R1, 0x88            
000399   f708     LD	R0, [R1]             
00039a   518a     MOV	0x8a, R0            
00039b   0e8a     MOVZ	R0, 0x8a           
00039c   8080     ADD	R0, #0x80           
00039d   5189     MOV	0x89, R0            
00039e   0e83     MOVZ	R0, 0x83           
00039f   8080     ADD	R0, #0x80           
0003a0   3889     SUB	R0, 0x89            
0003a1   7003     JNB	0x3, 0              
0003a2   c403     JMP	#0x403              
0003a3   50a2     MOV	R0, 0xa2            
0003a4   80c1     ADD	R0, #0xc1           
0003a5   5188     MOV	0x88, R0            
0003a6   5288     MOV	R1, 0x88            
0003a7   f708     LD	R0, [R1]             
0003a8   518a     MOV	0x8a, R0            
0003a9   9907     MOV	R1, #0x7            
0003aa   9812     MOV	R0, #0x12           
0003ab   d70d     CALL	#0x70d             
0003ac   6503     CLR	0x3, 5              
0003ad   5188     MOV	0x88, R0            
0003ae   0e8a     MOVZ	R0, 0x8a           
0003af   3888     SUB	R0, 0x88            
0003b0   7003     JNB	0x3, 0              
0003b1   c412     JMP	#0x412              
0003b2   9907     MOV	R1, #0x7            
0003b3   9812     MOV	R0, #0x12           
0003b4   d708     CALL	#0x708             
0003b5   6003     CLR	0x3, 0              
0003b6   ff18     RLC	R0                  
0003b7   6503     CLR	0x3, 5              
0003b8   5184     MOV	0x84, R0            
0003b9   52a2     MOV	R1, 0xa2            
0003ba   81c1     ADD	R1, #0xc1           
0003bb   f708     LD	R0, [R1]             
0003bc   3884     SUB	R0, 0x84            
0003bd   7803     JB	0x3, 0               
0003be   c3c3     JMP	#0x3c3              
0003bf   f708     LD	R0, [R1]             
0003c0   ff10     INC	R0                  
0003c1   f741     ST	[R1], R0             
0003c2   c402     JMP	#0x402              
0003c3   0208     CLR	R0                  
0003c4   f741     ST	[R1], R0             
0003c5   50a2     MOV	R0, 0xa2            
0003c6   80f5     ADD	R0, #0xf5           
0003c7   9906     MOV	R1, #0x6            
0003c8   7003     JNB	0x3, 0              
0003c9   ff11     INC	R1                  
0003ca   d708     CALL	#0x708             
0003cb   6003     CLR	0x3, 0              
0003cc   ff18     RLC	R0                  
0003cd   6503     CLR	0x3, 5              
0003ce   5184     MOV	0x84, R0            
0003cf   8071     ADD	R0, #0x71           
0003d0   9906     MOV	R1, #0x6            
0003d1   7003     JNB	0x3, 0              
0003d2   ff11     INC	R1                  
0003d3   d708     CALL	#0x708             
0003d4   ff00     CPL	R0                  
0003d5   6503     CLR	0x3, 5              
0003d6   29b7     AND	0xb7, R0            
0003d7   5084     MOV	R0, 0x84            
0003d8   ff10     INC	R0                  
0003d9   8071     ADD	R0, #0x71           
0003da   9906     MOV	R1, #0x6            
0003db   7003     JNB	0x3, 0              
0003dc   ff11     INC	R1                  
0003dd   d708     CALL	#0x708             
0003de   ff00     CPL	R0                  
0003df   6503     CLR	0x3, 5              
0003e0   29b8     AND	0xb8, R0            
0003e1   9800     MOV	R0, #0              
0003e2   3091     ORL	R0, 0x91            
0003e3   7a03     JB	0x3, 2               
0003e4   0791     DEC	0x91                
0003e5   9800     MOV	R0, #0              
0003e6   3091     ORL	R0, 0x91            
0003e7   7203     JNB	0x3, 2              
0003e8   c3f9     JMP	#0x3f9              
0003e9   5090     MOV	R0, 0x90            
0003ea   18a2     XOR	R0, 0xa2            
0003eb   7a03     JB	0x3, 2               
0003ec   c3fb     JMP	#0x3fb              
0003ed   508f     MOV	R0, 0x8f            
0003ee   1890     XOR	R0, 0x90            
0003ef   7a03     JB	0x3, 2               
0003f0   c3f6     JMP	#0x3f6              
0003f1   98ff     MOV	R0, #0xff           
0003f2   5190     MOV	0x90, R0            
0003f3   9800     MOV	R0, #0              
0003f4   5191     MOV	0x91, R0            
0003f5   c3fb     JMP	#0x3fb              
0003f6   508f     MOV	R0, 0x8f            
0003f7   5190     MOV	0x90, R0            
0003f8   c3fb     JMP	#0x3fb              
0003f9   98ff     MOV	R0, #0xff           
0003fa   5190     MOV	0x90, R0            
0003fb   98ff     MOV	R0, #0xff           
0003fc   518f     MOV	0x8f, R0            
0003fd   9800     MOV	R0, #0              
0003fe   51b1     MOV	0xb1, R0            
0003ff   51b2     MOV	0xb2, R0            
000400   51b3     MOV	0xb3, R0            
000401   51b4     MOV	0xb4, R0            
000402   c412     JMP	#0x412              
000403   9907     MOV	R1, #0x7            
000404   9812     MOV	R0, #0x12           
000405   d708     CALL	#0x708             
000406   ff10     INC	R0                  
000407   6503     CLR	0x3, 5              
000408   5184     MOV	0x84, R0            
000409   52a2     MOV	R1, 0xa2            
00040a   81c1     ADD	R1, #0xc1           
00040b   f708     LD	R0, [R1]             
00040c   3884     SUB	R0, 0x84            
00040d   7003     JNB	0x3, 0              
00040e   c412     JMP	#0x412              
00040f   f708     LD	R0, [R1]             
000410   ff08     DEC	R0                  
000411   f741     ST	[R1], R0             
000412   0008     CRET                    
                                           func.__KF8_LiBf_KEY_Deal_AND_BaseLine_Up
000009   9801     MOV	R0, #0x1            
00000a   6503     CLR	0x3, 5              
00000b   51ad     MOV	0xad, R0            
00000c   03ae     CLR	0xae                
00000d   0386     CLR	0x86                
00000e   9907     MOV	R1, #0x7            
00000f   9811     MOV	R0, #0x11           
000010   d70d     CALL	#0x70d             
000011   6503     CLR	0x3, 5              
000012   5188     MOV	0x88, R0            
000013   0e88     MOVZ	R0, 0x88           
000014   3886     SUB	R0, 0x86            
000015   7003     JNB	0x3, 0              
000016   c27a     JMP	#0x27a              
000017   6003     CLR	0x3, 0              
000018   1286     RLCR	0x86               
000019   5187     MOV	0x87, R0            
00001a   5086     MOV	R0, 0x86            
00001b   80f5     ADD	R0, #0xf5           
00001c   9906     MOV	R1, #0x6            
00001d   7003     JNB	0x3, 0              
00001e   ff11     INC	R1                  
00001f   d708     CALL	#0x708             
000020   6503     CLR	0x3, 5              
000021   5184     MOV	0x84, R0            
000022   981b     MOV	R0, #0x1b           
000023   9907     MOV	R1, #0x7            
000024   d708     CALL	#0x708             
000025   1884     XOR	R0, 0x84            
000026   7a03     JB	0x3, 2               
000027   c039     JMP	#0x39               
000028   981a     MOV	R0, #0x1a           
000029   9907     MOV	R1, #0x7            
00002a   d708     CALL	#0x708             
00002b   6503     CLR	0x3, 5              
00002c   5183     MOV	0x83, R0            
00002d   5086     MOV	R0, 0x86            
00002e   80b9     ADD	R0, #0xb9           
00002f   f701     LD	R1, [R0]             
000030   f7f9     JB	R1, 7                
000031   c034     JMP	#0x34               
000032   ff01     CPL	R1                  
000033   ff11     INC	R1                  
000034   3a83     SUB	R1, 0x83            
000035   7003     JNB	0x3, 0              
000036   c039     JMP	#0x39               
000037   6992     SET	0x92, 1             
000038   0393     CLR	0x93                
000039   6503     CLR	0x3, 5              
00003a   5086     MOV	R0, 0x86            
00003b   80b9     ADD	R0, #0xb9           
00003c   5188     MOV	0x88, R0            
00003d   5288     MOV	R1, 0x88            
00003e   f708     LD	R0, [R1]             
00003f   5189     MOV	0x89, R0            
000040   9907     MOV	R1, #0x7            
000041   9817     MOV	R0, #0x17           
000042   d70d     CALL	#0x70d             
000043   6503     CLR	0x3, 5              
000044   5188     MOV	0x88, R0            
000045   0e89     MOVZ	R0, 0x89           
000046   8080     ADD	R0, #0x80           
000047   518e     MOV	0x8e, R0            
000048   0e88     MOVZ	R0, 0x88           
000049   8080     ADD	R0, #0x80           
00004a   388e     SUB	R0, 0x8e            
00004b   7003     JNB	0x3, 0              
00004c   c070     JMP	#0x70               
00004d   5086     MOV	R0, 0x86            
00004e   80c9     ADD	R0, #0xc9           
00004f   f701     LD	R1, [R0]             
000050   9864     MOV	R0, #0x64           
000051   f941     XOR	R1, R0              
000052   7a03     JB	0x3, 2               
000053   c06f     JMP	#0x6f               
000054   5087     MOV	R0, 0x87            
000055   80ee     ADD	R0, #0xee           
000056   f701     LD	R1, [R0]             
000057   5087     MOV	R0, 0x87            
000058   80de     ADD	R0, #0xde           
000059   f748     ST	[R0], R1             
00005a   5087     MOV	R0, 0x87            
00005b   80ef     ADD	R0, #0xef           
00005c   f701     LD	R1, [R0]             
00005d   5087     MOV	R0, 0x87            
00005e   80df     ADD	R0, #0xdf           
00005f   f748     ST	[R0], R1             
000060   5086     MOV	R0, 0x86            
000061   80c1     ADD	R0, #0xc1           
000062   f701     LD	R1, [R0]             
000063   5384     MOV	0x84, R1            
000064   9812     MOV	R0, #0x12           
000065   9907     MOV	R1, #0x7            
000066   d708     CALL	#0x708             
000067   3884     SUB	R0, 0x84            
000068   7003     JNB	0x3, 0              
000069   c06f     JMP	#0x6f               
00006a   6503     CLR	0x3, 5              
00006b   5086     MOV	R0, 0x86            
00006c   80c1     ADD	R0, #0xc1           
00006d   9900     MOV	R1, #0              
00006e   f748     ST	[R0], R1             
00006f   c153     JMP	#0x153              
000070   5086     MOV	R0, 0x86            
000071   80b9     ADD	R0, #0xb9           
000072   5188     MOV	0x88, R0            
000073   5288     MOV	R1, 0x88            
000074   f708     LD	R0, [R1]             
000075   518a     MOV	0x8a, R0            
000076   9907     MOV	R1, #0x7            
000077   9818     MOV	R0, #0x18           
000078   d70d     CALL	#0x70d             
000079   6503     CLR	0x3, 5              
00007a   5188     MOV	0x88, R0            
00007b   0e88     MOVZ	R0, 0x88           
00007c   8080     ADD	R0, #0x80           
00007d   518e     MOV	0x8e, R0            
00007e   0e8a     MOVZ	R0, 0x8a           
00007f   8080     ADD	R0, #0x80           
000080   388e     SUB	R0, 0x8e            
000081   7003     JNB	0x3, 0              
000082   c0e8     JMP	#0xe8               
000083   9816     MOV	R0, #0x16           
000084   9907     MOV	R1, #0x7            
000085   d708     CALL	#0x708             
000086   6503     CLR	0x3, 5              
000087   3882     SUB	R0, 0x82            
000088   7803     JB	0x3, 0               
000089   c08c     JMP	#0x8c               
00008a   6992     SET	0x92, 1             
00008b   0393     CLR	0x93                
00008c   7992     JB	0x92, 1              
00008d   c0ac     JMP	#0xac               
00008e   5086     MOV	R0, 0x86            
00008f   80c9     ADD	R0, #0xc9           
000090   f701     LD	R1, [R0]             
000091   a9ec     XOR	R1, #0xec           
000092   7203     JNB	0x3, 2              
000093   c09b     JMP	#0x9b               
000094   9813     MOV	R0, #0x13           
000095   9907     MOV	R1, #0x7            
000096   d708     CALL	#0x708             
000097   6503     CLR	0x3, 5              
000098   1893     XOR	R0, 0x93            
000099   7a03     JB	0x3, 2               
00009a   c0ab     JMP	#0xab               
00009b   5087     MOV	R0, 0x87            
00009c   80ee     ADD	R0, #0xee           
00009d   f701     LD	R1, [R0]             
00009e   5087     MOV	R0, 0x87            
00009f   80de     ADD	R0, #0xde           
0000a0   f748     ST	[R0], R1             
0000a1   5087     MOV	R0, 0x87            
0000a2   80ef     ADD	R0, #0xef           
0000a3   f701     LD	R1, [R0]             
0000a4   5087     MOV	R0, 0x87            
0000a5   80df     ADD	R0, #0xdf           
0000a6   f748     ST	[R0], R1             
0000a7   50ad     MOV	R0, 0xad            
0000a8   31af     ORL	0xaf, R0            
0000a9   50ae     MOV	R0, 0xae            
0000aa   31b0     ORL	0xb0, R0            
0000ab   c153     JMP	#0x153              
0000ac   5086     MOV	R0, 0x86            
0000ad   80c9     ADD	R0, #0xc9           
0000ae   f701     LD	R1, [R0]             
0000af   5383     MOV	0x83, R1            
0000b0   9907     MOV	R1, #0x7            
0000b1   9815     MOV	R0, #0x15           
0000b2   d708     CALL	#0x708             
0000b3   6503     CLR	0x3, 5              
0000b4   1883     XOR	R0, 0x83            
0000b5   7a03     JB	0x3, 2               
0000b6   c0e7     JMP	#0xe7               
0000b7   5086     MOV	R0, 0x86            
0000b8   80c1     ADD	R0, #0xc1           
0000b9   f701     LD	R1, [R0]             
0000ba   5384     MOV	0x84, R1            
0000bb   9812     MOV	R0, #0x12           
0000bc   9907     MOV	R1, #0x7            
0000bd   d708     CALL	#0x708             
0000be   6503     CLR	0x3, 5              
0000bf   3884     SUB	R0, 0x84            
0000c0   7003     JNB	0x3, 0              
0000c1   c0df     JMP	#0xdf               
0000c2   5091     MOV	R0, 0x91            
0000c3   a802     XOR	R0, #0x2            
0000c4   7a03     JB	0x3, 2               
0000c5   c0d3     JMP	#0xd3               
0000c6   5087     MOV	R0, 0x87            
0000c7   80ee     ADD	R0, #0xee           
0000c8   f701     LD	R1, [R0]             
0000c9   5087     MOV	R0, 0x87            
0000ca   80de     ADD	R0, #0xde           
0000cb   f748     ST	[R0], R1             
0000cc   5087     MOV	R0, 0x87            
0000cd   80ef     ADD	R0, #0xef           
0000ce   f701     LD	R1, [R0]             
0000cf   5087     MOV	R0, 0x87            
0000d0   80df     ADD	R0, #0xdf           
0000d1   f748     ST	[R0], R1             
0000d2   c0e3     JMP	#0xe3               
0000d3   5087     MOV	R0, 0x87            
0000d4   80de     ADD	R0, #0xde           
0000d5   f701     LD	R1, [R0]             
0000d6   81ff     ADD	R1, #0xff           
0000d7   f748     ST	[R0], R1             
0000d8   7003     JNB	0x3, 0              
0000d9   c0e3     JMP	#0xe3               
0000da   ff10     INC	R0                  
0000db   f701     LD	R1, [R0]             
0000dc   ff09     DEC	R1                  
0000dd   f748     ST	[R0], R1             
0000de   c0e3     JMP	#0xe3               
0000df   50ad     MOV	R0, 0xad            
0000e0   31af     ORL	0xaf, R0            
0000e1   50ae     MOV	R0, 0xae            
0000e2   31b0     ORL	0xb0, R0            
0000e3   5086     MOV	R0, 0x86            
0000e4   80c9     ADD	R0, #0xc9           
0000e5   9900     MOV	R1, #0              
0000e6   f748     ST	[R0], R1             
0000e7   c153     JMP	#0x153              
0000e8   7192     JNB	0x92, 1             
0000e9   c0ee     JMP	#0xee               
0000ea   04ad     CPLR	0xad               
0000eb   29af     AND	0xaf, R0            
0000ec   04ae     CPLR	0xae               
0000ed   29b0     AND	0xb0, R0            
0000ee   5086     MOV	R0, 0x86            
0000ef   80c9     ADD	R0, #0xc9           
0000f0   f701     LD	R1, [R0]             
0000f1   5383     MOV	0x83, R1            
0000f2   9815     MOV	R0, #0x15           
0000f3   9907     MOV	R1, #0x7            
0000f4   d708     CALL	#0x708             
0000f5   6503     CLR	0x3, 5              
0000f6   1883     XOR	R0, 0x83            
0000f7   7203     JNB	0x3, 2              
0000f8   c100     JMP	#0x100              
0000f9   9907     MOV	R1, #0x7            
0000fa   9814     MOV	R0, #0x14           
0000fb   d708     CALL	#0x708             
0000fc   6503     CLR	0x3, 5              
0000fd   1883     XOR	R0, 0x83            
0000fe   7a03     JB	0x3, 2               
0000ff   c153     JMP	#0x153              
000100   5086     MOV	R0, 0x86            
000101   80c9     ADD	R0, #0xc9           
000102   9900     MOV	R1, #0              
000103   f748     ST	[R0], R1             
000104   5087     MOV	R0, 0x87            
000105   80de     ADD	R0, #0xde           
000106   f701     LD	R1, [R0]             
000107   53ab     MOV	0xab, R1            
000108   ff10     INC	R0                  
000109   f701     LD	R1, [R0]             
00010a   53ac     MOV	0xac, R1            
00010b   9901     MOV	R1, #0x1            
00010c   6003     CLR	0x3, 0              
00010d   11ac     RRC	0xac                
00010e   11ab     RRC	0xab                
00010f   6003     CLR	0x3, 0              
000110   ff19     RLC	R1                  
000111   f8c8     MOV	R0, R1              
000112   a808     XOR	R0, #0x8            
000113   7a03     JB	0x3, 2               
000114   c10c     JMP	#0x10c              
000115   5087     MOV	R0, 0x87            
000116   80ee     ADD	R0, #0xee           
000117   f701     LD	R1, [R0]             
000118   53a9     MOV	0xa9, R1            
000119   ff10     INC	R0                  
00011a   f701     LD	R1, [R0]             
00011b   53aa     MOV	0xaa, R1            
00011c   9901     MOV	R1, #0x1            
00011d   6003     CLR	0x3, 0              
00011e   11aa     RRC	0xaa                
00011f   11a9     RRC	0xa9                
000120   6003     CLR	0x3, 0              
000121   ff19     RLC	R1                  
000122   f8c8     MOV	R0, R1              
000123   a808     XOR	R0, #0x8            
000124   7a03     JB	0x3, 2               
000125   c11d     JMP	#0x11d              
000126   52ab     MOV	R1, 0xab            
000127   3ba9     SUB	0xa9, R1            
000128   52ac     MOV	R1, 0xac            
000129   7803     JB	0x3, 0               
00012a   ff11     INC	R1                  
00012b   3baa     SUB	0xaa, R1            
00012c   5087     MOV	R0, 0x87            
00012d   80de     ADD	R0, #0xde           
00012e   f701     LD	R1, [R0]             
00012f   22a9     ADD	R1, 0xa9            
000130   f748     ST	[R0], R1             
000131   ff10     INC	R0                  
000132   f701     LD	R1, [R0]             
000133   7003     JNB	0x3, 0              
000134   ff11     INC	R1                  
000135   22aa     ADD	R1, 0xaa            
000136   f748     ST	[R0], R1             
000137   5086     MOV	R0, 0x86            
000138   80b9     ADD	R0, #0xb9           
000139   f701     LD	R1, [R0]             
00013a   f7b9     JNB	R1, 7               
00013b   c148     JMP	#0x148              
00013c   5087     MOV	R0, 0x87            
00013d   80de     ADD	R0, #0xde           
00013e   f701     LD	R1, [R0]             
00013f   81ff     ADD	R1, #0xff           
000140   f748     ST	[R0], R1             
000141   7003     JNB	0x3, 0              
000142   c153     JMP	#0x153              
000143   ff10     INC	R0                  
000144   f701     LD	R1, [R0]             
000145   ff09     DEC	R1                  
000146   f748     ST	[R0], R1             
000147   c153     JMP	#0x153              
000148   5087     MOV	R0, 0x87            
000149   80de     ADD	R0, #0xde           
00014a   f701     LD	R1, [R0]             
00014b   8101     ADD	R1, #0x1            
00014c   f748     ST	[R0], R1             
00014d   7803     JB	0x3, 0               
00014e   c153     JMP	#0x153              
00014f   ff10     INC	R0                  
000150   f701     LD	R1, [R0]             
000151   ff11     INC	R1                  
000152   f748     ST	[R0], R1             
000153   6503     CLR	0x3, 5              
000154   7992     JB	0x92, 1              
000155   c165     JMP	#0x165              
000156   5086     MOV	R0, 0x86            
000157   80c1     ADD	R0, #0xc1           
000158   f701     LD	R1, [R0]             
000159   5384     MOV	0x84, R1            
00015a   9907     MOV	R1, #0x7            
00015b   9812     MOV	R0, #0x12           
00015c   d708     CALL	#0x708             
00015d   6503     CLR	0x3, 5              
00015e   3984     SUB	0x84, R0            
00015f   7003     JNB	0x3, 0              
000160   c165     JMP	#0x165              
000161   5086     MOV	R0, 0x86            
000162   80c1     ADD	R0, #0xc1           
000163   9900     MOV	R1, #0              
000164   f748     ST	[R0], R1             
000165   5086     MOV	R0, 0x86            
000166   80b9     ADD	R0, #0xb9           
000167   5188     MOV	0x88, R0            
000168   5288     MOV	R1, 0x88            
000169   f708     LD	R0, [R1]             
00016a   518b     MOV	0x8b, R0            
00016b   6803     SET	0x3, 0              
00016c   7f8b     JB	0x8b, 7              
00016d   6003     CLR	0x3, 0              
00016e   7003     JNB	0x3, 0              
00016f   c176     JMP	#0x176              
000170   5086     MOV	R0, 0x86            
000171   80c9     ADD	R0, #0xc9           
000172   f701     LD	R1, [R0]             
000173   ff09     DEC	R1                  
000174   f748     ST	[R0], R1             
000175   c17b     JMP	#0x17b              
000176   5086     MOV	R0, 0x86            
000177   80c9     ADD	R0, #0xc9           
000178   f701     LD	R1, [R0]             
000179   ff11     INC	R1                  
00017a   f748     ST	[R0], R1             
00017b   7192     JNB	0x92, 1             
00017c   c275     JMP	#0x275              
00017d   0e80     MOVZ	R0, 0x80           
00017e   1886     XOR	R0, 0x86            
00017f   7203     JNB	0x3, 2              
000180   c185     JMP	#0x185              
000181   0e81     MOVZ	R0, 0x81           
000182   1886     XOR	R0, 0x86            
000183   7a03     JB	0x3, 2               
000184   c262     JMP	#0x262              
000185   5086     MOV	R0, 0x86            
000186   80b9     ADD	R0, #0xb9           
000187   5188     MOV	0x88, R0            
000188   5288     MOV	R1, 0x88            
000189   f708     LD	R0, [R1]             
00018a   518b     MOV	0x8b, R0            
00018b   98fd     MOV	R0, #0xfd           
00018c   2086     ADD	R0, 0x86            
00018d   5188     MOV	0x88, R0            
00018e   9806     MOV	R0, #0x6            
00018f   518a     MOV	0x8a, R0            
000190   0208     CLR	R0                  
000191   7003     JNB	0x3, 0              
000192   ff10     INC	R0                  
000193   7203     JNB	0x3, 2              
000194   c196     JMP	#0x196              
000195   218a     ADD	0x8a, R0            
000196   528a     MOV	R1, 0x8a            
000197   5088     MOV	R0, 0x88            
000198   d70d     CALL	#0x70d             
000199   6503     CLR	0x3, 5              
00019a   518c     MOV	0x8c, R0            
00019b   0e8c     MOVZ	R0, 0x8c           
00019c   8080     ADD	R0, #0x80           
00019d   518e     MOV	0x8e, R0            
00019e   0e8b     MOVZ	R0, 0x8b           
00019f   8080     ADD	R0, #0x80           
0001a0   388e     SUB	R0, 0x8e            
0001a1   7003     JNB	0x3, 0              
0001a2   c262     JMP	#0x262              
0001a3   9801     MOV	R0, #0x1            
0001a4   5188     MOV	0x88, R0            
0001a5   9800     MOV	R0, #0              
0001a6   518a     MOV	0x8a, R0            
0001a7   0e86     MOVZ	R0, 0x86           
0001a8   ff10     INC	R0                  
0001a9   c1ae     JMP	#0x1ae              
0001aa   6003     CLR	0x3, 0              
0001ab   6503     CLR	0x3, 5              
0001ac   1388     RLC	0x88                
0001ad   138a     RLC	0x8a                
0001ae   ff58     DECJZ	R0                
0001af   c1aa     JMP	#0x1aa              
0001b0   0e88     MOVZ	R0, 0x88           
0001b1   518b     MOV	0x8b, R0            
0001b2   28a7     AND	R0, 0xa7            
0001b3   5188     MOV	0x88, R0            
0001b4   0e8a     MOVZ	R0, 0x8a           
0001b5   518c     MOV	0x8c, R0            
0001b6   28a8     AND	R0, 0xa8            
0001b7   518a     MOV	0x8a, R0            
0001b8   0e88     MOVZ	R0, 0x88           
0001b9   308a     ORL	R0, 0x8a            
0001ba   7203     JNB	0x3, 2              
0001bb   c1d5     JMP	#0x1d5              
0001bc   5086     MOV	R0, 0x86            
0001bd   80c1     ADD	R0, #0xc1           
0001be   5188     MOV	0x88, R0            
0001bf   5288     MOV	R1, 0x88            
0001c0   f708     LD	R0, [R1]             
0001c1   518b     MOV	0x8b, R0            
0001c2   9907     MOV	R1, #0x7            
0001c3   9812     MOV	R0, #0x12           
0001c4   d70d     CALL	#0x70d             
0001c5   6503     CLR	0x3, 5              
0001c6   5188     MOV	0x88, R0            
0001c7   0e88     MOVZ	R0, 0x88           
0001c8   388b     SUB	R0, 0x8b            
0001c9   7003     JNB	0x3, 0              
0001ca   c1d5     JMP	#0x1d5              
0001cb   5086     MOV	R0, 0x86            
0001cc   80c1     ADD	R0, #0xc1           
0001cd   5188     MOV	0x88, R0            
0001ce   5288     MOV	R1, 0x88            
0001cf   f708     LD	R0, [R1]             
0001d0   518c     MOV	0x8c, R0            
0001d1   0b8c     INC	0x8c                
0001d2   0e8c     MOVZ	R0, 0x8c           
0001d3   5288     MOV	R1, 0x88            
0001d4   f741     ST	[R1], R0             
0001d5   9900     MOV	R1, #0              
0001d6   9802     MOV	R0, #0x2            
0001d7   d70d     CALL	#0x70d             
0001d8   6503     CLR	0x3, 5              
0001d9   5188     MOV	0x88, R0            
0001da   9900     MOV	R1, #0              
0001db   9803     MOV	R0, #0x3            
0001dc   d70d     CALL	#0x70d             
0001dd   6503     CLR	0x3, 5              
0001de   518b     MOV	0x8b, R0            
0001df   0e88     MOVZ	R0, 0x88           
0001e0   308b     ORL	R0, 0x8b            
0001e1   7203     JNB	0x3, 2              
0001e2   c1ff     JMP	#0x1ff              
0001e3   0e91     MOVZ	R0, 0x91           
0001e4   a801     XOR	R0, #0x1            
0001e5   7a03     JB	0x3, 2               
0001e6   c1ff     JMP	#0x1ff              
0001e7   0e8b     MOVZ	R0, 0x8b           
0001e8   38b2     SUB	R0, 0xb2            
0001e9   7a03     JB	0x3, 2               
0001ea   c1ed     JMP	#0x1ed              
0001eb   0e88     MOVZ	R0, 0x88           
0001ec   38b1     SUB	R0, 0xb1            
0001ed   7003     JNB	0x3, 0              
0001ee   c1ff     JMP	#0x1ff              
0001ef   0bb1     INC	0xb1                
0001f0   7a03     JB	0x3, 2               
0001f1   c1f3     JMP	#0x1f3              
0001f2   0bb2     INC	0xb2                
0001f3   0e88     MOVZ	R0, 0x88           
0001f4   18b1     XOR	R0, 0xb1            
0001f5   7a03     JB	0x3, 2               
0001f6   c1ff     JMP	#0x1ff              
0001f7   0e8b     MOVZ	R0, 0x8b           
0001f8   18b2     XOR	R0, 0xb2            
0001f9   7a03     JB	0x3, 2               
0001fa   c1ff     JMP	#0x1ff              
0001fb   9802     MOV	R0, #0x2            
0001fc   5191     MOV	0x91, R0            
0001fd   0e90     MOVZ	R0, 0x90           
0001fe   518f     MOV	0x8f, R0            
0001ff   5086     MOV	R0, 0x86            
000200   80c1     ADD	R0, #0xc1           
000201   5188     MOV	0x88, R0            
000202   5288     MOV	R1, 0x88            
000203   f708     LD	R0, [R1]             
000204   518c     MOV	0x8c, R0            
000205   9907     MOV	R1, #0x7            
000206   9812     MOV	R0, #0x12           
000207   d70d     CALL	#0x70d             
000208   6503     CLR	0x3, 5              
000209   5188     MOV	0x88, R0            
00020a   0e88     MOVZ	R0, 0x88           
00020b   188c     XOR	R0, 0x8c            
00020c   7a03     JB	0x3, 2               
00020d   c275     JMP	#0x275              
00020e   0eb7     MOVZ	R0, 0xb7           
00020f   30b8     ORL	R0, 0xb8            
000210   7203     JNB	0x3, 2              
000211   c23a     JMP	#0x23a              
000212   5091     MOV	R0, 0x91            
000213   a801     XOR	R0, #0x1            
000214   7a03     JB	0x3, 2               
000215   c235     JMP	#0x235              
000216   9802     MOV	R0, #0x2            
000217   5191     MOV	0x91, R0            
000218   5086     MOV	R0, 0x86            
000219   518f     MOV	0x8f, R0            
00021a   5086     MOV	R0, 0x86            
00021b   80f5     ADD	R0, #0xf5           
00021c   9906     MOV	R1, #0x6            
00021d   7003     JNB	0x3, 0              
00021e   ff11     INC	R1                  
00021f   d708     CALL	#0x708             
000220   6003     CLR	0x3, 0              
000221   ff18     RLC	R0                  
000222   6503     CLR	0x3, 5              
000223   5184     MOV	0x84, R0            
000224   8071     ADD	R0, #0x71           
000225   9906     MOV	R1, #0x6            
000226   7003     JNB	0x3, 0              
000227   ff11     INC	R1                  
000228   d708     CALL	#0x708             
000229   6503     CLR	0x3, 5              
00022a   31b7     ORL	0xb7, R0            
00022b   5084     MOV	R0, 0x84            
00022c   ff10     INC	R0                  
00022d   8071     ADD	R0, #0x71           
00022e   9906     MOV	R1, #0x6            
00022f   7003     JNB	0x3, 0              
000230   ff11     INC	R1                  
000231   d708     CALL	#0x708             
000232   6503     CLR	0x3, 5              
000233   31b8     ORL	0xb8, R0            
000234   c239     JMP	#0x239              
000235   5086     MOV	R0, 0x86            
000236   80c1     ADD	R0, #0xc1           
000237   9900     MOV	R1, #0              
000238   f748     ST	[R0], R1             
000239   c25c     JMP	#0x25c              
00023a   5086     MOV	R0, 0x86            
00023b   80f5     ADD	R0, #0xf5           
00023c   9906     MOV	R1, #0x6            
00023d   7003     JNB	0x3, 0              
00023e   ff11     INC	R1                  
00023f   d708     CALL	#0x708             
000240   6003     CLR	0x3, 0              
000241   ff18     RLC	R0                  
000242   6503     CLR	0x3, 5              
000243   5184     MOV	0x84, R0            
000244   8071     ADD	R0, #0x71           
000245   9906     MOV	R1, #0x6            
000246   7003     JNB	0x3, 0              
000247   ff11     INC	R1                  
000248   d708     CALL	#0x708             
000249   6503     CLR	0x3, 5              
00024a   51b7     MOV	0xb7, R0            
00024b   5084     MOV	R0, 0x84            
00024c   ff10     INC	R0                  
00024d   8071     ADD	R0, #0x71           
00024e   9906     MOV	R1, #0x6            
00024f   7003     JNB	0x3, 0              
000250   ff11     INC	R1                  
000251   d708     CALL	#0x708             
000252   6503     CLR	0x3, 5              
000253   51b8     MOV	0xb8, R0            
000254   9801     MOV	R0, #0x1            
000255   5191     MOV	0x91, R0            
000256   51b1     MOV	0xb1, R0            
000257   03b2     CLR	0xb2                
000258   5086     MOV	R0, 0x86            
000259   5190     MOV	0x90, R0            
00025a   98ff     MOV	R0, #0xff           
00025b   518f     MOV	0x8f, R0            
00025c   5086     MOV	R0, 0x86            
00025d   80c1     ADD	R0, #0xc1           
00025e   f701     LD	R1, [R0]             
00025f   ff11     INC	R1                  
000260   f748     ST	[R0], R1             
000261   c275     JMP	#0x275              
000262   5086     MOV	R0, 0x86            
000263   80c1     ADD	R0, #0xc1           
000264   5188     MOV	0x88, R0            
000265   5288     MOV	R1, 0x88            
000266   f708     LD	R0, [R1]             
000267   518d     MOV	0x8d, R0            
000268   9907     MOV	R1, #0x7            
000269   9812     MOV	R0, #0x12           
00026a   d70d     CALL	#0x70d             
00026b   6503     CLR	0x3, 5              
00026c   5188     MOV	0x88, R0            
00026d   0e88     MOVZ	R0, 0x88           
00026e   388d     SUB	R0, 0x8d            
00026f   7003     JNB	0x3, 0              
000270   c275     JMP	#0x275              
000271   5086     MOV	R0, 0x86            
000272   80c1     ADD	R0, #0xc1           
000273   9900     MOV	R1, #0              
000274   f748     ST	[R0], R1             
000275   6003     CLR	0x3, 0              
000276   13ad     RLC	0xad                
000277   13ae     RLC	0xae                
000278   0b86     INC	0x86                
000279   c00e     JMP	#0xe                
00027a   0382     CLR	0x82                
00027b   7992     JB	0x92, 1              
00027c   c287     JMP	#0x287              
00027d   9813     MOV	R0, #0x13           
00027e   9907     MOV	R1, #0x7            
00027f   d708     CALL	#0x708             
000280   6503     CLR	0x3, 5              
000281   0b93     INC	0x93                
000282   5293     MOV	R1, 0x93            
000283   f841     SUB	R1, R0              
000284   7003     JNB	0x3, 0              
000285   c287     JMP	#0x287              
000286   6192     CLR	0x92, 1             
000287   9907     MOV	R1, #0x7            
000288   980b     MOV	R0, #0xb            
000289   d70d     CALL	#0x70d             
00028a   6503     CLR	0x3, 5              
00028b   5188     MOV	0x88, R0            
00028c   9907     MOV	R1, #0x7            
00028d   980c     MOV	R0, #0xc            
00028e   d70d     CALL	#0x70d             
00028f   6503     CLR	0x3, 5              
000290   518d     MOV	0x8d, R0            
000291   0e88     MOVZ	R0, 0x88           
000292   308d     ORL	R0, 0x8d            
000293   7203     JNB	0x3, 2              
000294   c2d7     JMP	#0x2d7              
000295   0eb7     MOVZ	R0, 0xb7           
000296   30b8     ORL	R0, 0xb8            
000297   7203     JNB	0x3, 2              
000298   c2d7     JMP	#0x2d7              
000299   0bb3     INC	0xb3                
00029a   7a03     JB	0x3, 2               
00029b   c29d     JMP	#0x29d              
00029c   0bb4     INC	0xb4                
00029d   980b     MOV	R0, #0xb            
00029e   9907     MOV	R1, #0x7            
00029f   d708     CALL	#0x708             
0002a0   6503     CLR	0x3, 5              
0002a1   18b3     XOR	R0, 0xb3            
0002a2   7a03     JB	0x3, 2               
0002a3   c2d7     JMP	#0x2d7              
0002a4   980c     MOV	R0, #0xc            
0002a5   9907     MOV	R1, #0x7            
0002a6   d708     CALL	#0x708             
0002a7   6503     CLR	0x3, 5              
0002a8   18b4     XOR	R0, 0xb4            
0002a9   7a03     JB	0x3, 2               
0002aa   c2d7     JMP	#0x2d7              
0002ab   03b7     CLR	0xb7                
0002ac   03b8     CLR	0xb8                
0002ad   5091     MOV	R0, 0x91            
0002ae   a802     XOR	R0, #0x2            
0002af   7a03     JB	0x3, 2               
0002b0   c2c0     JMP	#0x2c0              
0002b1   508f     MOV	R0, 0x8f            
0002b2   6003     CLR	0x3, 0              
0002b3   ff18     RLC	R0                  
0002b4   5184     MOV	0x84, R0            
0002b5   80ee     ADD	R0, #0xee           
0002b6   f701     LD	R1, [R0]             
0002b7   5084     MOV	R0, 0x84            
0002b8   80de     ADD	R0, #0xde           
0002b9   f748     ST	[R0], R1             
0002ba   5084     MOV	R0, 0x84            
0002bb   80ef     ADD	R0, #0xef           
0002bc   f701     LD	R1, [R0]             
0002bd   5084     MOV	R0, 0x84            
0002be   80df     ADD	R0, #0xdf           
0002bf   f748     ST	[R0], R1             
0002c0   5090     MOV	R0, 0x90            
0002c1   6003     CLR	0x3, 0              
0002c2   ff18     RLC	R0                  
0002c3   5184     MOV	0x84, R0            
0002c4   80ee     ADD	R0, #0xee           
0002c5   f701     LD	R1, [R0]             
0002c6   5084     MOV	R0, 0x84            
0002c7   80de     ADD	R0, #0xde           
0002c8   f748     ST	[R0], R1             
0002c9   5084     MOV	R0, 0x84            
0002ca   80ef     ADD	R0, #0xef           
0002cb   f701     LD	R1, [R0]             
0002cc   5084     MOV	R0, 0x84            
0002cd   80df     ADD	R0, #0xdf           
0002ce   f748     ST	[R0], R1             
0002cf   0391     CLR	0x91                
0002d0   98ff     MOV	R0, #0xff           
0002d1   5190     MOV	0x90, R0            
0002d2   518f     MOV	0x8f, R0            
0002d3   03b1     CLR	0xb1                
0002d4   03b2     CLR	0xb2                
0002d5   03b3     CLR	0xb3                
0002d6   03b4     CLR	0xb4                
0002d7   0008     CRET                    
                                           func.__KF8S_Init_Touch_General_
000621   6503     CLR	0x3, 5              
000622   0384     CLR	0x84                
000623   6092     CLR	0x92, 0             
000624   6192     CLR	0x92, 1             
000625   03af     CLR	0xaf                
000626   03b0     CLR	0xb0                
000627   03a2     CLR	0xa2                
000628   03b7     CLR	0xb7                
000629   03b8     CLR	0xb8                
00062a   0384     CLR	0x84                
00062b   6f2c     SET	0x2c, 7             
00062c   670c     CLR	0xc, 7              
00062d   7e92     JB	0x92, 6              
00062e   c633     JMP	#0x633              
00062f   9890     MOV	R0, #0x90           
000630   5153     MOV	0x53, R0            
000631   0350     CLR	0x50                
000632   c63b     JMP	#0x63b              
000633   682c     SET	0x2c, 0             
000634   600c     CLR	0xc, 0              
000635   030f     CLR	0xf                 
000636   030e     CLR	0xe                 
000637   9801     MOV	R0, #0x1            
000638   5110     MOV	0x10, R0            
000639   9880     MOV	R0, #0x80           
00063a   5153     MOV	0x53, R0            
00063b   98f5     MOV	R0, #0xf5           
00063c   9906     MOV	R1, #0x6            
00063d   d708     CALL	#0x708             
00063e   6503     CLR	0x3, 5              
00063f   3153     ORL	0x53, R0            
000640   9802     MOV	R0, #0x2            
000641   ff58     DECJZ	R0                
000642   c641     JMP	#0x641              
000643   6e53     SET	0x53, 6             
000644   0000     NOP                     
000645   7e53     JB	0x53, 6              
000646   c643     JMP	#0x643              
000647   7453     JNB	0x53, 4             
000648   035f     CLR	0x5f                
000649   6e0b     SET	0xb, 6              
00064a   6f0b     SET	0xb, 7              
00064b   0008     CRET                    
                                           func.__KF8_lib_Baihualv_get_
0005a4   6503     CLR	0x3, 5              
0005a5   50a9     MOV	R0, 0xa9            
0005a6   39ab     SUB	0xab, R0            
0005a7   52aa     MOV	R1, 0xaa            
0005a8   7803     JB	0x3, 0               
0005a9   ff11     INC	R1                  
0005aa   3bac     SUB	0xac, R1            
0005ab   7803     JB	0x3, 0               
0005ac   c5ae     JMP	#0x5ae              
0005ad   c5b5     JMP	#0x5b5              
0005ae   6492     CLR	0x92, 4             
0005af   05ab     CPL	0xab                
0005b0   05ac     CPL	0xac                
0005b1   0bab     INC	0xab                
0005b2   7203     JNB	0x3, 2              
0005b3   0bac     INC	0xac                
0005b4   c5b6     JMP	#0x5b6              
0005b5   6c92     SET	0x92, 4             
0005b6   50ac     MOV	R0, 0xac            
0005b7   88fc     AND	R0, #0xfc           
0005b8   7a03     JB	0x3, 2               
0005b9   c5d0     JMP	#0x5d0              
0005ba   9806     MOV	R0, #0x6            
0005bb   ff10     INC	R0                  
0005bc   c5c0     JMP	#0x5c0              
0005bd   6003     CLR	0x3, 0              
0005be   13ab     RLC	0xab                
0005bf   13ac     RLC	0xac                
0005c0   ff58     DECJZ	R0                
0005c1   c5bd     JMP	#0x5bd              
0005c2   9808     MOV	R0, #0x8            
0005c3   21a9     ADD	0xa9, R0            
0005c4   7803     JB	0x3, 0               
0005c5   c5c7     JMP	#0x5c7              
0005c6   0baa     INC	0xaa                
0005c7   9804     MOV	R0, #0x4            
0005c8   ff10     INC	R0                  
0005c9   c5cd     JMP	#0x5cd              
0005ca   6003     CLR	0x3, 0              
0005cb   11aa     RRC	0xaa                
0005cc   11a9     RRC	0xa9                
0005cd   ff58     DECJZ	R0                
0005ce   c5ca     JMP	#0x5ca              
0005cf   c5de     JMP	#0x5de              
0005d0   6003     CLR	0x3, 0              
0005d1   13ab     RLC	0xab                
0005d2   13ac     RLC	0xac                
0005d3   6003     CLR	0x3, 0              
0005d4   13ab     RLC	0xab                
0005d5   13ac     RLC	0xac                
0005d6   9880     MOV	R0, #0x80           
0005d7   21a9     ADD	0xa9, R0            
0005d8   7803     JB	0x3, 0               
0005d9   c5db     JMP	#0x5db              
0005da   0baa     INC	0xaa                
0005db   50aa     MOV	R0, 0xaa            
0005dc   51a9     MOV	0xa9, R0            
0005dd   03aa     CLR	0xaa                
0005de   0383     CLR	0x83                
0005df   50a9     MOV	R0, 0xa9            
0005e0   39ab     SUB	0xab, R0            
0005e1   52aa     MOV	R1, 0xaa            
0005e2   7803     JB	0x3, 0               
0005e3   ff11     INC	R1                  
0005e4   3bac     SUB	0xac, R1            
0005e5   7803     JB	0x3, 0               
0005e6   c5e8     JMP	#0x5e8              
0005e7   c5e9     JMP	#0x5e9              
0005e8   c5ef     JMP	#0x5ef              
0005e9   0b83     INC	0x83                
0005ea   5083     MOV	R0, 0x83            
0005eb   a07e     SUB	R0, #0x7e           
0005ec   7803     JB	0x3, 0               
0005ed   c5ef     JMP	#0x5ef              
0005ee   c5df     JMP	#0x5df              
0005ef   7c92     JB	0x92, 4              
0005f0   c5f3     JMP	#0x5f3              
0005f1   0583     CPL	0x83                
0005f2   0b83     INC	0x83                
0005f3   0008     CRET                    
                                           func.__R2PCHPCL
000708   530a     MOV	0xa, R1             
000709   5102     MOV	0x2, R0             
00070a   0008     CRET                    
                                           .cinit
000691   6503     CLR	0x3, 5              
000692   9880     MOV	R0, #0x80           
000693   997e     MOV	R1, #0x7e           
000694   0000     NOP                     
000695   d6a8     CALL	#0x6a8             
000696   6d03     SET	0x3, 5              
000697   0380     CLR	0x80                
000698   0381     CLR	0x81                
000699   0382     CLR	0x82                
00069a   0383     CLR	0x83                
00069b   0384     CLR	0x84                
00069c   0385     CLR	0x85                
00069d   0386     CLR	0x86                
00069e   0387     CLR	0x87                
00069f   0388     CLR	0x88                
0006a0   0389     CLR	0x89                
0006a1   038a     CLR	0x8a                
0006a2   038b     CLR	0x8b                
0006a3   038c     CLR	0x8c                
0006a4   038d     CLR	0x8d                
0006a5   038e     CLR	0x8e                
0006a6   038f     CLR	0x8f                
0006a7   0008     CRET                    
0006a8   020a     CLR	R2                  
0006a9   f750     ST	[R0], R2             
0006aa   ff10     INC	R0                  
0006ab   ff59     DECJZ	R1                
0006ac   c6a9     JMP	#0x6a9              
0006ad   0008     CRET                    
